:100000000C947B100C949A100C949A100C949A10E7
:100010000C940A2A0C949A100C949A100C943F2B6E
:100020000C949A100C949A100C949A100C949A10A8
:100030000C949A100C949A100C949A100C949A1098
:100040000C949A100C949A100C949A100C949A1088
:100050000C949A100C949A100C94032F0C949A10F0
:100060000C949A100C949A100C949A100C949A1068
:100070000C949A100C949A100C949A100C943724A7
:100080000C949A100C949A100C949A100C949A1048
:100090000C949A100C949A100C949A100C949A1038
:1000A0000C949A105645523A323430383237004068
:1000B000140B16D81525160A134016EE11CA15F69C
:1000C000118312A720F015EE11EE11B0216B14EE82
:1000D000110B16D81525160A1340165E15CA15AD54
:1000E000148312A720F0155812EE11B0216B14EEF4
:1000F000110B16D81525160A1340162313CA15F925
:10010000128312A720F0155E12EE11B0216B14EECF
:10011000110B16D81525160A1340168513CA15FC9F
:10012000128312A720F015BA15EE11B0216B141826
:10013000120B16D81525160A134016EE11CA150013
:10014000138312A720F0156714EE11B0216B141859
:10015000120B16D81525160A1340164C12CA1599FB
:10016000148312A720F0157316EE11B0216B14182A
:10017000120B16D81525160A1340165212CA15DC92
:10018000148312A720F015F811EE11B0216B14188A
:1001900012EE11EE11EE110A13EE115816EE1109BE
:1001A000128312A720EE11EE11EE11B021EE11EE26
:1001B000110B16D81525160A134016EE11CA150F85
:1001C000148312A720F0150A14EE11B0216B14EE5F
:1001D000110B16D81525160A134016B912CA154167
:1001E000148312A720F0156412EE11B0216B14EEE7
:1001F000110B16D81525160A134016C112CA15453B
:10020000148312A720F015EE11EE11B0216B14EE3D
:10021000110B16D81525160A134016C612CA15A7B3
:10022000108312A720F0152E15EE11B0216B14EEDD
:10023000110B16D81525160A134016EE11CA159C77
:10024000108312A720F0154914EE11B0216B14EEA3
:10025000110B16D81525160A1340168E12CA15232F
:10026000158312A720F0159516EE11B0216B14EE30
:10027000110B16D81525160A1340169A12CA1568BE
:10028000168312A720F0159F15EE11B0216B14EE06
:10029000118B1280151A140A13DF12A512EB12EF3C
:1002A000118312A720EE117512EE11B021EE119CF0
:1002B000ACCCB6F400C111214191A131B171F19CD6
:1002C000ACCCB6F4367491A1C111214131F1714425
:1002D0004547000055534552000052414400005329
:1002E0004849465400005052474D0000414C504888
:1002F000410000C0C1C2FFC4C5C618808182C3844A
:100300008586877071728374757677303132733475
:1003100035363710111213141516170304050A0881
:10032000060BFF0209070D010C00FF53554E004D4F
:100330004F4E00545545005745440054485500461B
:1003400052490053415400004A414E004645420084
:100350004D415200415052004D4159004A554E0006
:100360004A554C0041554700534550004F435400F7
:100370004E4F5600444543000000030205000305AC
:100380000104060204464B3A3A494A483A3A3A3A94
:100390003A4C4F3A3A3A3A3A3A3A3A3A3A3A3A3A96
:1003A0003A3A4D3A3A300000300000300000200068
:1003B00000300418355D80300C902000083BAEBC46
:1003C000359D9C318C9C2AAAA83BAEBC359D9C31A6
:1003D0008C9C2AAAA8300018355580300090200047
:1003E00008300418355D8030009020000830001877
:1003F0003555803000002000000057C007FFC402C0
:10040000FFC000028000FFC005FFD402FFE0002E05
:10041000000001F41557F82D100002800030000094
:1004200030000030000020000007FFF40B503C05B6
:100430007FF40A00283FFFFC000F00157D402AAA28
:10044000800007FC00783C07897C280028003C00DD
:10045000557D55AABEAA003C00000000555555AA7E
:10046000BEAA003C003FFFFC30000C30000C300006
:100470000C3FFFFC31554C32AA8C30000C3FFFFC86
:1004800031554C32AA8C33FFCC30000C30000C308C
:10049000000C35555C31554C32AA8C30000C35556A
:1004A0005C31554C32AA8C33FFCC35555C2AFFA801
:1004B000000000000000000000000000555400AAE9
:1004C000BC00003C00003C00557C00AAA8000000D5
:1004D00000003C00003D55002AAA0000000000007A
:1004E000001555003EAA003C00003C00003C000006
:1004F0003C00003C00003C00557C00AABC00003CD5
:100500000001414403C7E007E3C0228280003C00B1
:10051000003D55003EAA003C00003C00557D55AA18
:10052000AAAA000000000000000000000000000077
:10053000000000003FFF3C0000000000003FC00042
:100540000000001540002A800017D7D42BEBE83FAD
:10055000FFFC02828007F4D01F7DF40F3DF0020AF9
:10056000803C0078001E8007A0142800281F47F454
:100570003C343C2F8AF80002080000001440002A96
:10058000000000000007FFD03E00BC200008000073
:100590000034001C2F55F802AA80000000024C60B5
:1005A000017F50006E40020820003C0003FFC000A5
:1005B0003C000000000000000003D8000000000024
:1005C00000003C00003C00003C000028000000004F
:1005D0000000F0000000000000000078001E80070E
:1005E000A0002800001FFFF43C1E3C3DF57C0AAA39
:1005F000A005003C3FFFFC00003C0000001F01FC88
:100600003C1FBC3DF83C0A80281F00F43C143C3DD4
:100610007D7C0A82A0007F00078F003FFFFC000A5C
:10062000003FF0F43CF03C3CF57C282AA01FFFF48E
:100630003C3C3C3C3D7C280AA03C00003C1FFC3D6F
:10064000F8002A80001FD7F43C3C3C3D7D7C0A82A8
:10065000A01FF4F43C3C3C3D7D7C0AAAA0000000B5
:10066000014140028280000000000000014144027C
:1006700082A0000000001D0001E2D00E002C00004E
:100680000001414003C3C003C3C0000000040004D4
:100690000B407800B7800008001F00003C1F3C3D65
:1006A00078000A800006AAA431AA4C24AA4C02AA07
:1006B0000007FFFC3E0F002F5F5402AAA83FFFFC7B
:1006C0003C3C3C3D7D7C0A82A01FFFF43E00BC3DCB
:1006D000007C0A00A03FFFFC3C003C2F55F802AA1A
:1006E000803FFFFC3C3C3C3C283C2800283FFFFC72
:1006F0003C3C003C28002800001FFFF43C003C3C30
:100700000F7C080AA03FFFFC003C00157D542AAA7C
:10071000A83C003C3FFFFC3C003C0000001400F4FF
:100720003C003C3FFFF82800003FFFFC003C001766
:10073000C3D42800283FFFFC00003C00003C000020
:10074000283FFFFC0B40001F55542AAAA82FFFFC8E
:1007500002D000157D542AAAA81FFFF43C003C3D9E
:10076000557C0AAAA03FFFFC3C3C003D7C000AA04F
:10077000001FFFF43C053C3D57FC0AAAA03FFFFCCC
:100780003C3D003D7EF40AA0281FF4343C3C3C3C38
:100790003D7C080AA03C00003FFFFC3C000000003C
:1007A000003FFFF400003C15557C2AAAA03FFF4003
:1007B0000000B41555E02AAA003FFFF80007801595
:1007C00057D02AAAA83D417C02BE8017EBD428004E
:1007D000283FD400003FFC3FE8000000003C01FC43
:1007E0003C1E3C3DE03C2A00281555543EAABC3C2A
:1007F000003C0000002D000002B400000AD0000000
:10080000281400143C003C3FFFFC00000001E00005
:100810001E00000B400000A00000003C00003C0057
:10082000003C0000282D000002D000000000000065
:10083000000051F400F33C00F774002AA83FFFFCCD
:1008400000F03C00F57C002AA0007FF400F03C00A2
:10085000F03C002020007FF400FC3C157D7C2AAA9F
:10086000A8007FF400F33C00F73C002A20057D54EB
:100870003EBEA83D28000A0000007D1400F33C00A5
:10088000F77C002AA03FFFFC00780000F554002A06
:10089000A80050003CFFFC0000000000000000F435
:1008A00000503C3CFFF80000000FFFFC0007D000A8
:1008B000382C0000081400003FFFFC00000000007E
:1008C0000000FFFC002D00007D5400AAA800BFFC22
:1008D00000F80000BD54002AA8007FF400F03C009E
:1008E000F57C002AA000FFFC007AD000F5F0002A79
:1008F00080007FD000F0F0007FD400AAA800FFFCA9
:1009000000780000F400002800007D3C00F33C006B
:10091000F37C00A0A015F5502AFABC00007C000072
:10092000A000FFF400003C00557C00AAA000FF409E
:100930000000B40055E000AA0000FFFC0001E00048
:1009400055F400AAA800F47C002BA0007EF400A0BF
:100950002800FD14000F3C005F7C00AAA000F07C82
:1009600000F3BC00FE3C00A028000000057D503ACA
:1009700082AC000000000000555555AAAAAA00004C
:100980000000000035415C0ABEA00000003F41FCB1
:100990003CBE3C3D007C2A00A83FFFFC003C000020
:1009A0003C00002800005FFF07A0057807FEF03E2E
:1009B00000F03FFFBD2AAA0AF555FFD400502B4096
:1009C000BFC2F007C0BCFF007CABC0A05F80001FAF
:1009D000FFFFFFFFFFFF800FFF000FFF400FFFFF34
:1009E000FF2FFFFFFFFFFCFFFFFCF00000F0000007
:1009F000F00000FFFFFCFFFFFCFFFFFFFFFFFFFF1A
:100A0000003FFF003FFF407FFFFFFF2FFFE0FFFFA2
:100A1000FCFFFFFCC003FCC003FCD007FCFFFFFC95
:100A2000BFFFE01FFFFFFFFFFFFF8000FF0000FF91
:100A30004000FFF0002FF000FFFFD0FFFFFC000B95
:100A4000FC0003FC0007FC00FFFC00FFE0FFFFFFD1
:100A5000FFFFFFFF0000FF0000FF40003FFFFF0A15
:100A6000FFFFFFFFFCFFFFFC0003FC0003FC00078F
:100A7000FCFFFFF0FFFE80FFFFFFFFFFFFFF003FD7
:100A8000FF003FFF003FFF0000FF0000FFFFFCFFF3
:100A9000FFFCC003FCC003FCC003FC0003FC00031C
:100AA000FCFFFFFFFFFFFFFF003FFF003FFF002AAB
:100AB000FF0000FF0000FFFFFCFFFFFCC00000C0C4
:100AC00000008000000000000000001FFFFFFFFF8B
:100AD000FFFF8000FF0000FF4000FFF0002FF0004C
:100AE000FFFFD0FFFFFC000BFC0003FCFF07FCFF37
:100AF000FFFCFFFFE0FFFFFFFFFFFF00003F0000E4
:100B00003F00003FFFFFFFFFFFFFFFFFFCFFFFFC79
:100B1000C00000C00000C00000FFFFFCFFFFFCFFA2
:100B20000000FF0000FF5555FFFFFFFFAAAAFF00CE
:100B300000FF00000003FC0003FC5557FCFFFFFC16
:100B4000AAABFC0003FC0003FC000000000000FF57
:100B50000000FF0000FFFFFFFFFFFFFF000000FF9E
:100B6000D000FFFC000BFC0007FCFFFFFCFFFFE0D8
:100B7000000000FFFFFFFFFFFF00003F0001FF003C
:100B80001FF8FFFF80FFF800FFFFFCFFFFFCD00015
:100B900000FD0000BFD0000BFFFC00BFFCFFFFFF0B
:100BA000FFFFFF0000000000000000000000000048
:100BB0000000FFFFFCFFFFFC0003FC0003FC000340
:100BC000FC0003FC0003FCFFFFFFFFFFFF0AFF50D8
:100BD000000FFF05FFA0FFFFFFFFFFFFFFFFFCFF70
:100BE000FFFC000000000000000000FFFFFCFFFF12
:100BF000FCFFFFFFFFFFFF2BFF50002BFF00002B30
:100C0000FFFFFFFFFFFFFFFFFCFFFFFC00000050A6
:100C10000000FF5000FFFFFCFFFFFC1FFFFFFFFF76
:100C2000FFFF8000FF0000FF4000FFFFFF2FFFFFDE
:100C3000FFFFD0FFFFFC000BFC0003FC0007FCFFE4
:100C4000FFFCFFFFE0FFFFFFFFFFFFFF003FFF0094
:100C50003FFF407FFFFFFF2FFFFEFFFFFCFFFFFC7A
:100C6000C00000C00000C00000C00000000000176D
:100C7000FFFF7FFFFFFF8000FF0000FF4000BFFF7E
:100C8000FF2BFFFFFFFF50FFFFF0000BFC0FF6FCF8
:100C90000AFF6CFDBFF4FFDBFCFFFFFFFFFFFFFF60
:100CA000003FFF003FFF407FFFFFFF2FFFFEFFFFE2
:100CB000FCFFFFFCFF0000FFD000EFFD00C2FFFCC7
:100CC000002FFC17FFF57FFFFFFF80BFFF003FFFF6
:100CD000403FBFF02F2BF00A003F50403FF4C00BC5
:100CE000FCC003FCD007FCFFFFF8FFFFA0FF0000E3
:100CF000FF0000FF5555FFFFFFFFAAAAFF0000FFFE
:100D00000000000000000000555554FFFFFCAAAA97
:100D1000A8000000000000FFFFFFFFFFFF00000031
:100D2000000000000000FFFFFFFFFFFFFFFF50FF7C
:100D3000FFF4000BFC0003FC0007FCFFFFF8FFFFC3
:100D4000A0FFFFFFFFFFFF00000000000000000009
:100D5000FFFFFFFFFFFFFFD000FFFD0000BFD0003F
:100D60000FFC007FE0FFFE00FFE000FFFFFFFFFF42
:100D7000FF000000000000000000FFFFFFFFFFFF7A
:100D8000FFFFFCFFFFFC017FA03FF00002BF50FF10
:100D9000FFFCFFFFFCFF5000FFFF5000AFFF000013
:100DA0003F005FFFFFFFA0FFA0000017FC17FFFC44
:100DB000FFE800F00000FFD4002BFFFC002BFCFF3D
:100DC000FFD0FFFFFD0000BF00000F00007FFFFF0E
:100DD000FEFFFFE0000000000000D55554FFFFFCBF
:100DE000EAAAA8000000000000FF0000FF0000FFCA
:100DF0000007FF007FFF07FFFFFFFEFFFFE007FF89
:100E0000FC7FFFFCFFE3FCFE03FCE003FC0003FCB3
:100E10000003FCFFFFFFFFFFFFFF0000FF0000FFDC
:100E20000000FF0000FF0000FFFFFCFFFFFC0003CD
:100E3000FC0003FC0003FC0003FC0003FC140000A6
:100E40003FD4002BFFD4002BFF00002B000000003C
:100E50000000000000000000000000D40000FFD4EB
:100E6000002BFFC0002BC0FF0000FF0000FF0000B0
:100E7000FF0000FF0000FFFFFFFFFFFF0003FC007B
:100E800003FC0003FC0003FC0003FCFFFFFCFFFF6E
:100E9000FC001F0001FF001FFFFFFFFFFF2FFFFFF0
:100EA00002FF00002F00000000000000FFFFFCFF19
:100EB000FFFCFFFFFC00000000000000000000003D
:100EC0000000000000000000000000000000000022
:100ED0000003FC0003FC0003FC0003FC0003FC0017
:100EE00003FC0003FC000000000000000000000004
:100EF00000000000000000000000000000000000F2
:100F000000000000000000000000000000000000E1
:100F10000000000000555555FFFFFFAAAAAA0000D7
:100F200000000000000000000000554154FFC3FC19
:100F3000AA82A8000000000000555500FFFF00AA8B
:100F4000AA00000000000000FFFF00FFFF000000FB
:100F50000000000000000000000000000000000091
:100F6000000000000FF00FFFFF0FFFFF000FF00F5A
:100F7000FFFF0FFFFF000FF03FC000FFFFC0FFFFAC
:100F8000C03FC000FFFFC0FFFFC03FC0000055547E
:100F900007FFFF0FE02FFFFFFFAFEAAF0FF40F02D5
:100FA000FC0200540040FF40C02FC0FFFFFCEAAF2E
:100FB000E8F57FC0FFFE0001540003FC0002A80119
:100FC00000017F017FFE3FFE803E80000001400166
:100FD0007FC07FFE80FE800080000003FC0003FCD9
:100FE0000000000101551F1FFFFF3E03FF3FDFE030
:100FF0000AFA00000003FFFD40EAAFF04002FCF5F2
:1010000000FCBFF5F802FFD0FFFAB0000000FFFFC0
:1010100000FFFF00000000000000000000000000D2
:1010200000000000000000000000000000000000C0
:1010300000000000000000000007FF01FFFF0FFAA2
:10104000007E0000A80000000000000000FF40003B
:10105000FFFD0002BFC00002F40000A80000000075
:101060000000F400003F40000BFD5500BFFF0002F0
:10107000AF00000000000000007C0007F055FF807A
:10108000FFF800EA0000000000003D0F000BDF0049
:1010900015FF003FFF002AFF0007EF003E0FF07C26
:1010A00000F7E000FF5400FFFC00FFA800FBD000A9
:1010B000F0BC0000000F00000F00155F003FFF00B4
:1010C0002AAF00000F00000FF00000F00000F55400
:1010D00000FFFC00FAA800F00000F000000000078C
:1010E00000000F00000F00005B0007CF01FA0F00A7
:1010F000000B400000C00000C00000940000CF4082
:1011000000C2BD0080000000000500000F00000FBD
:1011100000000F00000F00000F00000F500000F053
:101120000000F00000F00000F00000F00000F0000F
:101130000000000702F50F000BCF0000A700000F12
:1011400000000F00000B400000C17E00CF8000684F
:101150000000C00000C0000080000000000000008F
:101160000000000100017F017FFE3FFE803E800005
:10117000000140017FC07FFE80FE800080000000F3
:10118000000000000017FFFF7FFFFFFF8001FF004E
:101190001FFF41FFBFFFFF2BFFFFFFFF50FFFFF4CB
:1011A000FF8BFCF803FC8007FCFFFFF8FFFFA000AB
:1011B000000007FC007FFD55FFFFFFAAAAAA000060
:1011C000000000000003FC0003FC5557FCFFFFFC7F
:1011D000AAABFC0003FC0003FC1FF0007FF000FF43
:1011E0008000FF0001FF401FFFFFFF2FFFF8001FDF
:1011F000FC01FFFC1FFBFCFF83FCF803FC8003FCED
:101200000003FC1FF000FFF000FF8000FF003FFF25
:10121000407FFFFFFF2FFFE0003FD0003FFC000BAF
:10122000FCC003FCD007FCFFFFFCBFFFE000007F19
:101230000007FF007FF807FF807FFD55FFFFFFAA33
:10124000AAAAFF0000FF0000FF0000FF0000FF55FA
:1012500054FFFFFCFFAAA8FFFFFDFFFFFFFF00FFF9
:10126000FF00FFFF00FFFF00FFFF002F003FD00047
:101270003FFC000BFC0003FC4007FCFFFFFCFFFFF2
:10128000E01FFFFFFFFFFFFF807FFF00FFFF00FF6A
:10129000FF00FFAA002FFFFFD0FFFFFC800BFC0028
:1012A00003FC4007FCFFFFFCFFFFE0550000FF00D0
:1012B00000FF0000FF0001FF001FFFFFFFFFFFF81E
:1012C000000000000000155554FFFFFCFAAAA8809A
:1012D00000000000001FFFD0FFFFFFFF80BFFF00E6
:1012E0003FFF407FFFFFFF2FFFE27FFFD0FFFFFCAC
:1012F000E00BFCC003FCD007FCFFFFFCFFFFE01F7E
:10130000FFF5FFFFFFFF80BFFF003FFF407FFFFFB4
:10131000FF2FFFFF003FD0403FFCC00BFCC003FC91
:10132000C007FCFFFFFCFFFFE06FFFF9F4550FFC67
:101330000A8FFCFFF3FC054FFCAA0FE7FFF6BFFF87
:10134000E4C1547CCA80FC3FFCFCC540FCC2A8FC44
:101350007FFF6C00000700000F00000F00000B0073
:101360000000000000000000400000C01500C7E8B9
:10137000009E0000000000000000000000000007C8
:1013800000007F0007F8007F8007F8003F800038EA
:101390000000400000F40000BF40000BF40000BF5C
:1013A00040000BF00000B0000FF0000FF0000FF055
:1013B000000FF0000FF0000FF0000FF00FF0000F23
:1013C000F0000FF0000FF0000FF0000FF0000FF032
:1013D000003400003F40000BF40000BF40000BF45D
:1013E0000000BF00000B0000700007F0007F8007C6
:1013F000F8007F8000F8000080000017FC007FFCF0
:1014000000FF8001FF001FFF41FFBFFFF82BFF809F
:10141000000000000000555154FFF3FCAAA2A800F0
:1014200000000000002FFFF902AA8F00000F00004B
:101430000B000000000000000000BFFFE0CAAA008F
:10144000C00000800000000000000000000000005C
:101450000000003FC0003FC0003FC0003FD0003F41
:10146000FF000BFF1FFFD0FFFFFCFF8BFCFF03FC07
:10147000FF03F8FFFFFCFFFFFC0FFFFF0FFFFF0064
:10148000001F00003F00003F00003F00000BFFFF77
:10149000FCFFFFFCF80BFCC003FCD007FCFFFFFCCB
:1014A000FFFFE000007F0003FF0003FE0003FC00DD
:1014B00003FD0003FF0000BFFFFFD0FFFFFC000B98
:1014C000FC0003FC0007FC000FFC000FE000000123
:1014D00000001F00003F00003F00002F0FFFFF0F24
:1014E000FFFFFFFFD0FFFFFCE00BFCC003FCD007B9
:1014F000FCFFFFFCFFFFFC00007F0003FF0003FE7A
:101500000003FC0003FD0003FF0000BFFFFFD0FF4E
:10151000FFFC3FCBFC3FC3FC3FC3FCFFC3FCFFC34E
:10152000FC400000F40000FC0000FC0000FC000097
:10153000FC0000E0000000000000000000000000CF
:101540000000000000000000000000400000F40067
:1015500000FC0000FDFFF4FCAAA0FC0000E000007D
:10156000000000000000000000000000000000007B
:101570000000000000400000F40000FC0000FDFF3F
:10158000FDFCAAA8FC0000E000000000000015001F
:1015900007E800AA00000000000000000000004072
:1015A0000000F40000FC0000FDFFFDFCAAA8FC0008
:1015B00000E0000000000000150007E800AA00009D
:1015C000AF400002BD00000000400001F4000FFC2D
:1015D000000FFDFFF7FCAAA0FC0000E000000000E7
:1015E00000C01500C7E8002A0000AF400002BD009F
:1015F000000000400001F4000FFC000FFDFFF7FCAD
:10160000AAA7FC000FE0000B000000C01500C7E80F
:10161000002A00006F4000C2BD00800000000015DD
:1016200000003F00000000000500000F0000000067
:101630000000555550FFFEA000BF00555F00FFFFA2
:1016400000001600000000000FF0000FF0000FF087
:10165000000FF5000FFF15FFF03FAFF00FF5FC0F87
:10166000FFA85FF000FFF0000FF0000FF0000FF098
:1016700000FD4000FFFD40FC2BFDFC002FFD0002A3
:10168000FFC000FFC0000005FC05FFFCFFA0FCE060
:1016900000FC0001FC000FFC000FFC00000000003B
:1016A000000000000000070001FE007F800FE00046
:1016B0000001FC007FFC1FE0FCFF00FC0BD0FC00E5
:1016C000BFFC0000FC00000100000F00003F000014
:1016D0003F00003F00003F00003EF001F0C17FF0FE
:1016E000DFFA00E00550DFFFF0EA03F0000A000037
:1016F000000500007F0003FF0003F80003FD000168
:10170000FF0003FAFFFF40FFFFF0A00FF0001FE013
:1017100057FF50FFFFF0AA03F017FFFF3FEAAAFEB2
:101720000054FC00FCFF01FD3FFFFF0BFE8FFFFF9D
:10173000FFABFEAA00FF0000FF0001FF00FFFE005C
:10174000FFF80000000114001FFC007FFC00FCFDFE
:10175000403F3FFFFF0ABFFF5FF500FFFFF0800241
:10176000FC0003F8517FE0FFFE00EA8000001FD478
:1017700001FFFD07F82F0FF00F0FF00F0FF00A0217
:10178000FC001FFD00FFFFD0F00BF4E003FCC003E2
:10179000FC8003FC000FF000001500003F07FFFF76
:1017A0003FFFFFFE003FFC002ABF00000003FC01DA
:1017B0005FFCFFFFFCFEA3FC0003FC0003FC000336
:1017C000FC0000FC005FFF0FFEFE3F80FCFE00FC03
:1017D000FD00FC3F4000FC0000FFD400FEFFC0FC09
:1017E0000BF0FC02FCFC01FC0007E000001400010F
:1017F000F80013F007F3C0FE83F0A002FF00000A18
:101800000155001FFFD07E02FCFC00FCFC07E0FF3E
:10181000FFFCAAAAA800001F0001FE0173F05FE30D
:10182000F0F803F50000BF00000AFFFF40FEAFF430
:10183000FC02FCFC00FCFC01FCFC03F0A800000026
:1018400000500000F0007CF51FE0FF3E00000000AB
:10185000000000000000FC0000FC5555FCFFFFFCF0
:101860000000FC0000FC00000000005F0001FE0121
:10187000F3F05FA3F0F802FF00002B000000FFFD73
:1018800040AAAFF40002FC0001FC555FF8FFFE80A7
:101890000000000003FF0010AA45F0003F80002870
:1018A00001FF0002AA000000FFFFD0AAABFC00006D
:1018B000FC0005F8FFFFFCAAAAA800000000000039
:1018C00000000005FFFF3FFFFFFE00003C0000009E
:1018D000000000001F00003FFFFFFFFFFFE80000C7
:1018E00000000000000000001FE0003FC0003FD0EB
:1018F000000FF00003FC0003FC001FF07F8000FFDE
:101900000000FF00003FC0000FF0000FF0007F80DC
:10191000000000FF07F0FF0F007E0BD3F007F3FD80
:101920000F80FF00002FFFFFFCFFFFFC0000000006
:101930000000000000FFFFFCFFFFFC0017FF01FF9D
:10194000EA0FE8000FC0000FD40002FFD5002BFF04
:10195000FF50FCAFFDFC000BFC0000000007FC5F2B
:10196000FEFCFA80FC400000F40000FC0000FDFFDB
:10197000F4FCAAA0FC0000E0000000000000000051
:101980000000000000000000000000000000000057
:1019900000000003FC0003FC0003FC0003FD000347
:1019A000FF0000BF07FFD03FFFFC3F8BFC3F03FC65
:1019B0003F03F8FFFFFCFFFFFC0FFFFF0FFFFF00DF
:1019C000001F00003F00003F00003F00000BFFFF32
:1019D000FCFFFFFCF80BFCC003FCD007FCFFFFFC86
:1019E000FFFFE000000700003F00003F00003F0055
:1019F000003F00003F00000BFFFFD0FFFFFCE00BAB
:101A0000FCC003FCC003FCF00FFCF00FE000000181
:101A100000001F00003F00003F00002F0FFFFF0FDE
:101A2000FFFFFFFFD0FFFFFCE00BFCC003FCD00377
:101A3000FCFFFFFCFFFFFC00000100001F00003F57
:101A400000003F00003F00003F00000B555540FFE5
:101A5000FFF4EFEFFC0FC3FC4FC3FCFFC3FCFFC35D
:101A6000FC000003007FFF03FFFF03FE0303FD03F1
:101A700003FFC000BFC0FC0000FFFFFCFFFFFCFC39
:101A80000000FC000000000000000000007F0003D8
:101A9000FF0003FE0003FC0003FD0003FF0000BF86
:101AA000FD03F4FFC3FF2FC0BF0FC03F1FC07FFF68
:101AB000FFFFFFFFF803FFFF03FFFF000007000029
:101AC0000F00000F00000F000002FFFFFCFFFFFCF3
:101AD000F80000F00000F40000FFFFFCFFFFFC0036
:101AE000000000000000001500FF3F00FF3F000065
:101AF00000000000000000000000400000FFFFFCAC
:101B0000FFFFFC00000000000000000000000000DB
:101B1000000000000000001500FF3F00FF3F000331
:101B2000F40003FF0000BF00003F40007FFFFFFF05
:101B3000FFFFF800FFFF00FFFF00000000000100B2
:101B4000003F00003E000000FFFFFCFFFFFC1FF411
:101B500000FEBF40E00BFC0000BC000000000000E5
:101B6000000000000000003FFF003FFF00000000F9
:101B70000000000000000000000000FFFFFCFFFF6D
:101B8000FC00000000000000000700003F00003FD4
:101B900000000F00003F00003F00000BFFFFFCFAB9
:101BA000AAA8D40000FFC000E80000F55554FFFFCC
:101BB000FC00003F00003F00001F00003F00003F0E
:101BC00000003F00000BFFFFFCFFFFFCE00000C037
:101BD0000000C00000FFFFFCFFFFFC00000700004A
:101BE0003F00003F00003F00003F00003F00000BAF
:101BF000FFFFD0FFFFFCE00BFCC003FCD007FCFFA5
:101C0000FFFCFFFFE0003FFF003FFF0007FE000F6B
:101C1000F0000FF4000FFF0002FFFFFFFCFFFFFCCE
:101C200002FD0000FF0001FF00FFFF00FFF80000C1
:101C3000007F0007FF000FF8000FF0000BF4003FDB
:101C4000FF003FFFFFF400FFFF0002FF0000FF0066
:101C500001FE00FFFFFCFFFFFC00003F00003F0013
:101C6000000700003F00003F00003F00000BFFFFA7
:101C7000FCFFFFFCFE0000E00000D00000FC0000C4
:101C8000FC000000001F0000FF0000FE0000FC0040
:101C900000FC0000FF0000BFFD0FD0FFCFFC2FC2F3
:101CA000FC0FC0FC0FD1FC0FFFFC02FFE0000003A3
:101CB00001555703FFFF02AAAB000003000000001C
:101CC0000000FC0000FD5540FFFFF4FEABFCFC01F2
:101CD000FC003FFC003FE000003F00003F00000030
:101CE00000000000000000003F00003FFFFFD0FFA9
:101CF000FFFC000BFC0003FC0007FCFFFFFCFFFFE8
:101D0000E000003F00003F00000000000000000075
:101D100000003F00003FFFD000FFFD0002FFD000A9
:101D20003FFC01FFE0FFFE00FFE00000003F00007D
:101D30002A00000000000000000000001500003F25
:101D4000FFFFD0AAAFFC0007FC03FFF0000BFC551F
:101D50005FFCFFFFE000003F00002B0000000000E0
:101D60000000000000001700003F4001FCF41FE8E5
:101D7000BFFE000FF0007FFD00F82FD48002FC00B2
:101D8000003F00003F0000000000000000150000C0
:101D90003F00003FFD03F4FFC3FC2FC0BC1FC03C4D
:101DA000FF807CFFFFFCFFFFF800003F00003F00CA
:101DB000003F00003F00003F00003F00003FC00127
:101DC000FCC01FFCC1FFFCDFFFFCFFE3FCFE03FCCB
:101DD000E003FC00000000000301400F7FFFFFFE56
:101DE000AAA8F00000A00000000000C00000F00160
:101DF00040FFFFFD2AAABF00000F00000A000000FC
:101E0000000000555555FFFFFFAAAAAA00000000D8
:101E10000000000000000000555554FFFFFCAAAA76
:101E2000A8000000000000000000F00000FC00001E
:101E3000FFFFFD2BEAAF00000300000200000000DE
:101E4000000F00001F1FFFFFFAABE8E0000080005A
:101E500000FD4000FFFD40FC2BFDFC002FFD0002BB
:101E6000FFC000FFC0000005FC05FFFCFFA0FCE078
:101E700000FC0001FC000FFC000FFC1FFFFFFFFF38
:101E8000FFFF800FFF000FFF400FFFFFFF2FFFFF3F
:101E9000FFFFD0FFFFFCC00BFCC003FCC007FCFF32
:101EA000FFFCFFFFE0000000000000000000000059
:101EB0000000000000000000000000000000000022
:101EC0000001540003FC0002A80550000FF0000AB6
:101ED000A000000550000FF0000AA0000000000064
:101EE00000000000001547003FFE002AA00101018C
:101EF000FF02EB0202D76802D10102C0F607C12837
:101F0000282828140005C20606060602CB0802B3DC
:101F1000940BB4E56685FFFF5285FFFF5202B03F88
:101F200003B20005011101FF03C7A6E90236200232
:101F30003A1102B809012001FF02B9230138012931
:101F400000010101FF02EB0202D76802D10102C0C9
:101F50008007C128282828140005C20000000002BC
:101F6000CB1702B3940BB4A566010000400100003A
:101F70004002B03F03B20105011101FF03C7A6E90A
:101F8000023620023A1102B8090120012902B9E300
:101F900001FF02B923013900010101FF02EB020236
:101FA000D76802D10102C08007C128282828140060
:101FB00005C20000000002CB170BB4E577F1FFFF6C
:101FC0004FF1FFFF4F02B064011101FF03C7A6E903
:101FD000023620023A1102B80902D01F012001295D
:101FE00002B9E301FF02B923027200013900425530
:101FF000494C543A20417567203237203230323410
:102000002031303A35333A353000534E3A00564598
:10201000523A20302E393031004241543A004E417C
:102020004D4520202020506720426B0050582D3411
:1020300031435800426174742E20456D7074793AB2
:10204000004465626F756E636520542E3A004B65DF
:102050007920204379636C65733A0044697370207A
:102060004379636C65733A0052756E20204379633F
:102070006C65733A00726573746F72696E672E2EA9
:102080002E002D20202D00202D2D2D2D20005349F8
:102090005A453A004D454E552000444953502000C2
:1020A000424545502000434F4D20200053504545A8
:1020B0004400494E464F2000534C45455000564978
:1020C000455720004D4F52452000524547532000B0
:1020D000464C414753004D4F445320004144562045
:1020E0002000524F4D532000434F4E462000532EA8
:1020F000494D4700000011241FBECFEFCDBFDFE7E1
:10210000DEBF10E4A0E0B0E4E4E9FBE700E00BBFD1
:1021100002C007900D92A639B107D9F72EE6A6E9BD
:10212000B0E401C01D92A03FB207E1F70E94FB3A64
:102130000C94C83D0C94000090913B6E81E0982770
:1021400090933B6E809307408093064008951092D1
:102150003B6E81E08093074080930540809306406A
:10216000089581E08093EF6E1092FC421092FD4240
:102170008093C85DE3EBF2E411921586138E11A6ED
:1021800017AA82E4E13CF807B9F7109208431092CD
:10219000094310920A4310920C4310920D4310927F
:1021A000BE5D1092BF5D1092F9421092FA421092F9
:1021B000FB4280E180930B431092EE5D1092C35D71
:1021C00008958091FB42813019F089EF92E40895DF
:1021D0008AEF92E408958031910508F0C097E3EB0F
:1021E000F2E427E0289FB001299F700D112490E0B0
:1021F00080E0DC01A60FB71FA25FBC4B258D30E14C
:10220000239FA0011124248D242B2C930196329618
:102210008730910571F70895CF93DF93DC01EB01CF
:102220003EE049914D933A95E1F7DF91CF910895C2
:10223000CF93DF93342FDC01EB01231BA30FB11DE0
:10224000C30FD11D49914D932A95E2F7DF91CF91AC
:102250000895242FDC01261BA60FB11D1D922A957F
:10226000EAF70895CF93DF93342FDC01EB01231BB2
:10227000A30FB11DC30FD11D4C9158815D9349939C
:102280002A95D2F7DF91CF910895CF93DF93DC01A8
:10229000022E000C330B51E0E42FF0E02E173F0725
:1022A0001CF4DF91CF91089580E06115710521F054
:1022B000EB01CE0FDF1F8881EA0FFB1F9081C091D9
:1022C000C85D9C0F980F908380910B43981730F056
:1022D000981B90835093C85D4F5FDECF1092C85D0E
:1022E000FBCF0F93FC0131E0021714F40F91089516
:1022F00090E06115710531F0DB01A20FB11D27FDE2
:10230000BA959C9180E04115510531F0DA01A20F98
:10231000B11D27FDBA958C91981B8091C85D981BC3
:1023200097FF0FC080910B43980F3093C85D309793
:1023300031F0DF01A20FB11D27FDBA959C932F5FED
:10234000D3CF1092C85DF3CFCF93DF93242FEC014E
:10235000C60FD11D261B498149932A95E2F71A928F
:10236000DF91CF910895CF93DF93DC011092C85D88
:102370002417A4F0E42F042E000CFF0B90E061154D
:10238000710521F0EB01CE0FDF1F9881EA0FFB1FD3
:102390008081891731F081E08093C85DDF91CF9112
:1023A00008954F5FE5CFA0E0B3E48D919C91119724
:1023B000E2E0F3E4208131812D933C93A4E0B3E487
:1023C0002D913C91119720833183E6E0F3E4208145
:1023D00031812D933C9310821182089508950E94BB
:1023E000D3118093FC429093FD4208950C94D31135
:1023F0000E94D311E3EBF2E4292F22952F7022A340
:102400009F7091A3982F92959F7090A38F70878F44
:102410000895E3EBF2E482A1829591A1892B90A12A
:102420009295278D922BECEFF2E4908381830895AF
:102430008295837090E09C01220F331F2270959546
:102440008795822B9091FF42292F22952F7030E0A3
:1024500096E1929FF001939FF00D1124E355FF4BFD
:102460009589EDEAF0E444E0840290011124458965
:1024700049130CC0DF01A20FB31F4D915D916D9107
:102480007C91452B462B472B09F0848B769642E4B2
:10249000ED30F40761F708956FEC72E48DED92E48E
:1024A0000C940C116DED72E48FEC92E40C940C1111
:1024B0006FEC72E48BEE92E40C940C116BEE72E410
:1024C0008FEC92E40C940C11E3EBF2E4968D858D85
:1024D0008295807F248D822B8093EC5D9093ED5DBF
:1024E00010922642109227420895E3EBF2E4858D84
:1024F00020E1829FC0011124248D822B80932642EB
:1025000090932742089582958F708093C05D85E0F7
:102510008093EE5D089510920C430895E3EBF2E48E
:10252000858D90E1899F90011124848D822B809369
:102530000C430895E3EBF2E480910C43982F9F70D5
:10254000948F82958F70858F0895E3EBF2E4ACE071
:10255000B3E48C91958D40E1949F90011124948D6A
:10256000922B9C93982F9F70948F82958F70858F5C
:10257000089580910C4380930A4380EA8093070476
:10258000089580910A4380930C43089580910C43F1
:1025900090910A4390930C4380930A4380EA80937E
:1025A000070480910240811109C088ED9DE180936C
:1025B00003409093044081E08093024008950E947C
:1025C000E110FC019081911103C08DE0808308959A
:1025D0009150908308950E94E110FC0190819F5FCB
:1025E00090830E94E110FC0120812E3008F01082BF
:1025F00008951092FB42089581E08093FB42089574
:102600009091F9428091FA42981303C081E080933F
:10261000C85D0895CF93C82F0E94E110DC01EC91B2
:10262000F0E0ED54FD4BC295CF70C48F0E94E110D5
:10263000FC019081911104C08DE08083CF910895B9
:1026400091509083FBCFCF93DF930E94E110DC0188
:10265000EC91D0910943C0910843ED30B1F48091E1
:102660009740982F9F7B953B11F0873F49F4C0938B
:10267000DC42D0930843C0930943DF91CF91089582
:10268000D093DC42C093CF42F8CF809196408D30FA
:1026900079F580919740853F61F0982F9F70973032
:1026A00039F582958F70982F977F973009F18B308D
:1026B000F9F0D0930843C09309430E94E110DC0174
:1026C000EC91F0E0ED54FD4BC58F0E94E110DC0170
:1026D000EC91F0E0ED54FD4BD48F0E94E110DC0151
:1026E000EC91F0E0ED54FD4B858D8093CF42C5CF4A
:1026F000F0E0ED54FD4BD58F0E94E110DC01EC9130
:10270000F0E0ED54FD4BC48FB8CFCF93DF930E9420
:10271000E110DC018C91C09108438D3001F590915E
:1027200097408091DC42292F2F7B253B11F0973F6A
:1027300049F48093094380930843C093DC42DF91BE
:10274000CF910895909109432091CF42209308435F
:10275000809309439093DC42C093CF42F0CF209105
:102760009640D091094390E02D3099F52091974003
:10277000253F61F0322F3F70373059F522952F7089
:10278000322F377F373029F12B3019F18D549D4B83
:10279000FC01858D809309430E94E110DC01EC91DE
:1027A000F0E0ED54FD4B848D809308430E94E110CE
:1027B000FC019091CF42E081F0E0ED54FD4B958F0C
:1027C0000E94E110DC01EC91F0E0ED54FD4BD48F60
:1027D000C3CF8D549D4BFC01858D809309430E948E
:1027E000E110DC01EC91F0E0ED54FD4B848D809321
:1027F00008430E94E110DC01EC91F0E0ED54FD4B48
:10280000D58F0E94E110DC01EC91F0E0ED54FD4B1E
:10281000C48F95CF8091B2428093FC4208958091FD
:10282000B242E3EBF2E4982F92959F7090A38F70E1
:10283000878F089580913C6E90913D6E892B91F029
:1028400080913C6E90913D6E019780933C6E909389
:102850003D6E81E090912542911101C080E080930E
:10286000C85D08958091C35D823099F71092C35D71
:10287000109225421092B2428091A74290E0E5CF9B
:10288000089580E180930B4308958AE080930B4381
:102890000895E3EBF2E482A1829591A1892B90A1A6
:1028A0009295278D922B9093AB408093AC4082E021
:1028B0008093EE5D0895E3EBF2E4968F982F929566
:1028C0009F70958F8F70848F1092EE5D089583E0D6
:1028D0008093EE5D0895CF93DF93CDB7DEB72E974B
:1028E000CDBFDEBF82958F70E82FF0E0E55EFC4F34
:1028F000E491DE0111969E01215F3F4FBD0181E011
:102900008E0F0E2E000CFF0BED54FD4B948D9D93FE
:10291000E0E08E300CF4E82FA217B30781F78FECBC
:1029200092E40E940C112E96CDBFDEBFDF91CF91B5
:1029300008958091A9422AE0829FC001112420912C
:102940004B6E30914C6E8217930720F081E080939C
:10295000C85D08951092C85D089584E08093EE5D8F
:102960000895F8948091015E8823B9F0E091FF5DAD
:10297000F0E0E151F24A80819091FF5D9F5F90937A
:10298000FF5D9091FF5D9F709093FF5D9091015E60
:1029900091509093015E7894089580E0FCCF9091DF
:1029A000240895FFFCCF8093220808952EE0FC01B7
:1029B00011922A95E9F7089583EB92E40E94D614C8
:1029C00081EC92E40E94D6148FEC92E40C94D6141D
:1029D000EEE0F3E480EB9AE1DF019C011D922150CF
:1029E0003040E1F70895CF93DF93DC01FC013B9683
:1029F0006B3061F41B968C911B9792919183EA172F
:102A0000FB07D9F78083DF91CF9108958C91ED0179
:102A100099819993CE17DF07D9F71B968C93F3CF43
:102A20009C014097C09768F0211582E0380749F073
:102A3000C901805F9240419720F081E0203F334000
:102A400008F080E008958091B142882331F00E941F
:102A5000D3118093FC429093FD420895CF93DF936E
:102A60008091264290912742009731F08D3F910549
:102A700089F0DF91CF910895C091EC5DD091ED5D2B
:102A8000CE010E9410158823A1F3CE01DF91CF91D2
:102A90000C94EB102091D1428091D04230E1839F81
:102AA000C0011124922B2091CF42822B8093376E4C
:102AB0009093386E81E080930640DBCF0E94E11056
:102AC000DC01EC91ED30A1F4909197408091DC42D3
:102AD000292F2F7B253B11F0973F39F49091094323
:102AE000909308438093094308959091CF42F8CF83
:102AF000F0E0ED54FD4B848D80930843858DF2CF3B
:102B000080913C6E90913D6E892B51F080913C6E8E
:102B100090913D6E019780933C6E90933D6E089529
:102B20008091C35D8130D9F7809135428111F7CF13
:102B300082E08093C35D8091A74290E0ECCF8EE06D
:102B4000815078F48091B142882351F08091C15D29
:102B50008D3031F48091CF428093DC428093C0422B
:102B60000895E82FF0E0ED54FD4B948D20819223E1
:102B7000948FE6CFCF93DF93AFECB2E4CBEED2E409
:102B80003EE04C9158815D9349933A95D1F7DF919E
:102B9000CF910895CF9382958F70E82FF0E0E55E96
:102BA000FC4FC4910E94E110FC01C083CF910895B5
:102BB00082958F70E82FF0E0E55EFC4FE491ACE089
:102BC000B3E421E030E002C0220F331FEA95E2F7C0
:102BD0008D919C911197822B932B8D939C930895AB
:102BE0002091BE5D3091BF5D82958F70E82FF0E03F
:102BF000E55EFC4FE49181E090E002C0880F991FF0
:102C0000EA95E2F78223932321E0892B09F420E05F
:102C10002093C85D089582958F70E82FF0E0E55EFF
:102C2000FC4FE491ACE0B3E481E090E002C0880F97
:102C3000991FEA95E2F7809590952D913C91119717
:102C4000822393238D939C93089582958F70E82F10
:102C5000F0E0E55EFC4FE49181E090E002C0880F77
:102C6000991FEA95E2F720910C4330910D4382239E
:102C7000932321E0892B09F420E02093C85D089577
:102C8000CF93C82F0E94E110C295CF70EC2FF0E0D7
:102C9000E55EFC4FE491DC018C910E2E000CFF0BE5
:102CA0008E171F0619F481E08093C85DCF910895B7
:102CB000CF93DF93AFECB2E4CDEDD2E43EE04C91A4
:102CC00058815D9349933A95D1F7DF91CF9108955B
:102CD0008091B142811106C00E94D3118093FC42C1
:102CE0009093FD420895E3EBF2E482A1829591A1D5
:102CF000892B90A19295278D922BE4E0F3E420811B
:102D000031812093064330930743A2E0B3E42D9131
:102D10003C91119720833183E0E0F3E420813181FD
:102D20002D933C939083818308958EE0815078F4B5
:102D30008091B142882351F08091C15D8D3031F492
:102D40008091CF428093DC428093C0420895E82F67
:102D5000F0E0ED54FD4B948D2081922B948FE6CFC3
:102D6000E0E4F4E081818D608183E0E0F4E0818142
:102D700080648183E0E6F9E084E0818381E38083FD
:102D80000895809364098091630987FFFCCF0895BB
:102D90001F93CF93DF93C0E0D4E010E41E830E9422
:102DA000C1161D83DF91CF911F91089527E731E070
:102DB000829FF001839FF00D1124EE5FF14A20E025
:102DC000818192819695969530E4839FA00111248C
:102DD000942B928390818695869530E4939FA001F1
:102DE0001124842B81839695969590832F5F33963B
:102DF0002D3731F7089527E731E0829FF001839F57
:102E0000F00D1124EE5FF14A2DE781819081990F39
:102E1000990F382F3295369536953370932B9083D2
:102E20009281880F880F392F3295369536953370F9
:102E3000832B8183990F990F92832150339621110F
:102E4000E4CF0895E2E0FEE58DE190E1DF019C0131
:102E50001D9221503040E1F70895E2E0FEE59191A6
:102E6000DF01119798279C939EE6EF31F907B9F798
:102E70000895E2E0FEE59191DF01119798239C937C
:102E80009EE6EF31F907B9F7089527E731E0829F11
:102E9000F001839FF00D1124EE5FF14A9F01295844
:102EA0003E4F8191DF01119786238C93E217F30740
:102EB000C1F7089527E731E0829FF001839FF00D6D
:102EC0001124EE5FF14A629FD001639FB00D11247F
:102ED000AE5FB14ACF0189589E4F21912D93E817DB
:102EE000F907D9F7089570E027E731E0482F429FAE
:102EF000C001439F900D112447E751E08E5F914A36
:102F00000C94C13D0F931F93CF93DF93182F8AE248
:102F10000E94C816C9E1C10F8C2F0E94C1168C2FC8
:102F20000E94C1168BE20E94C81680E00E94C11662
:102F30008CE70E94C1168CE20E94C81687E791E0D8
:102F4000189FE001199FD00D1124CE5FD14A8E0148
:102F500009581E4F89910E94C116C017D107D1F799
:102F6000DF91CF911F910F910895CF93DF938AE264
:102F70000E94C81689E10E94C11683E20E94C11610
:102F80008BE20E94C81680E00E94C1168CE70E9466
:102F9000C1168CE20E94C816C2E0DEE589910E944B
:102FA000C1168EE6CF31D807C9F7DF91CF910895CA
:102FB000CF93DF938F773CE0839FC00111248B5523
:102FC0009C4FC62FC695E7E7F1E04E9FD0014F9F7B
:102FD000B00D1124AE5FB14A33E0C39FE00111246C
:102FE0008A1B9B0B60FF30C0AE014D5F5F4FCA0F65
:102FF000DB1FA40FB51F3CE0841B950BFC01EA0FFF
:10300000FB1F2636F1F0E491E22748814A7A488393
:103010004C9145754C93F0E0AF0155954795542F71
:1030200055754881452B4993EE0FFF1FEA7A4C9165
:10303000E42BED93315011F788E0860FDF91CF91AB
:103040000895E491E676E1CFAC0FBD1F3CE08C1B08
:103050009D0BFC01EA0FFB1F263641F0E491E227AD
:10306000EC93315011963111F4CFE6CFE491E6762E
:10307000F7CFFF920F931F93CF93DF938C01D42F41
:10308000F22EC0E0F801EC0FF11D8081811107C024
:10309000862FDF91CF911F910F91FF9008952F2DD3
:1030A0004D2F0E94D817682FCF5FECCFFF920F9360
:1030B0001F93CF93DF938C01D42FF22EC0E0F80141
:1030C000EC0FF11D8491811107C0862FDF91CF9104
:1030D0001F910F91FF9008952F2D4D2F0E94D8170B
:1030E000682FCF5FECCF5F926F927F928F929F920B
:1030F000AF92BF92CF92DF92EF92FF920F931F9306
:10310000CF93DF93CDB7DEB72597CDBFDEBF8983E1
:103110006A834B832C830D831092C45D1092C55D2E
:103120001092C65D41E35BE68091C45D9091C55D00
:10313000A091C65DFA0180839183A2839A01285BE6
:103140003F4FF90180839183A283455B5F4FFCE68B
:10315000483A5F0749F76AE089E00E945A17CE01B2
:1031600001967C0110E000E096E0692E22E3C22E79
:10317000D12C80E098E7A1E0BB27F70181907F0187
:10318000869C40011124092C000CAA08BB08880E5B
:10319000991EAA1EBB1EABBEF4017790B601F8E0E3
:1031A0007F9E60197109112477FF02C06F5F7F4F06
:1031B00075956795600F711F512C8FEF881A980ACB
:1031C000A80AB80A57101AC00E5C1F4F0A3F110513
:1031D00081F689E02596CDBFDEBFDF91CF911F91AB
:1031E0000F91FF90EF90DF90CF90BF90AF909F90A6
:1031F0008F907F906F905F900C94D616ABBEF401C9
:1032000087912FEF49E00E94D817682F5394D5CFAC
:1032100099E1899F802D112461E0282F260F30E04D
:10322000A901440F551F240F351F2E5F314AF901A4
:10323000E15DF24F9081492F440F440FD901A05D09
:10324000B24F9C919295969596959370942B9083FE
:103250009C91492F440F440F3296908192959695F8
:1032600096959370942B9C93408194E0499FA00184
:103270001124436040832A55314FF90110826F5F5A
:10328000683159F608952F923F924F925F926F9254
:103290007F928F929F92AF92BF92CF92DF92EF92E6
:1032A000FF920F931F93CF93DF9380E090E8A1E00C
:1032B000BB276C017D0128E7D20EE11CF11C0E94A6
:1032C000221730E020E087E7882E99249394A1E02C
:1032D000B0E05524539450E040E0289D3001299DF2
:1032E000700C389D700C112426C0EBBEF6011791AE
:1032F0008FEFC81AD80AE80AF80A90E0EBBEF60188
:103300008791EFEFCE1ADE0AEE0AFE0A980F092F18
:103310000095C92FC81B811111C015259A3F70F364
:10332000625071096E3F8FEF7807F9F64F5F5F4F7C
:103330004330510539F166E070E0D7CF113001F527
:10334000C695D0E0FE01EE0FFF1FEC0FFD1FE60D4E
:10335000F71DEE5FF14AE40FF51FC02FC80FC0FB49
:10336000AA24A0F8B12CE501C60FD71F1D0102C089
:10337000220C331CCA95E2F7E101D081CD2BC0832A
:103380008150C7CF2F5F3F4F2B30310509F0A3CFBE
:10339000DF91CF911F910F91FF90EF90DF90CF9031
:1033A000BF90AF909F908F907F906F905F904F9065
:1033B0003F902F900C94B517BF92CF92DF92EF926F
:1033C000FF920F931F93CF93DF93362F9AE2899F3B
:1033D000800111240B55164F83E0689F7001112462
:1033E000B0E0A0E085E1B82E50E097E7C92EDD24DB
:1033F000D3948A2FAA32B10561F487E0830FDF915D
:10340000CF911F910F91FF90EF90DF90CF90BF90E1
:103410000895FD01E00FF11FE4916B2D0E94733CB4
:10342000BA01680F711D6C9DE0016D9DD00D7C9DF2
:10343000D00D1124CE0DDF1DC90FD11DCE5FD14A95
:10344000E227E8831196D5CFCF92DF92EF92FF92D9
:103450000F931F93CF93DF93D62E92E1899FE001C4
:103460001124CB55D14E83E0689F8001112430E0B8
:1034700020E089E0C82E50E097E7E92EFF24F3947E
:10348000822F2231310559F483E08D0DDF91CF91E8
:103490001F910F91FF90EF90DF90CF900895F90169
:1034A000EC0FFD1FE4916C2D0E947F3CBA01680F68
:1034B000711D6E9DD0016F9DB00D7E9DB00D1124CC
:1034C000A00FB11FA90FB11DAE5FB14AEC932F5FE2
:1034D0003F4FD6CFCF93DF938AE20E94C81689E18F
:1034E0000E94C11683E20E94C1168BE20E94C81698
:1034F00080E00E94C1168CE70E94C1168CE20E94F7
:10350000C816CDE1D0E180E00E94C1162197D9F71D
:10351000DF91CF91089580E10C94C81681E10C945D
:10352000C816262F2150330BF901E758FC4FE491C0
:1035300091E0633008F090E0891B282F26952695AE
:10354000280F3327331F64E60E94733CB901681BC0
:103550007109CB018E0F911D840F911D67E070E002
:103560000E94A13C8F5F0895823021F4637081F442
:103570008DE108958150990B67E070E00E94A13CB5
:1035800062E070E00E94A13C9FE1981B892F0895A2
:103590008CE108958D3010F08C500895811101C098
:1035A0008CE00895CF93DF93DC01362F4423C1F0E4
:1035B0006A30B0F4E0E0222311F02C93E1E0ED0159
:1035C000CE0FD11D832F6AE00E94733C905D9883DB
:1035D000EF5FEA0FFB2FF11D1082DF91CF9108956D
:1035E000832F6AE00E94733C805D8C93E7CFFF924B
:1035F0000F931F93CF93DF93CDB7DEB72597CDBF42
:10360000DEBF0CE912E4D8015096EC91B4E0EB0275
:10361000F00111242FEF40E0682FCF01895D9C4F0E
:103620000E9456182FEF40E0682F8DE20E94D817B5
:10363000D8011796EC91B4E0EB02F00111242FEFC2
:1036400040E0682FCF018C5B9C4F0E9456182FEFF3
:1036500040E0682F8DE20E94D817F82EF8016085AF
:1036600020E041E0CE0101960E94D21A2FEF40E007
:103670006F2DCE0101960E9439182596CDBFDEBF71
:10368000DF91CF911F910F91FF9008951F93CF93DA
:10369000DF93CDB7DEB72597CDBFDEBF182F809162
:1036A0009E42813009F040C06091AB4220E241E08F
:1036B000CE0101960E94D21A2FEF40E0612FCE0179
:1036C00001960E9439182FEF40E0682F8AE30E948C
:1036D000D817182F6091A04220E040E0CE0101965B
:1036E0000E94D21A2FEF40E0612FCE0101960E9476
:1036F0003918682F80919E42813079F480919F42E1
:103700002FEF40E08C30ACF080E50E94D8172FEF0F
:1037100040E0682F8DE40E94D8172596CDBFDEBF0C
:10372000DF91CF911F91089560919F4220E240E088
:10373000BFCF81E4EACFCF93DF9310923B6E85E059
:1037400080939B42EFE9F0E4CFE3DEE6AEEDBDE52A
:10375000119219921D9280E4EB3AF807C9F7109282
:10376000376E1092386EDF91CF91089560E089E056
:103770000E9473178091376E80FF07C020E049E0F8
:1037800060ED8CEE92E00E9456188091376E81FFBA
:1037900007C020E049E06AEA86EE92E00E945618EF
:1037A0008091376E82FF06C020E049E06CE984E337
:1037B0000E94D8178091376E83FF06C020E049E051
:1037C00064E983E30E94D8178091376E84FF06C0B6
:1037D00020E049E06CE882E30E94D8178091376EC0
:1037E00085FF06C020E049E064E881E30E94D81725
:1037F0008091376E86FF06C020E049E06CE780E3E9
:103800000E94D8178091376E87FF07C020E049E0FB
:103810006EE48FED92E00E9456188091376E909181
:10382000386E90FF07C020E049E060E38AED92E047
:103830000E9456188091376E9091386E91FF06C0A5
:1038400020E049E068E287E40E94D8178091376E53
:103850009091386E92FF07C020E049E062E084ED6D
:1038600092E00E9456188091376E9091386E8827AA
:103870009370892B39F420E049E060E38FEC92E00B
:103880000E94561889E00E94D61689E00C9482178F
:103890000F931F93CF93DF9380913B6E882331F179
:1038A0000AEE1DE52FE33EE6CFE9D0E4EDE0F2E4D9
:1038B0006EED7DE5D9011B969C91D8018E918D010D
:1038C000B4E08B9FA0011124892F8370842B8295F3
:1038D000807F4B85840F868B96959695978B21508C
:1038E0003109219732976017710721F7DF91CF9146
:1038F0001F910F910895CF93DF9388E1EDE0F2E4FB
:10390000AFE1BEE601900D928A95E1F760E087E0B5
:103910000E94731760E088E00E947317CDE0D2E444
:1039200085E020E047E0682F8E890E94DC1947E09F
:10393000682F8F890E94241A229791E4C53FD907E6
:1039400081F78091376E9091386E83709927892B1B
:1039500031F420E048E061E088E50E94D81787E074
:103960000E94821788E0DF91CF910C948217EDE0DE
:10397000F2E4AFE1BEE691918D91981306C082E426
:10398000E432F807C1F781E0089580E00895DC0192
:103990001596FB0135963E912291321305C0A8176A
:1039A000B907C9F781E0089580E00895FC0110820D
:1039B00011821282138214820895DC011596FB0194
:1039C00035963E912291231728F0321728F0A81738
:1039D000B907B9F781E0089580E008956F927F926A
:1039E0008F929F92AF92BF92CF92DF92EF92FF920F
:1039F0000F931F93CF93DF938B01DB011D921D92D9
:103A00001D921C921397EC0122963C01BEE06B0EB6
:103A1000711CC12CD12C7601C394A991B0E0A701EF
:103A200096010E94E73CF80180809180A280B380DB
:103A3000DC01CB01880D991DAA1DBB1D80839183DC
:103A4000A283B383AAE0B0E00E94E73C6B017C0153
:103A50006C167D0611F7DF91CF911F910F91FF90AA
:103A6000EF90DF90CF90BF90AF909F908F907F901E
:103A70006F900895AC0190E070E0292F092E000CA2
:103A8000330B261737070CF00895240F351FF90163
:103A900010829F5FF2CF4F925F926F927F928F92D0
:103AA0009F92AF92BF92CF92DF92EF92FF92CF930D
:103AB000DF9300D000D0CDB7DEB7F894BE016F5FC2
:103AC0007F4F87E492E40E94EE1C7894C980DA80EC
:103AD000EB80FC808CE3882E912CA12CB12CC701AB
:103AE000B601A50194010E94B53C6093A142CA01B0
:103AF000B901A50194010E94B53C6093A042C701A1
:103B0000B60120E13EE040E050E00E94B53CCA0131
:103B1000B90128E130E040E050E00E94B53C6093FC
:103B20009F4280919F420E94CA1A8093AB42C70174
:103B3000B60120E831E541E050E00E94B53C690162
:103B40007A01C982DA82EB82FC82CA01B9016C5522
:103B50007C498F4F9F4F22E0660F771F881F991F68
:103B60002A95D1F721EB3AE342E050E00E94B53CC0
:103B7000215F3F4F4F4F5F4F82EAC80E8FEDD81E37
:103B800084E2E81EF11CC20ED31EE41EF51E62E0A4
:103B900056954795379527956A95D1F7C21AD30A56
:103BA000E40AF50AA4E1B0E0A70196010E94E73C0F
:103BB0002B013C012AE8421A29E0520A61087108E7
:103BC000C301B20129E83CE140E050E00E94B53C6D
:103BD00049015A01ADE6B1E00E94E73CC61AD70A96
:103BE000E80AF90AC301B20124E232E740E050E0FA
:103BF0000E94B53CC21AD30AE40AF50AA8EEB3E063
:103C0000A70196010E94E73C29E837E740E050E031
:103C10000E94B53C29013A018EE1289FC018112469
:103C2000A9E5B2E00E94E73C28EE33E040E050E036
:103C30000E94B53CC21AC092A4422EE04216510422
:103C40006104710480F58CE6881A82E1980AA10863
:103C5000B10821E0421A51086108710880E3880E1A
:103C60008092A2424092A3424091A4426091A3421A
:103C70008091A2420E94911A8093AC4281E080938D
:103C80009B402496CDBFDEBFDF91CF91FF90EF9098
:103C9000DF90CF90BF90AF909F908F907F906F906C
:103CA0005F904F9008958BE6881A82E1980AA108E8
:103CB000B1082DE0421A510861087108CFCF2F9248
:103CC0003F924F925F926F927F928F929F92AF92AC
:103CD000BF92CF92DF92EF92FF920F931F93CF93F9
:103CE000DF93CDB7DEB72997CDBFDEBFC090A2422C
:103CF0000C2C000CDD0820E3C21A28EFD20A0D2C90
:103D0000000CEE08FF083091A342232E022C000C79
:103D1000330829823A8291012330310548F4245F27
:103D20003F4F29833A8331E0C31AD108E108F108F3
:103D30001091A442ADE6B1E0A70196010E94E73CD4
:103D40004601570122E0B694A794979487942A9548
:103D5000D1F7860E971EA81EB91EC701B60120E92D
:103D600031E040E050E00E94B53C820E931EA41E5C
:103D7000B51EC701B60124E630E040E050E00E94E5
:103D8000B53C821A930AA40AB50A29813A812F5FA9
:103D90003F4FC901880F991F820F931F65E070E0A4
:103DA0000E948D3C2EE129803A80229DC001239DF6
:103DB000900D1124810F911D17FD9A95FB01E80FBD
:103DC000F91F9F0150E040E060E070E0CB01E98323
:103DD0003A834B835C836D837E838F8398879401C2
:103DE000A50160E070E080E090E0A980BA80C12C7D
:103DF000D12CE12CF12C00E010E00E94A93D2A5EBC
:103E000036494A4051096109710981099109E0E87F
:103E1000AE2EF1E5BF2ECC24C3940E94F23C590192
:103E20006A017B018C01A0919F424091A042409089
:103E3000A1420A2E000CBB0B20E13EE00E94E03CB8
:103E4000042C000C550866087708DC01CB01840DB2
:103E5000951DA61DB71D3CE34302A0011124840F4C
:103E6000951FA11DB11D1C012D01612C712C430159
:103E70003A82AB835C826D827E828F8298869C01BF
:103E8000AD0160E070E080E090E00E94A93D290172
:103E90004A01698779831C01F8941092C75DA9E4EF
:103EA0006A2EA2E47A2E8AE0A82EB12CC12CD12C45
:103EB000E12CF12C00E010E09201A40169857981E8
:103EC000C1010E944A3DF30121933F019201A401E7
:103ED00069857981C1010E944C3D29014A016987A8
:103EE00079831C0125E532E426153705E1F667E400
:103EF00072E48FE792E40E940C1178942996CDBF6A
:103F0000DEBFDF91CF911F910F91FF90EF90DF9077
:103F1000CF90BF90AF909F908F907F906F905F9069
:103F20004F903F902F900895FC0195E020E0819103
:103F3000980FDF0111979A3060F49C9390E0211163
:103F400001C09E5F2F5F2E3011F09111F0CF892FAD
:103F500008959A509C9391E0F2CFCF93803108F06E
:103F60004AC0E82FF0E0E954F04E0C94D73CC71F4C
:103F7000D41FEC1FFD1F35204020FB1F56205C2066
:103F80006F208020882090209820A020A42080915D
:103F900046422EE0829FC00111246FEC72E4895BDF
:103FA0009D4BCF910C940C1180914642CEE08C9F9A
:103FB000C00111246FEC72E4895B9D4B0E940C11CF
:103FC000E0914642CE9FF0011124EA5CFD4B118A3C
:103FD000128ACF910C944B1D809146422EE0829F15
:103FE000C00111246FEC72E48D599D4B0E940C119D
:103FF00081E080939B40CF9108958091464281114A
:1040000026C0909136422091D04280E1289F9001B5
:1040100011248091CF42806C822B89238093364279
:10402000809136428F7339F78091BE5D9091BF5D6C
:104030009F7D8093BE5D9093BF5D8091BE5D9091AA
:10404000BF5D9F7E8093BE5D9093BF5DD4CF23E024
:1040500040E060ED72E488E392E40E9418118091E0
:104060003B42817080933B42C6CF809146422EE016
:10407000829FC00111246FEC72E481589D4B91CF57
:1040800024E040E06FEC72E481E492E40E941811B5
:104090008CE392E40E94D61C809136429091374284
:1040A00094608093364290933742A5CF80913642F8
:1040B000909137429B7FF5CF4091364250913742E5
:1040C00020914642255F81E090E002C0880F991F51
:1040D0002A95E2F78095909584239523E2CF40912D
:1040E00036425091374220914642255F81E090E070
:1040F00002C0880F991F2A95E2F7842B952BD1CF08
:10410000409136425091374220914642285FDBCFA2
:10411000409136425091374220914642285FE6CF87
:104120004091364250913742209146422A5FCBCF90
:104130004091364250913742209146422A5FD6CF75
:1041400081E08093464257CF1092464254CF7F92EF
:104150008F929F92AF92BF92CF92DF92EF92FF9297
:104160000F931F93CF93DF93082F02950F70C02FEB
:10417000D0E0E090EC5DF090ED5D20EFE22223E0F6
:10418000F222E02AFD2AE092EC5DF092ED5DC7019B
:104190000E941015182F882381F0C701DF91CF915D
:1041A0001F910F91FF90EF90DF90CF90BF90AF9055
:1041B0009F908F907F900C94EB108091264290916D
:1041C00027428B3F910509F469C08D3F910541F568
:1041D000C154DD4FFE01C49180E0C7FD8BE0FC2F90
:1041E000FF709F2E00E02C2F2071822EDBE0D81B69
:1041F00090E0FC01E156FF4B7F01FC2FF0727F2E17
:104200009C01215C31496901C074FC01E252F24A0F
:104210005F01901213C081E08093074080930540B6
:10422000DF91CF911F910F91FF90EF90DF90CF9092
:10423000BF90AF909F908F907F900895882069F0F5
:104240006D2F8FE990E40E94F314E12FF0E0ED541C
:10425000FD4B848DF70180831F5F772069F06D2F00
:104260008FE39EE60E94F314E12FF0E0ED54FD4B46
:10427000848DF60180831F5FCC2371F06D2F8EED4E
:104280009DE50E94F314E12FF0E0ED54FD4B848D89
:104290008170F50180831F5F0F5FBBCF802FDF919F
:1042A000CF911F910F91FF90EF90DF90CF90BF9033
:1042B000AF909F908F907F900C94AD1F8230A1F0B3
:1042C00038F08430E9F1C8F0853009F442C008952F
:1042D000609146428EE0689FB0011124695B7D4B7E
:1042E0008FEC92E40C940C11609146428EE0689F32
:1042F000B00111246D597D4BF3CF8091464281115D
:1043000017C0809136428F708093CF4280913642A1
:1043100082958F708093D042809137428F708093C6
:10432000D14280913742829581708093D242089524
:1043300023E040E068E372E480ED92E40C9418110D
:10434000609146428EE0689FB001112461587D4B18
:10435000C7CF24E040E061E472E48FEC92E4EECF5A
:104360006F927F928F929F92AF92BF92CF92DF9285
:10437000EF92FF920F931F93CF93DF93182F129515
:104380001F708FEC92E40E94D61480912642909187
:1043900027428B3F910509F4B9C08D3F910509F47F
:1043A00040C0892B79F5112359F08091EC5D9091F3
:1043B000ED5D807F9370812B8093EC5D9093ED5D3C
:1043C0000091EC5D1091ED5DC8010E9410158823ED
:1043D000C9F00031110510F00053110987E0809FEA
:1043E000E001819FD00D1124C25FDC4BAFECB2E441
:1043F00067E04991542F52955F704F704D935D93D4
:104400006A95B9F7DF91CF911F910F91FF90EF90CF
:10441000DF90CF90BF90AF909F908F907F906F90E4
:104420000895153001F58091376E9091386E909314
:10443000D1429C0194E0369527959A95E1F72F702B
:104440002093D0428F708093CF4280913B6E88231F
:10445000C9F21330B8F21530A9F281E08093074019
:1044600080930540CFCFE12FF0E0E155FD4FC4919F
:104470000BE0C7FF00E02C2F2F70822ED0E0912C94
:104480003C2F3071732E802F90E0DC01A156BF4B82
:104490007D01BC2FB0726B2E9C01215C31496901FA
:1044A000C074DC01A252B24A5D01891471F2772016
:1044B00069F0ED2FF0E0ED54FD4BD7018C91848F26
:1044C000DF5F602F8FE990E40E94F314662069F0AB
:1044D000ED2FF0E0ED54FD4BD6018C91848FDF5F22
:1044E000602F8FE39EE60E94F314CC2369F0ED2F3A
:1044F000F0E0ED54FD4BD5018C91848FDF5F602F90
:104500008EED9DE50E94F3149394CFCF812FDF9120
:10451000CF911F910F91FF90EF90DF90CF90BF90C0
:10452000AF909F908F907F906F900C945E216EE083
:1045300087E492E40E943A1D6EE083E692E40E94D2
:104540003A1D6EE08FE792E40E943A1D6EE085E529
:1045500092E40E943A1D6EE081E792E40E943A1DC7
:104560006EE08DE892E40E943A1D64E088E392E4F4
:104570000E943A1D8CE392E40E94D61CE6E3F2E42A
:10458000108A808191818064808391838081918170
:104590009160808391834AE050E069E070E084E7B5
:1045A00092E40E94C13D80E280938E420C945F1E93
:1045B0008F929F92AF92BF92CF92DF92EF92FF9233
:1045C0000F931F93CF93DF93EDEAF0E480E691E041
:1045D000DF019C011D9221503040E1F7EDE4FEE641
:1045E00082EADF011D928A95E9F7C0E0D8EFDF018A
:1045F00040E096E1992E56E0A12C24E1B22E8824C9
:104600008394FE01049131962491319684913196E0
:10461000E49111960C93119716962C931697179672
:104620008C9317971896EC931897003108F04DC0AB
:1046300010E030E0909EF001919EF00D1124BF013A
:1046400063557F4B7B01620F731FFB01408BF701AA
:10465000858B842F652F0E94733C9A9D60019B9DE2
:10466000D00C11240D2C000CEE08FF08813009F449
:104670003FC0823009F441C060E070E880E09927D3
:10468000C60ED71EE81EF91E1296CD92DD92ED924F
:10469000FC9215974630C8F48C92F901EE0FFF1F7B
:1046A000EE0FFF1F909E9001919E300D1124E20F9E
:1046B000F31FE355FF4B12960D911D912D913C91E7
:1046C000159700831183228333834F5F24961996B5
:1046D000423109F096CFDF91CF911F910F91FF905A
:1046E000EF90DF90CF90BF90AF909F908F90089504
:1046F00060E070E081E09927C3CF60E070E881E07E
:104700009927BECFE62FE69527E0AC01249FC00194
:10471000259F900D11248D549D4BE80FF92FF11D0D
:10472000E55AFF4F808160FD82958F700895CF928A
:10473000DF92EF92FF929C01892F992782958F70CB
:1047400066E1689FA001699F500D1124FA01E355AD
:10475000FF4B948984E0989FF0011124E40FF51F2A
:10476000E355FF4BC080D180E280F38080E090E091
:10477000C114D104E104F10449F1C9019F70B701EA
:10478000A601480F591F611D711D6BBFFA01A7914A
:10479000AC01569547955695479570E060E0505F9F
:1047A0006F4F7F4F4C0D5D1D6E1D7F1D6BBFFA015E
:1047B000479150E0880F991F8670992702C0559540
:1047C00047958A95E2F78A2F942F9370FF90EF9088
:1047D000DF90CF9008958091015E8823E1F30E94DD
:1047E000B11490ED980F9A3030F09FE9980F963001
:1047F00020F499EA980F892F08959FEB980F96302F
:1048000010F499ECF7CF803231F390E0F4CF8A3393
:1048100010F08755089580530895F894EFEEFDE564
:10482000108A118A128A78940895F8949091015E02
:104830009031B1F0E091005EF0E0E151F24A808306
:104840008091005E8F5F8093005E8091005E80317A
:1048500010F01092005E8091015E8F5F8093015E88
:10486000789408958091240886FFFCCF08951F92C4
:104870000F920FB60F9211240BB60F928F93EF93F6
:10488000FF93E091005EF0E080912008E151F24A50
:1048900080838091005E8F5F8093005E8091005ED8
:1048A0008F708093005E8091015E8F3028F480913C
:1048B000015E8F5F8093015EFF91EF918F910F906A
:1048C0000BBE0F900FBE0F901F9018950F931F9364
:1048D000CF93DF93EC018C01FE0101900020E9F7FA
:1048E0003197EC1BFD0BC8018C1B9D0B8E179F078E
:1048F00028F0DF91CF911F910F910895F8018191D8
:104900008F010E94CF14E8CF813408F0875F8F7049
:10491000089547E0489F9001499F300D11242D5480
:104920003D4BBC016C5F7F4F8617970710F080E00E
:10493000089550E040E0FA01E55AFF4FE20FF31FFF
:10494000E081E11109C04F5F5F4F4730510599F792
:104950000196295F3F4FE8CF81E0089597E0899F56
:10496000B001112430E020E0A901460F571FFA01E1
:10497000E753F24A425F5C4BDA019C9190832F5FD0
:104980003F4F2730310581F7089527E0829FC0010E
:10499000112430E020E0A901480F591FFA01E75324
:1049A000F24A425F5C4B6081FA014081641307C0A8
:1049B0002F5F3F4F2730310571F781E0089580E088
:1049C0000895FB016AE00E94733C905D928381111F
:1049D00007C080E2818380E280838383148208950C
:1049E000805DF8CFCF93DF93EC01FB016AE070E0CC
:1049F0000E948D3C9B01805D82836A30710590F03E
:104A0000CE0164E670E00E948D3C605D6083C90168
:104A10006AE070E00E948D3C805D81831382DF91AB
:104A2000CF9108954083672B91F74183F7CFCF93C0
:104A3000DF93EC01FB016AE070E00E948D3C9B017A
:104A4000805D83836A30710570F0CE0164E670E0AA
:104A50000E948D3C605D6083C9016AE070E00E9445
:104A60008D3C805D04C080E38083672BA9F782833F
:104A70008EE2818386E584831582DF91CF9108954C
:104A800081E08093000624E090E080E031E0309304
:104A90000A0640910D0640FFFCCF40911006509150
:104AA0001106840F951F215091F79695879596953D
:104AB00087956AE070E00E948D3C059710F06F5F6B
:104AC0007F4F10920006CB010895262F30E0082E6C
:104AD000000C990BB9010E94A13C820F931FB901F0
:104AE0000E94A13C0895E62FE69527E0829FC00131
:104AF00011248D549D4BE80FF92FF11DE55AFF4FFE
:104B0000808160FD82958F70089527E0289FD001F5
:104B1000299FB00D112430E020E0F901EA0FFB1FBE
:104B2000E25FFC4B9081492F4F70FB0140839295CF
:104B30009F7091832F5F3F4F6E5F7F4F273031050E
:104B400061F708958F929F92BF92CF92DF92EF927A
:104B5000FF920F931F93CF93DF93CDB7DEB7689784
:104B6000CDBFDEBFD42E8E010F5F1F4FAE01435F5E
:104B70005F4F780120E2D7012D937D011B961C9297
:104B80001B974A175B07B9F7382F4C0120E072E0FA
:104B9000CC24C39483E0B82E882D831B8617D8F4C9
:104BA000D401ED914D01822F90E0E7FD54C0E03635
:104BB00018F4E03488F1E054800F911FDC01EC938D
:104BC000F4018081982F9D7F9C3219F08A3309F07F
:104BD00040C02C3008F385E020E04D2D682FD8012F
:104BE0008D918D010E94DC194D2D682FF801838570
:104BF0000E94241A0E151F0579F76896CDBFDEBFF7
:104C0000DF91CF911F910F91FF90EF90DF90CF90A8
:104C1000BF909F908F900895E03238F0EA3349F4C6
:104C2000840F951FDC017C9314C0F0E0EB57FC4F20
:104C3000E491EE3251F0EA3B99F3EC3209F0BCCF4B
:104C4000840F951FFC01B08204C0840F951FFC01E6
:104C5000C0822F5FBECFEAE3AFCF4F925F926F92D9
:104C60007F928F929F92AF92BF92CF92DF92EF92FC
:104C7000FF920F931F93CF93DF93CDB7DEB7A69725
:104C8000CDBFDEBF8C014B018430910510F40E9432
:104C9000AE24BE016F5F7F4F7B013E017DE0670E5A
:104CA000711C570180E2D5018D935D011B961C920A
:104CB0001B97A615B705B9F787E0809F9001819FE4
:104CC000300D1124F901EC5EFC4B8081803109F03C
:104CD00089C085E090E0682FF901E80FF91FE25FD5
:104CE000FC4B4081411103C00197A8F76FEF6F5F44
:104CF00090E0462F50E087E0809FD001819FB00D6B
:104D00001124AD54BD4B292F092E000C330B241751
:104D10003507FCF00430110508F045C0402F440F62
:104D20004F5FCE0149960E94A225A696CDBFDEBF59
:104D3000DF91CF911F910F91FF90EF90DF90CF9077
:104D4000BF90AF909F908F907F906F905F904F90AB
:104D50000895FA01E21BF30BEA0FFB1FE65AFF4F1F
:104D6000808187FD1EC0803280F48823C1F07EEFF1
:104D7000780F7230B0F079EF780F753090F072EFF5
:104D8000780F7F3070F08E3160F4E9E1F0E0EC0FE5
:104D9000FD1F2E0F3F1FF90180839F5FB4CF8AE074
:104DA000F4CF82E0F2CF8BE0D4018C9380E21196B5
:104DB0008C9320E0822F022E000C990BFC0132967E
:104DC000E80DF91D8417950714F01082AECF69E144
:104DD00070E06C0F7D1F860F971FDC018C91808324
:104DE0002F5FE8CF6E01B9E1CB0ED11CB601C8012F
:104DF0000E9485255090734341E0A3E04A2E53FC66
:104E000003C043E0442443949091714392959C7075
:104E1000A0917243AF705A2F898D2A8DF82FEAE046
:104E20002E9FF00D11242F2F3B8D3323F9F034E604
:104E30003F1B232F31E09830D9F4E22F022E000CD3
:104E4000FF0B6A2F70E06F5F7F4F6E177F070CF4C8
:104E50005AC031E0E617F70721F49DA131E0953003
:104E600018F098E02A3024F090E002C09830C9F39E
:104E70006EA1662311F06DE26983943009F4D4C009
:104E8000983009F442C0911121C1332311F08DE211
:104E90008A87822F6AE00E947F3C90E3980F9B876D
:104EA00090E3920FF6EF8F9F900D11249C874E8711
:104EB000A83008F0B6C0F601EA1BF109A1E083852D
:104EC000853008F4A0E0B1E0B50F6DE070E08B2F05
:104ED0000B2E000C990BFB01E81BF90BEC0DFD1DD3
:104EE000E081EA0FA0E0EA3010F0E0E0A1E08E0DF2
:104EF0009F1DF0E37F2E7E0EFC017082B15039F7CA
:104F00002111EAC039C031E0AFCF313009F04EC0D5
:104F1000AF5F8A2F821BF601E81BF10987FDF3952D
:104F200051E08485853008F450E01EA2022E000C6A
:104F3000330B8DE090E06701C20ED31E6A2F0A2E5C
:104F4000000C770BFB01E21BF30BF7FD0BC0FC0120
:104F5000E61BF70BEC0DFD1DE08DE50F50E0EA3090
:104F600010F051E0E0E06E0D7F1DB0E3BE0FFB01DD
:104F7000B083A15019F74E870430110508F0DCC04A
:104F8000000F0F5F85E020E0402F682FF70181912F
:104F90007F010E94DC19402F682FD7011B968C914E
:104FA0000E94241AAE14BF0471F7BFCE8F5F8A0F20
:104FB0008A3034F551E0F601E81BF10987FDF395DD
:104FC0009485953008F450E0082E000C990BF601FA
:104FD000E81BF90B3D961816B4F0E1E0E20FE60D80
:104FE000F72DF11D4083225052FEC6CF121624F633
:104FF000F301E20FF11D27FDFA9540822350F6CF11
:10500000532F8AE0E1CF6191650F532F6A3010F082
:10501000632F51E0D701A80FB91F605D6C93019712
:10502000DACFA0E057E04FCFA83008F046C0F60135
:10503000EA1BF109A1E08385853008F4A0E0B1E026
:10504000B50F6DE070E08B2F0B2E000C990BFB0160
:10505000E81BF90BEC0DFD1DE081EA0FA0E0EA3042
:1050600010F0A1E0E0E08E0D9F1DF0E35F2E5E0EDC
:10507000FC015082B15039F7332309F1121614F4B0
:105080008DE28A872E5FE3E0822F6E2F0E947F3CA5
:10509000E91B291BE60DF72DF11D4083822F6AE0E5
:1050A0000E947F3C90E3980F9B8790E3920FF6EF6E
:1050B0008F9F900D11249C8723CF57E0BFCF822F65
:1050C00063E00E947F3CE1E0E90FE3CF222309F493
:1050D00053CF983009F450CF8A81803309F04CCFF8
:1050E0002336A9F461E0252F550F330B2F5F3F4F77
:1050F00059E305C08E0D9F1DDC015C936F5F862F09
:10510000062E000C990B28173907A4F735CF81E339
:105110008A83332379F02150822F6AE00E947F3CFA
:1051200090E3980F9B87205DB6EF8B9F200D112495
:105130002C8722CF2F5FF0CF80E09CE22EE2F70198
:1051400031917F01F401E80FF11D3083E1E0E80FB8
:10515000D7011B963C91341310C0E80DF92DF11DB9
:10516000413049F420838E5FAE14BF0441F7880EAE
:10517000911CF4012ACE9083F6CF8E2FF5CFF894B0
:10518000E8E2F2E4118610861286138614861586EC
:10519000789408958F708A3010F0895A0895805D50
:1051A0000895CF93C82F82958F700E94CA280E94BD
:1051B000CF148C2F8F700E94CA28CF910C94CF14DB
:1051C0001F93CF93DF9327E0289FE001299FD00D05
:1051D0001124CB5EDC4B16E08A9182958F700E9481
:1051E000CA280E94CF1488818F700E94CA280E940A
:1051F000CF14115088F7DF91CF911F9108950F932D
:105200001F93CF93DF938C01EC012E968A918F70C0
:105210000E94CA280E94CF140C171D07B9F7DF910E
:10522000CF911F910F9108950F931F93CF93DF9309
:105230008C01EC0125968A918F700E94CA280E94E9
:10524000CF140C171D07B9F7DF91CF911F910F9164
:105250000895CF93C82F892F0E94CA28803311F058
:105260000E94CF148C2F82958F700E94CA280E94B2
:10527000CF148C2F0E94CA28CF910C94CF141F9367
:10528000CF93DF93D82F162FC42F82958F700E9453
:10529000CA2820E04C2F612F0E94D817182F8D2F7D
:1052A0000E94CA2820E04C2F612FDF91CF911F91DF
:1052B0000C94D8171F93CF93DF9320E046E060E66D
:1052C0008AE090E20E945618CFE1D1E116E0988181
:1052D000412F682F892F0E943F29C03191E1D907C2
:1052E00021F4DF91CF911F910895C83111F41F5F10
:1052F00088E72197ECCFEF92FF920F931F93CF9304
:10530000DF93E82EC62FD42F0E943F2968E06C0F50
:1053100020E04D2F8AE30E94D817C45F87E0E89E03
:105320007001112410E000E0F701E01BF10BEC5ECE
:10533000FC4B4D2F6C2F80810E943F290F5F1F4F28
:10534000C85F0730110581F7DF91CF911F910F9151
:10535000FF90EF900895909132429730BCF4E09125
:105360003042F0E0E85DFD4B8083809130428F5FFA
:105370008093304280913042877080933042809198
:1053800032428F5F8093324281E0089580E0089539
:10539000F894809132421816BCF4E0913142F0E06A
:1053A000E85DFD4B8081909131429F5F9093314247
:1053B0009091314297709093314290913242915046
:1053C00090933242789408958FEFFCCF8091EF6EE6
:1053D000811104C080913B6E8823D9F08091C35D18
:1053E000811117C00E94C8298F3F99F0E82FF0E083
:1053F000ED50FD4FE491E093B24281E0809325426D
:105400008093C35D8091A74290E080933C6E90931F
:105410003D6E08951F920F920FB60F9211240BB696
:105420000F922F933F934F935F936F937F938F933D
:105430009F93AF93BF93CF93DF93EF93FF938091AD
:10544000C75D8F5F8093C75D8091C75D83708093D8
:10545000C75D809136429091374286FF26C087E42F
:1054600092E40E94941F882349F0809136429091E3
:105470003742826080933642909337428091364221
:105480009091374290FF11C067E472E483E692E4A2
:105490000E94C71C882349F0809136429091374280
:1054A000816080933642909337428091364290914A
:1054B000374287FF26C085E592E40E94941F882327
:1054C00049F080913642909137428860809336420D
:1054D00090933742809136429091374291FF11C0AC
:1054E00065E572E481E792E40E94C71C882349F0D5
:1054F00080913642909137428460809336429093F7
:105500003742809136429091374292FF19C08CE326
:1055100092E40E94941F61E472E48CE392E40E949E
:10552000DD1C882369F08CE392E40E94D61C8091F4
:105530003642909137428061809336429093374251
:10554000809136428F73B9F08091BE5D9091BF5DBE
:1055500090628093BE5D9093BF5D8091BE5D90919F
:10556000BF5D90618093BE5D9093BF5D81E080934D
:10557000EF6E109299408091C75D811168C0809153
:105580009940823049F080913E6E882329F08091C5
:105590003E6E815080933E6E8091A1428F5F8093DA
:1055A000A1428091A1428C330CF451C0C1E0C09360
:1055B0009B401092A1428091A0428F5F8093A042B5
:1055C0008091A0428C330CF442C01092A042809192
:1055D0009F428F5F80939F4280919F4288318CF1E0
:1055E00010929F428091A4428F5F8093A442D091F9
:1055F000A4426091A2428091A3420E94B41A2D2F2E
:10560000DD0F330B8217130694F4C093A4428091EC
:10561000A3428F5F8093A3428091A3428D303CF0E0
:10562000C093A3428091A2428F5F8093A242409197
:10563000A4426091A3428091A2420E94911A809359
:10564000AC4280919F420E94CA1A8093AB4281E093
:1056500080935301FF91EF91DF91CF91BF91AF9173
:105660009F918F917F916F915F914F913F912F917A
:105670000F900BBE0F900FBE0F901F9018951F92AA
:105680000F920FB60F9211242F933F934F938F9346
:105690009F9381E080939A4080913542813089F5D3
:1056A000809108408150809308408091084081118A
:1056B00028C08091A842809308404EB18091396EF5
:1056C00090913A6E880F991F21E030E04F3F11F41E
:1056D00030E020E0822B932B8093396E90933A6ECA
:1056E0008091396E90913A6E892B59F4109235421F
:1056F000109202408FEF8FB99DE090936B048093DE
:105700006C0481E080930B0A9F918F914F913F91A0
:105710002F910F900FBE0F901F901895CF93DF938E
:1057200000D000D0CDB7DEB780919B40813009F02A
:1057300045C00E94402580934B6E90934C6E209103
:10574000A9424CE251E0BA01EAE02E9F60197109CA
:1057500011249B013695279536952795BA01621B32
:10576000730B6817790780F582E1898385E18A8365
:1057700086E18B831C826FEF80E00E9473172FEF0E
:1057800040E062EECE0101960E94391881E00E944D
:10579000F71A80E60E94461BE3E6F2E481E792E412
:1057A0002191211137C08E179F07D1F780E00E9409
:1057B000FB1680E00E94821710929B402496CDBF7A
:1057C000DEBFDF91CF910895B901660F771FFA010F
:1057D000E61BF70BE817F90720F482E1898384E1DF
:1057E000C6CF620F731FFA01E61BF70BE817F90724
:1057F00020F482E1898383E1BACF220F331F220F85
:10580000331F421B530B4817590710F481E1F2CFA5
:1058100080E1F0CF2FEF40E068EC87E00E94D817DE
:10582000C5CF0895CF92DF92EF92FF920F931F930F
:10583000CF93DF938091994081118CC0D12CC2E02D
:10584000CC2ED4E7ED2ED4E0FD2E11E08091EE5D5C
:105850008230F1F58091AB409091AC408093FE4254
:105860009093FF42D09297400E94E110FC0180810A
:10587000809396408091FE429091FF422091024099
:1058800021110AC08C3FF1E19F0739F5E0920340F6
:10589000F0920440109302400E9497239C01369599
:1058A000279536952795D22E7091C85D7093B14299
:1058B0001092C85D4091EE5D423009F4FEC1A0F443
:1058C000442331F1413009F49EC11092EE5D3EC097
:1058D0008091FC429091FD42C1CF883C20E192072B
:1058E000D9F6C0920240D8CF443009F4F6C108F48A
:1058F000E7C1453051F72091FC423091FD422F5FC6
:105900003F4F2093FC423093FD4280FDDECF9ECF7F
:105910004091FC425091FD42FA013196E093FC42E5
:10592000F093FD42682F6370623031F1633009F407
:1059300059C16130C1F0F901FF27EE0FFF1FE1559A
:10594000FF4F45915491822FFA0109958091EE5DA8
:1059500081117CCFDF91CF911F910F91FF90EF903C
:10596000DF90CF9008956093EE5D8093EA5D909311
:10597000EB5D70939E40EACFD22FD695D695D69503
:10598000C22FC770EFEFEC0FE73078F4F0E0E5538B
:10599000F34D0C94D73C1C2D052DD22C0A2D132D24
:1059A000162D192D2DE060E005C00E94E110FC01CC
:1059B0006081262F2093C15DD150DF3108F03EC0B9
:1059C000ED2FF0E0EA51F34D0C94D73C242D282D17
:1059D0002C2D342D3C2D402D462D4C2D522D5A2D45
:1059E0005E2D642D6E2D832D882D8D2D932D992D5B
:1059F000A12DAC2DAA2DB32DBB2DC12DCA2DCF2D80
:105A0000D52DD92DDF2DE32DE72D0E94E110FC01CE
:105A10002081C9CF6091F9422091FA4226170CF0FB
:105A2000C9CF2DE0C7CF22E062E0C4CF2CE063E015
:105A3000C1CF2DE06DE0BECF22E0B5CF422F83EB8A
:105A400092E40E94291182CF422F81EC92E4F9CF97
:105A5000422F8FEC92E4F5CF462F61EC72E483EB9A
:105A600092E40E94321172CF462F63EB72E481EC14
:105A700092E40E9418116ACF462F6FEC72E4EFCFC8
:105A8000462F61EC72E48FEC92E4F3CF462F6FEC7B
:105A900072E481EC92E4E5CF462F6FEC72E483EB85
:105AA00092E4E7CF462F61EC72E483EB92E40E942C
:105AB00045114CCF462F6FEC72E4F7CF1093C85DC1
:105AC000462F70E060E0F1CF022F262F41EC52E428
:105AD00063EB72E4CB010E94711138CF1093C85D63
:105AE000C73061F480910B438A3041F48091C04209
:105AF0008B3020F089508093C04228CF022F262F70
:105B000050E040E0E5CF022F262F4FEC52E4E0CFEB
:105B1000462F6FEC72E4CB01CACF462F63EB72E4E1
:105B20008FEC92E4C4CF1093C85D462F70E060E024
:105B3000F7CF022F262F4FEC52E463EB72E4CA0139
:105B4000CACF1093C85D022F262F50E040E06FECC3
:105B500072E4C0CF1093C85D022F262F4FEC52E4A1
:105B600070E060E0ECCF462F70E060E081EC92E402
:105B70000E94B311EBCE462F70E060E08FEC92E410
:105B8000F7CF022F262F4FEC52E463EB72E490E044
:105B900080E0A1CF022F262F41EC52E4F6CF462F12
:105BA00070E060E083EB92E4E3CF462F6FEC72E4A9
:105BB000F9CF422F83EB92E40E94A411C7CE422F6B
:105BC00081EC92E4F9CF422F8FEC92E4F5CFC3EB56
:105BD000D2E4C20FD11D261B4A9149832A95E1F7D1
:105BE0001882B4CE822F86958F7327FD8054217042
:105BF0002713B0CE480F511D87FD5A954093FC42A4
:105C00005093FD42A3CE4091FC425091FD424F5F24
:105C10005F4F4093FC425093FD421092EE5D6091C5
:105C20009E409C01217033276217130609F092CE23
:105C30002091EA5D3091EB5D369527953695279555
:105C4000BC01E6E0660F771FEA95E1F76627262B91
:105C5000372B81FF05C02093FC423093FD4276CE66
:105C600080910443909105438093064390930743AA
:105C700080910243909103438093044390930543A2
:105C8000809100439091014380930243909303439A
:105C900040930043509301432093FC423093FD42D4
:105CA000C9010E949723892B09F050CE0E94D3117D
:105CB0008093FC429093FD4249CE0E945B1446CEF5
:105CC0002091FC423091FD422F5F3F4F2093FC42D8
:105CD0003093FD420E945B1439CE882351F08091AD
:105CE000FC429091FD4201968093FC429093FD42CC
:105CF000ECCD1092FC421092FD4280913B6E8823C5
:105D000019F010939940E1CD1092EF6E1093C85D99
:105D1000C0929940DACD2091AD42022E000C330B97
:105D20002F5F3F4FAC01249FC001259F900D349FF2
:105D3000900D1124019708F40895EFECF7E03197E6
:105D4000F1F700C00000F6CF1F93CF93DF9383E0FD
:105D500090E00E948B2EC0E4D4E018E01E8383E024
:105D600090E00E948B2E1D8381E090E0DF91CF9127
:105D70001F910C948B2EEF92FF921F93CF93DF9382
:105D80000E94A42EC8E9DFE1FE0114911123F1F075
:105D90003196849122968F3F29F484E690E00E9408
:105DA0008B2EF2CF84910E94C8167E01F7018FEFEF
:105DB000E81AF80A8E2D8C1B811720F01150C10FA4
:105DC000D11DE2CF84910E94C116F0CFDF91CF9117
:105DD0001F91FF90EF9008952091AD42022E000C8C
:105DE000330B2F5F3F4FAC01249FC001259F900DC7
:105DF000349F900D1124019708F4089552E05A95AC
:105E0000F1F700C0F8CF1F920F920FB60F92112436
:105E10000BB60F92BF92CF92DF92EF92FF920F9349
:105E20001F932F933F934F935F936F937F938F9322
:105E30009F93AF93BF93CF93DF93EF93FF9388E04C
:105E400080936B048FEF80936C04DFB18FB9DD23F7
:105E500009F492C0ED2EF12C9701215031092D2328
:105E60003F21232B09F088C090919940923049F44A
:105E7000109299408FB99DE090936B0480936C04CD
:105E800055C010E000E08FE1B82ECC24C394D12C93
:105E9000C02FB0920204C601002E01C0880F0A94E0
:105EA000EAF78093010485E090E00E94EC2E8EB129
:105EB00090E0809590958E219F21892B31F40F5F82
:105EC0001F4F0530110521F7C5E080E0D69509F098
:105ED00049C0CC0FCC0FCC0FC80FC83208F044C05B
:105EE000D6E910EA80919D428111109307048EE556
:105EF00091E00E94EC2ED150A9F78C2F0E94AB2983
:105F0000882359F081E08093354224E632E32093E0
:105F1000034030930440809302408FE1809301045A
:105F20001092994080919C4280933E6EFF91EF9138
:105F3000DF91CF91BF91AF919F918F917F916F91A1
:105F40005F914F913F912F911F910F91FF90EF9093
:105F5000DF90CF90BF900F900BBE0F900FBE0F90B1
:105F60001F9018958F5FB2CF8FEF8FB99DE0909300
:105F70006B0480936C04D1CF8FEF7CCFCF92DF92F4
:105F8000EF92FF92CF93DF93ADE4BEE626E036E1D9
:105F9000D7964C91D7974F3F61F150E0DC968C91AA
:105FA000DC9790E0D6966C91D697613069F5DD96D6
:105FB0006C91DD97EC01CC0FDD1FCC0FDD1F349F02
:105FC000F001359FF00D1124CE0FDF1FC355DF4BBD
:105FD000D896CD90DD90ED90FC90DB97C882D98269
:105FE000EA82FB82E355FF4B8E0F9F1FEC01288B4B
:105FF000658B2F5F1996223159F6DF91CF91FF9073
:10600000EF90DF90CF900895349FB001359F700DD1
:106010001124EB01C355DF4BC80FD91F4889421328
:10602000E8CFFC01EE0FFF1FEE0FFF1FE60FF71F7B
:10603000E355FF4B1082118212821382DACF1F9335
:10604000CF93DF93CDB7DEB76C97CDBFDEBF11E046
:1060500060E0812F0E9473171F5F1730C9F780918E
:10606000AE42823009F441C0833069F0813079F565
:1060700020E046E061E089E50E94D81770E060E02A
:1060800082E090E022C020E042E061E084E50E94EE
:10609000D81720E044E061E08AE50E94D81720E0AC
:1060A00046E061E089E50E94D81770E060E082E098
:1060B00090E00E942D2670E060E081E090E00E9478
:1060C0002D2670E060E090E080E00E942D2611E037
:1060D000812F0E9482171F5F1730D1F76C96CDBFBA
:1060E000DEBFDF91CF911F91089520E046E061E08F
:1060F00081E40E94D817E9E4F3E467E18291811119
:1061000002C06150D8F76F5F89F520E045E065E097
:1061100082E00E94DC1963E0680F20E045E08CE03B
:106120000E94DC1963E0680F20E045E081E00E94F6
:10613000DC1963E0680F20E045E08EE00E94DC1986
:1061400063E0680F20E045E08BE00E94DC1966E622
:1061500085E00E94451766E686E00E94451720E02C
:1061600046E061E081E40E94D817B1CFE62FF0E06D
:10617000EF5CFC4BCE010196DC0122912D932A2F7E
:10618000281B2617D4F345E00E94A225E8CF7F9272
:106190008F929F92AF92BF92CF92DF92EF92FF9237
:1061A0000F931F93CF93DF93CDB7DEB76597CDBF26
:1061B000DEBF4C017A01CA0140968B01041B150B0E
:1061C0006817790710F000E110E040E3BE016F5F4F
:1061D0007F4FC7010E94F2248DE28C831D822FEF36
:1061E00040E06EEBCE0101960E94391840E3BE01FB
:1061F0006F5F7F4FC7010197800F911F0E94F224AC
:106200002FEF40E06EEDCE0101960E9439188E0C02
:106210009F1CC12C8AE3782EAC2CB12CA016B106A1
:1062200088F06596CDBFDEBFDF91CF911F910F91B2
:10623000FF90EF90DF90CF90BF90AF909F908F90A6
:106240007F900895BE016F5F7F4FC501880D991D36
:106250000E942D26DC2CD694D394C0FC21C040E2B1
:10626000BE016F5E7F4FC5018E0D9F1D0E94F224FF
:106270007C8A1D8A20E04D2D61E0CE0141960E946E
:10628000391820E04D2D62E2CE0101960E943918A6
:1062900020E04D2D6AE88CE70E94D817C394BCCF4C
:1062A00020E04D2D62E9CE0101960E943918F6CF0B
:1062B0008130A9F028F08230F9F0833031F108956F
:1062C00088ED94E184BF909368008AE990E0809320
:1062D000260A9093270A8AE080930206089588EDA3
:1062E0009CE184BF9093680085E391E08093260A47
:1062F0009093270A8CE0F0CF88ED25E230E084BF50
:106300002093680080ED91E0F1CF88ED2DE230E040
:1063100084BF209368008BE692E08093260A9093D6
:10632000270A8DE0D9CF84EF91E00E948B2E81E384
:10633000809360098091AD420C94583183E00E94B3
:106340005831E0E2F8E087E594E08087918783E0C8
:1063500087838681806C868380E8858384E690E0ED
:106360000C948B2ECF93DF93109260090E949E3184
:106370008CE00E94CF1489E090E40E946624C2E081
:10638000DEE5899182958F700E94CA280E94CF1401
:10639000FE01319780818F700E94CA280E94CF141D
:1063A0008EE6CF31D80769F78AE00E94CF148FE0DC
:1063B00090E40E94662484E00E94CF14DF91CF9184
:1063C0000C9493310F931F93CF93DF931092600936
:1063D0000E949E318CE00E94CF148AE00E94CF146C
:1063E00080E50E94CF1488E50E94CF1484E30E94C8
:1063F000CF1481E30E94CF148AE00E94CF14D0E032
:10640000C0E0CE010E9489248823E1F0CE01C03192
:10641000D10508F0C0960E94292980E20E94CF147D
:1064200010E000E0C8018C0F9D1F0E94E02880E270
:106430000E94CF140F5F1F4F0430110599F78AE0B7
:106440000E94CF142496C03D43E0D407D1F681E4E6
:106450000E94CF148AE30E94CF1480E20E94CF14DE
:1064600083EB92E40E94FF2880E20E94CF1480E236
:106470000E94CF1482E40E94CF148AE30E94CF14BA
:1064800080E20E94CF1481EC92E40E94FF2880E217
:106490000E94CF1480E20E94CF1483E40E94CF14A4
:1064A0008AE30E94CF1480E20E94CF148FEC92E422
:1064B0000E94FF288AE00E94CF1483E50E94CF1437
:1064C0008AE30E94CF1480E20E94CF14CDE0D0E096
:1064D00001E010E020910C4330910D43C8010C2ED7
:1064E00002C0880F991F0A94E2F782239323892B15
:1064F00009F055C080E30E94CF14219758F78AE035
:106500000E94CF148DE40E94CF148AE30E94CF141E
:1065100080E20E94CF148DED92E40E94FF2880E279
:106520000E94CF1480E20E94CF148EE40E94CF1408
:106530008AE30E94CF1480E20E94CF148BEE92E493
:106540000E94FF2880E20E94CF1480E20E94CF14B4
:1065500087E40E94CF148AE30E94CF1480E20E9455
:10656000CF14809109438F700E94CA280E94CF14D3
:10657000809108438F700E94CA280E94CF148AE03D
:106580000E94CF148FE090E40E94662484E00E9471
:10659000CF14DF91CF911F910F910C94933181E330
:1065A000AACF109260090E949E318AE00E94CF1407
:1065B0008AE00E94CF1484E190E40E9466248091D6
:1065C000FD420E94D1288091FC420E94D1288AE09D
:1065D0000E94CF1485E190E40E9466248FEC92E43F
:1065E0000E94FF288AE00E94CF1488E190E40E9474
:1065F00066248091BE5D9091BF5D892F0E94D12855
:106600008091BE5D9091BF5D0E94D12880914642ED
:10661000811166C08DE190E40E9466248AE00E94A8
:10662000CF148FE290E40E94662487E492E40E94F3
:10663000FF2886E390E40E94662483E692E40E94A9
:10664000FF288EE390E40E9466248FE792E40E9484
:10665000FF288AE00E94CF1486E490E40E9466241A
:1066600085E592E40E94FF288DE490E40E94662470
:1066700081E792E40E94FF2885E590E40E94662469
:106680008DE892E40E94FF288AE00E94CF148DE5F5
:1066900090E40E94662481E492E40E94142985E635
:1066A00090E40E9466248CE392E40E9414298FE611
:1066B00090E40E946624809137420E94D128809104
:1066C00036420E94D1288AE00E94CF140E943224D0
:1066D00084EF91E00E94EC2E81E38093600908959D
:1066E00086E290E499CF8F929F92AF92BF92CF9221
:1066F000DF92EF92FF92CF93DF93C2E0812C912C37
:10670000540180E090E8A0E0BB278A539748AF4F40
:10671000BF4F6C017D01C80CD91CEA1CFB1CDFE1DA
:1067200061E0EBBEF6018791882369F020E04C2FF1
:106730000E94D817682FD1508FEFC81AD80AE80ADC
:10674000F80AD111EECF80E2880E911CA11CB11C79
:10675000CF5FC630B1F6DF91CF91FF90EF90DF9021
:10676000CF90BF90AF909F908F900895CF9388E780
:1067700090E00E948B2EC0E080913542813019F06C
:106780008C2FCF91089582E390E00E948B2E729916
:10679000F3CF8FEF0E942D170E94B5170E94B231E0
:1067A0008FEF0E942D170E94B517C1E0E5CF2F9201
:1067B0003F924F925F926F927F928F929F92AF9291
:1067C000BF92CF92DF92EF92FF920F931F93CF93DE
:1067D000DF93CDB7DEB76C97CDBFDEBF80916B4343
:1067E00020E1829FC001112420916A4322952F70DD
:1067F000822B20E032E04901881A990AAC0140530B
:1068000051094B8F5C8FD12CC12C10E0E12CF12C65
:106810002FEF31E0F901E81BF90BE98FFA8F59EB03
:10682000452E5EE6552E0E9422176FEF80E00E94F3
:1068300073176FEF89E00E9473176FEF8AE00E9471
:106840007317F6E0FF9EC00111242FEF40E061E0D6
:106850008C569F4D0E9456182FE02F15E8F0EF2D13
:10686000F0E0EB5CFB4C0C94D73C45348834983416
:1068700059355F3569354235AE347C34F234B43441
:10688000F235963561368234A43409E026E042E0E0
:1068900065E080E00E9473180E94B5178091500057
:1068A000897F846080935000809150008160809344
:1068B00050008895809150008E7F80935000809189
:1068C0003E6E8111BAC287E00E94AB296C96CDBFA3
:1068D000DEBFDF91CF911F910F91FF90EF90DF907E
:1068E000CF90BF90AF909F908F907F906F905F9070
:1068F0004F903F902F90089508E026E244E06EE12B
:106900008BE2C8CF08E02CE243E067E081E0C2CF31
:1069100008E026E147E168E189E10E94731880916F
:10692000AE420E9408190E947B1C0E941F30B4CF07
:1069300008E026E246E26CE08DE00E947318809148
:106940009D420E940819A8CF08E026E246E26DE2C7
:106950008EE20E9473188091AA42F3CF08E026E2EB
:1069600046E26BE18AE196CF08E026E246E266E283
:1069700086E20E94731846E7642E43E4742E1E8A52
:1069800001E02E88312C37E0A32EB12CBE016F5FC1
:106990007F4F822D0E94E124F301808190E00A2C38
:1069A00002C0959587950A94E2F720E080FF26E6DD
:1069B000402F632DCE0101960E9439182394F1E0F7
:1069C000AF1AB10820E2320E3FEFA316B306F1F67C
:1069D0000F5F4E89485F4E8B51E0651A7108083091
:1069E00081F65ACF8114910409F447C081E090E107
:1069F000C916D1040CF480E09601215F3F4FE98D68
:106A0000FA8D2E173F0708F4826008E026E246E27E
:106A1000823071F1833079F166E2813051F58DE198
:106A20000E9473182FEF40E06CE58EE890E20E9420
:106A3000561840E2BE016F5F7F4FC4010E94F224EE
:106A40002FEF40E064E8CE0101960E9439188114CE
:106A5000910431F0A601B4018B8D9C8D0E94C7304A
:106A600001E0802F0E9482170F5F0930D1F714CF09
:106A70006CE186E2D5CF6CE1D2CF08E026E246E2B7
:106A800066E2F7CF08E025E144E163E182E10E949C
:106A9000731880919C42883751F0803F21F08C33ED
:106AA00021F480E04ECF82E04CCF83E04ACF81E0FA
:106AB00048CF08E026E246E26BE08AE0EBCE08E051
:106AC00021E140E16FE08EE00E9473188091AD42B9
:106AD00038CF2FEF40E061E68CE290E20E9456183A
:106AE0000E9473330E945A290E944025BE016F5FA5
:106AF0007F4F0E9417252FEF40E062EDCE010196F7
:106B00000E94391820E046E061E08EE090E20E94A9
:106B1000561820E048E061E08EEE9FE10E94561892
:106B200008E026E246E266E281E2B4CE20E042E0FE
:106B3000410F61E088E00E94D81720E042E069E060
:106B400088E690E20E94561820E043E069E08BE579
:106B500090E20E94561820E044E069E08EE490E262
:106B60000E94561820E045E069E081E490E20E942E
:106B7000561820E046E069E084E390E20E9456184F
:106B800099E0A92EB12C00E02AE0722E0430F1F435
:106B90008091A942BE016F5F7F4F879DC001112484
:106BA0000E94172542E0400F20E06CE6CE010196DE
:106BB0000E9439180F5FFFEFAF1ABF0A053031F797
:106BC00008E025E244E263E282E264CEF501E456A5
:106BD000FD4B808140E3BE016F5F7F4F90E00E94DC
:106BE000F224E0CF08E026E246E268E280E2E1102B
:106BF0008FE10E94731848E0E49E9001112446E161
:106C0000429FC001439F900D1124FC01E355FF4BAF
:106C10005F0100E02E2C220C220C220C2A940F5F24
:106C2000822D800F0E94CA2820E0402F62E00E943F
:106C3000D817AE8ABF8A8CE0382E712C612C20E0E8
:106C4000402F632D8CE70E94D817EE89FF89819130
:106C50009191A191B191EE8BFF8B892B8A2B8B2B7C
:106C600049F1F501E60DF71D808929E0289FF00123
:106C70001124E35BF149908126E6911120E037E091
:106C8000839FC0011124402F6AE0630D885B974009
:106C90000E9456184FEF641A740A5CE3350E84E0C4
:106CA0006816710461F696E1A90EB11C083009F06E
:106CB000B6CFF2CD26E6402F6CE0630D87E890E278
:106CC000E7CF812F012E000C990B069629E0289F13
:106CD000F001299FF00D1124E35BF149818108E067
:106CE00026E28F3F39F0808108E026E24BE08823DE
:106CF00011F02AE246E263E282E20E94731820E089
:106D000041E06AE08EE190E20E94561820E041E006
:106D10006AE88EE190E20E9456180FE181E020E0DF
:106D200042E0682F8BE10E94D8170150C1F720E0A4
:106D300042E068E78EE00E94D81720E041E068E773
:106D40008CE70E94D817812F66E00E947F3C9D5FF0
:106D50009E8B8795882787958F5F888FADE4AA2EB5
:106D6000AEE6BA2EB2E76B2EB8EF7B2E312CF501D2
:106D700086A900E0813009F006E6F5E0F31510F190
:106D8000F3E02F2E230C202F422D6AE0C3010E9436
:106D90005618F50187A9202F422D6AE48F3F41F153
:106DA0000E94CA28202F422D6AE40E94D817F501BC
:106DB00084AD8F5F0E94CA28202F422D62E60E9478
:106DC000D8171AC0EDEF2E2E230C20E0422D68E7D5
:106DD0008CE70E94D817202F422D6AE8C3010E9439
:106DE0005618F50187A98F3FC1F4202F422D6CEC76
:106DF00082E890E20E94561820E04E89688D88E073
:106E00000E94D8173394F9E0AF0EB11C27E0620E50
:106E1000711C3CE03312ABCF3FCD0E94CA28202F1B
:106E2000422D6CEC0E94D817F50184AD8F5F0E9453
:106E3000CA28202F422D64EEC2CF80913642857041
:106E400029F480913542882309F428CD0E94C8296D
:106E5000082F0E94B633813009F40FEF0E94BF283B
:106E60004FE04F15F8F0EF2DF0E0E75CF84C0C9494
:106E7000D73C49376D378937F2374B396839CB37CB
:106E8000A3372539AF37B337AB397139B83934390E
:106E90009837003109F4EFC2C8F4002339F0083004
:106EA00009F460C2033011F0073049F50E9422173F
:106EB0000E94B51781E080939B400E948E2B0E9418
:106EC000481C0E947B1C0E941F3000CD083109F431
:106ED000CFC2003239F701E08BC00031C1F048F475
:106EE000002309F485C083E00830E1F68093AE42C8
:106EF00006C0083151F00032A9F61092AE428091DE
:106F00003642857009F48FCCD1CF81E0EFCF82E09B
:106F1000EDCF083149F0003221F00111C3CF0EE06E
:106F200067C010929D42EBCF81E080939D42E7CFF6
:106F3000083129F0003289F71092AA42E0CF81E0AF
:106F40008093AA42DCCF083139F0003209F49CC2A8
:106F50000111A8CFF12CD3CF7AE0F72ED0CF083192
:106F600071F0003221F001119DCF07E041C050E1E6
:106F7000C51AD108D7FEC3CFD12CC12CC0CFC601B2
:106F80000F96E98DFA8D8E179F0708F0B8CFF0E1C4
:106F9000CF0ED11CB4CF0031C9F048F40023F9F072
:106FA0000830B1F080919C4280933E6E7BCF0831D7
:106FB00059F08CE30032B1F780939C428091714389
:106FC000877F80937143EECF88E7F6CF80EFF4CFD1
:106FD0008FEF80939C42809171438860F2CF6EE086
:106FE000F62EE0CF083149F0003221F001115ACFDE
:106FF000F02E85CF0E94E23182CF20E044E062E0B3
:1070000085E790E20E94561884E00E94821785E08E
:10701000E0E9F0E4DE01519601900D928A95E1F7E6
:10702000109260090E949E310E94E8148AE00E943A
:10703000CF1487E790E40E9466240E940D241092EA
:10704000C25DF12CE12C7724739494E0992E6E01AB
:1070500021E1C20ED11C25E0622E30E3832E42E0F6
:10706000442E53E0552E8091C25D823089F040F469
:107070008823D9F1813009F463C09092C25D93C036
:10708000833009F4DBC08530C1F70E94E814DAC010
:1070900037E03E9D80013F9D100D11240D541D4B86
:1070A00084E0382EA5E0AA2EB12C0E94EB23282ED6
:1070B0002294B0EF2B220E94EB23F501E45AFF4FFC
:1070C000E00FF11F8229808341E0A41AB1085EEF2E
:1070D000A5165FEFB50649F73A94095F1F4F3110C7
:1070E000E1CF84E0E80EF11CA2C010E08091015EC7
:1070F000882359F00E94B114F601E10FF11D90812F
:10710000891711F01230B8F41F5F0E94C8298F3F11
:10711000A1F06092C25D8091C25D853009F443C0E8
:107120000E94B1148A3021F00E94C8298F3FC1F318
:107130007092C25D38C010E0E8CF1430B9F6EBCFE2
:10714000898A8A8A8B8A10E000E08091015E882318
:1071500061F00E94B114182F80ED810F8A30B8F5CC
:10716000F601E00FF11D10830F5F0E94C8298F3FC9
:1071700009F442C06092C25D8091C25D833099F093
:107180000C0D1D2D111DB12CA12CF12CE12C0C1579
:107190001D05B1F520E1E216F10418F030E3E31A21
:1071A000F1084092C25D8091C25D843009F05BCFEE
:1071B0008CE890E40E9466240E9493310E9422177A
:1071C0000E94B51781E080939B4083E07DCB8FE9DF
:1071D000810F863028F28FEB810F863038F4F6016C
:1071E000E00FF11D80E2810F8083BECF1A3309F0DA
:1071F000BCCF5092C25DB9CF103209F0A6CFBCCF40
:10720000F80182918F010E94072490E00A2C02C0AD
:10721000880F991F0A94E2F7E82AF92AF4E0AF0EE2
:10722000B11CB5CF0E94C8298F3F09F081CF0E94C1
:10723000B1148A30B9F77CCF0E94B1148091015EFD
:107240008111FACF0E94B11018CF003109F416C194
:1072500008F47ECE083121F0003209F460CE22CE4F
:10726000E12CFBE0FF2E4BCE003109F40AC148F4BB
:10727000002309F477C0083009F014CE7FE0F72E20
:107280003ECE083129F0003209F00CCE02E0B0CE3B
:10729000E6E0FE2E34CE0031B1F050F40023A9F028
:1072A00083E0083069F08091AD420E945831FACDF8
:1072B000083129F00032B9F71092AD42F4CF81E0E5
:1072C0008093AD42F0CF82E0FBCF6EE0F62EEBCFA5
:1072D000002309F447C0003209F0E4CD10E00CE0CF
:1072E00087CE003141F1B8F4002309F4D1C0083051
:1072F00009F0D8CDE12F012E000CFF0BEB55FD4B13
:107300008081815080838091A9428F3108F4F7CD2C
:107310008EE18083F4CD083141F0003209F0C2CD16
:10732000115008F0ECCD14E0EACD1F5F153008F4E1
:10733000E6CD10E0E4CDE12F012E000CFF0BEB5564
:10734000FD4B80818F5F80838091A9428F3108F44B
:10735000D6CD1082D4CD083109F49CC0003229F07A
:107360000111A0CD88E0F82ECACD81E0E826C7CD76
:107370000031B9F138F5002309F48FC0083009F065
:1073800091CD812F012E000C990B069629E0289FA4
:10739000F001299FF00D1124E35BF1492085EDE414
:1073A000FEE636AD321301C016AA39964E165F06B8
:1073B000C1F739E0389FF001399FF00D1124E35BEC
:1073C000F149C7CF083141F0003209F06BCD1150BF
:1073D00008F095CD1BE093CD1F5F1C3008F0A9CFBE
:1073E0008ECD812F012E000C990B069629E0289F47
:1073F000F001299FF00D1124E35BF14940855DE424
:10740000A52E5EE6B52ED501DE968C91DE9784130F
:107410001DC08DE49EE6FC0156AD451791F0D79650
:107420003C91D79727A932130CC02DE43EE6F90111
:1074300066AD561301C016AA275F3F4F421653068A
:10744000B1F70996FEE6893B9F0729F719962EE6C4
:10745000A93BB207C9F681E0F50196AD491301C019
:1074600086ABF9E0AF0EB11C4A145B04A9F747CD17
:1074700047E0F42E44CD33E0F32E41CD25E0F22E4B
:107480003ECD94E0F92E3BCDD12CC12C09E0B0CDFE
:1074900005E0AECD10E00DE0ABCDE12C10E00BE04F
:1074A000A7CD1F93CF93DF9381E08093AD4280916E
:1074B000AD420E94583180917C008E7F98ED94BF40
:1074C00080937C008091630083FDFCCF80917C00E1
:1074D00098ED8B7F94BF80937C0080917C008160CD
:1074E00094BF80937C00809141018111FCCF82E0A8
:1074F00080934701C1E0C093520181E6809350011F
:10750000C0930A0A1092010A8091090A8E7F809323
:10751000090A86E08093000A8091000A81608093C6
:10752000000ADFEFD0930104D093060480E8809333
:1075300005040E94B016D09362048DE080936B0422
:10754000D0936C04DFB91092A000D5E0D093A400D2
:1075500080E48093850689E48093080610920006F3
:107560000E94BF2887E38093A1428BE38093A042CF
:1075700010929F428CE08093AB42D093A44213E0E0
:107580001093A34285E18093A2424091A44260916E
:10759000A3428091A2420E94911A8093AC42C09370
:1075A0009B401093AE421092C75DC0939E421092D2
:1075B0009D4288E780939C4284E68093A5428CE1BB
:1075C0008093A6428CE38093A742D093A84288E19F
:1075D0008093A942C093AA420E94402580934B6E9B
:1075E00090934C6E80919C4280933E6E7894DF9194
:1075F000CF911F9108950E94513A84E690E00E9435
:107600008B2E0E94BB2E0E94431980ED97E00E94B2
:107610008B2E0E9422178AE00E9482170E948E2BD6
:107620000E941F300E9497220E94BF280E94E814E7
:107630000E94B1100E94D822FF24F394D1E018E0F8
:10764000CFEF8EEFE82E0DE090E8D92E8091994093
:10765000813009F406C108F474C08230B9F7109380
:107660006B04C0936C04CFB98091AA42813031F48D
:107670000E94431988EE93E00E948B2E0E946A1AA2
:107680000E948B1A0E94BF28F0920004E09204042A
:107690008AE090E00E94EC2E10936B04C0936C047F
:1076A00000937704CFB980915000897F84608093E4
:1076B00050008091500081608093500088958091A7
:1076C00050008E7F8093500080919940823059F312
:1076D000C09300040E948E1AC0930604D092050441
:1076E0000E94BE2F82E390E00E948B2E739906C009
:1076F0000E94E8140E94B1100E94D8228091354265
:10770000813009F4A9C0D093EF6E1092FC42109220
:10771000FD421092EE5DD093C85D1092C35DD09390
:107720003B6E0E94481C0E94B61B0E941F30D093E3
:107730009B400E948E2BCFB900936B04C0936C04C6
:1077400085CF8091A54290E080939C4090939D408E
:1077500080919A40813021F08091024081114AC08D
:107760008091C35D811116C00E94C8298F3F91F09E
:10777000E82FF0E0ED50FD4FE491E093B242D0935A
:107780002542D093C35D8091A74290E080933C6EE8
:1077900090933D6E0E94122C80910240813061F4E2
:1077A0008091034090910440009709F452C00197E2
:1077B000809303409093044080910540813079F498
:1077C0008091A64220919C4030919D40820F932F42
:1077D000911D80939C4090939D4010920540809114
:1077E0009C4090919D40019780939C4090939D4038
:1077F00010929A4080919C4090919D40892B09F075
:10780000A7CF809106408823B9F02091376E309140
:10781000386E80910040909101402817390751F04F
:107820000E94B61B8091376E9091386E8093004015
:10783000909301401092064080910740882331F0D8
:107840000E94481C0E947B1C109207400E948E2BB5
:10785000FDCE10920240B0CF82E390E00E948B2ECA
:107860004DCF109202400E941F300E94481C0E947F
:107870007B1C80915000897F8460809350008091B0
:1078800050008160809350008895809150008E7FD9
:10789000809350000E948E2B80913E6E811109C012
:1078A0008091714383FD05C087E00E94AB2910924F
:1078B000994080913542813071F4109299400E9434
:1078C000C829833069F40E94B633811102C00E9436
:1078D000D7330E94B61B80919940813051F2B6CEC9
:1078E0000E94AB29F6CF991B79E004C0991F961727
:1078F00008F0961B881F7A95C9F78095089587FB35
:10790000082E062687FD819567FD61950E94733CD0
:107910000EF4919507FC81950895AA1BBB1B51E1BC
:1079200007C0AA1FBB1FA617B70710F0A61BB70BEF
:10793000881F991F5A95A9F780959095BC01CD0194
:10794000089597FB072E16F4009407D077FD09D011
:107950000E948D3C07FC05D03EF4909581959F4F89
:107960000895709561957F4F0895A1E21A2EAA1B84
:10797000BB1BFD010DC0AA1FBB1FEE1FFF1FA217DF
:10798000B307E407F50720F0A21BB30BE40BF50BDC
:10799000661F771F881F991F1A9469F76095709565
:1079A000809590959B01AC01BD01CF010895EE0F2C
:1079B000FF1F0024001C0BBE0790F691E02D0994D8
:1079C0000E94B23DB7FF0895821B930B08950E9459
:1079D000B23DA59F900DB49F900DA49F800D911D69
:1079E00011240895DF93CF931F930F939A9DF02D49
:1079F000219FF00D8B9DF00D8A9DE02DF10D039FD1
:107A0000F00D029FE00DF11D4E9DE00DF11D5E9DFC
:107A1000F00D4F9DF00D7F936F93BF92AF925F93E8
:107A20004F93D5010E94B23D8B01AC01D7010E945A
:107A3000B23DEB01E80FF91FD6010E94413D2F91A5
:107A40003F91D6010E94B23DC60FD71FE81FF91F14
:107A5000AF91BF910E94413D2F913F910E94B23D55
:107A6000C60FD71FE81FF91FD6010E94B23DE60FCF
:107A7000F71F9801BE01CF010F911F91CF91DF91A8
:107A800008950E94B23D460F571FC81FD91F08F422
:107A900031960895689401C0E8948F929F92CF9395
:107AA000DF930E94583DDF91CF919F908F90089572
:107AB00088249924F401E401B0E49F93AA279A153D
:107AC0008B049C04ED05FE05CF05D007A10798F4B3
:107AD000AD2FDC2FCF2FFE2FE92D982C892E982F3C
:107AE000872F762F652F542F432F322F2227B85000
:107AF00031F7BF9127C01B2EBF91BB27220F331F29
:107B0000441F551F661F771F881F991F881C991CCB
:107B1000EE1FFF1FCC1FDD1FAA1FBB1F8A149B0473
:107B2000EC05FD05CE05DF05A007B10748F08A1872
:107B30009B08EC09FD09CE09DF09A00BB10B216000
:107B40001A94E1F62EF49401AF01BE01CD01000CB0
:107B500008952A0D3B1D4C1D5D1D6E1D7F1D801F50
:107B6000911F0895A29FB001B39FC001A39F700D04
:107B7000811D1124911DB29F700D811D1124911D35
:107B80000895DC0101C06D9341505040E0F7089525
:047B9000F894FFCF97
:107B9400FF0001C80001010105444953500A004592
:107BA4004F460A0050433D002046493D0020546999
:107BB4006D65723D41002054696D65723D4200431C
:107BC4004C4B5F413A0020414C4D5F413A002053F9
:107BD40043525F413A00434C4B5F423A0020414CD0
:107BE4004D5F423A00205343525F423A00494E549B
:107BF4005F54563D0020494E545F434E543D00208F
:107C0400544D525F533D0057616974696E67206635
:107C14006F7220646174612E2E2E0A004F4B0A008D
:067C24005058343100004D
:108000000106B5064E70F858985684D84C5B8C4BD8
:108010004C3B1C427070384BAE783C0670B958CE61
:108020008CA08D08849B76761908AE58FC58F3997D
:108030009E990AB5960D9E1596BD966262C6CA5067
:108040001C231908AE58FC58E21BE2371100EE5C05
:10805000981C45028CA08411008D08580CA0B5A274
:108060007B9BCBC313E3DB4B43CB3B434B535BBD0E
:10807000B25100E30E1C5016B523110CAE0E93C482
:108080008370FA70A033F0B80E6150F86550C4F0F8
:108090007C30147C3050BCE0C8CCF73008C8CC66CB
:1080A000EBE0D5884FA550F0D44FA550D43FA8F0B1
:1080B000EECBA550AEB87C58AE8CA74C3344983C60
:1080C000A883B5BC84634C6100431300A550EED473
:1080D000D3B87C588C33A3B070E0A550EED433B83D
:1080E0007C588CC378A84E703868F828EEE8B5BC88
:1080F0008860A04E70B85860434C3748ED04711C3E
:10810000EC1F0C1B919CCC9BCCA3203C560630183A
:108110006621463087662F110C1D02C8CC5C5AD0F0
:108120007038CC9704624728707C3014FCE090666D
:10813000281C70381B2E28BC30EB33B898A8E00000
:10814000A383634323387C8338FC6B383C53387CEF
:108150003B387C2338083C8C1BADBC300670FCE0FF
:1081600048711C8C7F0C238914538C2B0441B02341
:10817000F8992C4C3F305166FB610044ED040CC76C
:108180000100D50CCC0F3008999C0CCFB83C580C92
:10819000D91C6000711CEB5924305006CC4F300CB8
:1081A000B19CA6CB091E201CE2153221460100E03D
:1081B000D50CCC3F300A999C0CBBB8F10C7CD80490
:1081C000884484D83C467CA8C46100CC4B30C306AC
:1081D000203C1C6ADB78EE30BF0E66267BA606705C
:1081E00038EE4B3EB75EF0FC56468B300770999CDC
:1081F00051844E7020B8BC588CC50284983CA8E0CD
:108200006D5820091EC8CC6046F070306906787C35
:10821000660FBC6670380EBAF038BA6EB7F04670AA
:10822000B858CCA03846BC30E660C4783C1C420A42
:10823000BD8E60A0587058585870707070E0DCA007
:10824000C44484C44404B1702DD91C610030FF0EB5
:108250004EF0E020F0AE70AEF0A6DB309C3C30A7D4
:108260003C309B685A2E28704E9C103020E84E708F
:108270009C90105C1010A8883006999C3069067894
:108280007CA63C68D5060ECC1F4CA038CC432E28CB
:10829000BC30B606E00C6B90662870387C1C0A1C5B
:1082A0004E70E06228E01908AE581C58F6BDBE4476
:1082B000F64348F62BF6603D02568C33841100B12C
:1082C0000EAE8E301EC63F4CC3301AC6A36E3008A9
:1082D000EE4E702E3C86F313EE66F3EEB8AE3D0222
:1082E000D588387E7E8953065E04467056607CA62B
:1082F0004708FCA627FCA64B3CED08E606E6E6464A
:1083000046FC06E01C8ECECC474C37784C1758E024
:10831000CC8338BC3AEEE2DFCE308E1A3C7E1E4E65
:108320001CAE3A30AEAA3CBECB133CEAF358AE6E5C
:108330001C53CE3A303C46FC6E1A3A3CEA38CA2806
:10834000E044E23349A459A41B49A4E5A43C1E4ED1
:10835000BE4F58E5A4D898D83CBB2550581CDD8C9E
:108360006EB858E065BC8C1BCCA0044841B0336D9E
:10837000BCCE992CF90C8C2F3C580C6765204670AC
:10838000B85888D3C4B83C5804987C58042B492466
:10839000B8587CD804D8FCD88404D87C8498A8E049
:1083A00085BC390C048CBBB85804ED04C4E0B01A89
:1083B00030E61B1C50BCAEC1B0AE4D14DDAC492440
:1083C00065205DBC651C4C752EB85888987C580893
:1083D000983CA81D02B85884987C5804A341B0F971
:1083E0000C3330A7C8CCF91E66DB2DAA8D08F681A8
:1083F0000B1C98B10A30FD70F0B8150A46A809BAEE
:108400008BA3ABDBB3ABA39B93FBA3F3032B23C9DE
:108410001230CFA663B51230903B1D140912309173
:108420000286061D146684E37330D04330CE0663A3
:1084300065169C021D1411B41DB4D884D81B30A835
:108440000629BF30AE06AF19B4D8D91C8C2330E052
:108450001B30D02D149388309C0613841D1411B446
:1084600006D91CA6D88C7384D884E6BD1C090E04DA
:10847000DD14661BD806163066066B1E7E8C177ED2
:10848000A1140CDDAC5D1E307006C7668B307466BF
:10849000D3069B3071463C301A7E3766EB305C4623
:1084A000E80B3065DB307A4636BB30689B301D0602
:1084B000CB3B301A06CF6667B8D8485CA2E2178873
:1084C000D8E88B266637DD1430053B302D23A61CFB
:1084D000D0E51411B46E5606D91C301D1C621F065F
:1084E000970C2B301FE5140912E6161D1411B46EFB
:1084F000060404CC13081C02A65A56BC1AD91CB890
:108500003007E8BAEF6E49241C0C2DB50CE5A46EBB
:1085100006D91CA675B0E9145B6E3DA41DB48E0689
:10852000D91C1C627330CF2D1449246E3DA46EAE4D
:10853000C512AA625830C02D14CCEF8CDBE0B8B85D
:108540003044E86914061ED91CA1143020E8F89CB8
:10855000E213A83060A820045330C848C8CCA066F5
:10856000E34404048449242DA806864C2BAD7043B3
:1085700093C1B01EA114C66FCC4F6914061ED91C3E
:10858000A11409123020E84924B80E41A41DB41CDE
:10859000EAE38E56063C3040FCE0BD1C2012050785
:1085A000204924785A0E43660E7038EE477A30C060
:1085B000661BAEA3AE3CE03020E80C57302006F836
:1085C000A85666A00879B2D91CA6063C30147C30A7
:1085D0001C50BC087A3056D84C1B36448C1B048483
:1085E000D8E80C8F3020E8E09E4EA0A60E3C266610
:1085F000EEEEEEEEE6A63C266606BEEEEEEEEE06ED
:10860000AEFC2E6E0E60DE77DC101E7CFE7FFCBEA4
:10861000FE5FFCBE437E9EBE1F3CEB7E3C1A9EFC72
:108620009CBE603003FCE8D34670CEED28041413E2
:1086300008AE58FECD7DE05CE0D460D0DC6202D7AD
:10864000629362E97CE0C2E223302C1B302ED4A07E
:10865000D57C33E97CE0D414030CA01C98E217D439
:10866000A03045D57C98F6CD7D7B1C38BC44137A70
:108670003076EF76DF7617483C0AE0CC1BAA7339D8
:1086800088E60952D5883ED74DA6251CD91C302036
:10869000E81538004C73B0E22F302DE813B8957C04
:1086A000D91C7B30C30E203C0A2365202B4E203C76
:1086B000D026E806303404661708B0C606C61CD0BB
:1086C0000C1BE21722E866F13A0E30410660304B8F
:1086D00006F3302506FCE61C0A301E6A23666A375C
:1086E000FC0E66813A30CD6A2F3C3E3EA366E030F8
:1086F000610660306606A0301ADBB03C0E660401ED
:10870000AC0C0F1CE22F0E16913E70012053AED818
:108710000C27B0B13E088BC1B0B1BC492444B0A114
:108720001CF93E589DBC981C1D88FC1EBEBEDDA4D5
:108730004E70E5A4D8B0D83CBEC32550704670B08A
:1087400068301E7CA11C0441EEB83CD844D8FCA87B
:10875000D91C78D884D8F04926410CA83080A6E6E8
:108760004EF070B858CC1F0C1B66664C17168C1355
:108770006E3C588C233080464C2F8C23767676BC0A
:10878000588C2B76767676BC56EE3C56EEEE4E3016
:10879000107030FDF0AEF046F070B858E07CD80CA8
:1087A000DD2F580C2B30844D320CDF890C4C3304F8
:1087B000B170434BF8E61F26E865144C19387DBCB0
:1087C000651CC8F84666E8B858F6F62B9DBC410C07
:1087D00004B898A859248C47C1B0302EA84924C1A8
:1087E000024E28E8A89868E0FC5C0AB8AAA8E0B0A5
:1087F00030E83AF6E3E030107030FDF0E0000000C1
:108800005AEEEEFCC6E6E6C63C06BC5CEA5A505C94
:1088100030662B22E399C63AC60E3006C3A6E67A26
:108820005ABC1A30F6F63C58FC0E3C3A301C0A3C56
:108830005AB03AE07AF30438BC585C98FE9526FCAE
:1088400010D0900EEE7E93EE0C31237EDBEE7EA3F5
:10885000FE13081C78221BDCEB1465238C27787E22
:108860006881228CAF88DB780EDC901E6F080CC705
:108870004E6E56DC5050087B0C5F0C1F0CE30C1F37
:1088800008330423780E561C561750DB7E63EE7EA9
:108890004B9C78221BDCEB9443E030D066FB20E05D
:1088A000D400980278A26838BC983C28E01CAE58E6
:1088B0000813044E6E56DC90688DB8B8580C2BC95E
:1088C0008C89B68CB551884EE80CDDB641A48A4936
:1088D00024DD20792419B46A1C0A301D623F0A2B5A
:1088E000AE9C58636E1DA4DD8CC1026E601CCB383B
:1088F000BC58780ED91CE9501C622B62BEDCDBA28E
:108900000C471437D4A250DCDC8C5BBE1FDCEB8C34
:108910001BD013D0DC4C9BD47F1EBE2F5467DCDBF6
:108920008C1BD013D0DC9BBE131EBE5EDC0C135020
:10893000BEE0DCA0760C831C6247A29C622FA222C0
:10894000230AA2501CE0169CE0D2D268AED2D228F4
:108950004EA846F070E0D91C78D808D8F0AB781C47
:10896000221BDCEB6206569C622BC6DC14DBA05695
:1089700013860EDC50BEDE774277FABEE3A6426F66
:108980007E07A6FAD31EBBBE2766EBE31E0C13BE02
:10899000AE0C83A550E854670CAD2355BC410C1DAB
:1089A000024EE860E078E05CA01E0C1B9C131C22C9
:1089B0002B62BEDCDB0C83144742F21F0404D00B95
:1089C0007676130456DBD45F8C2F543F3E63BE5340
:1089D0008483B8580C2B410CFD8A4EE8203077E098
:1089E000689D2244781CEA31B60EB8AAAE3C68F8FD
:1089F000AAAE3CA838AAAE3CE8387C4AFC2878FEEF
:108A00003B09B8B8D84C578C47D8DE3EFE31B8F396
:108A10004484D8063020665746F07038566637D9F9
:108A20001CA6E853D91C230841B0CE6DB81902B872
:108A30003C5806F804A0965C1427D4B6E30EF62B37
:108A40008C63DC541F66E333D4144FA6E32E8A3ABA
:108A50005B0E0A061C2A4F0E7E8E9C0ABA60E0AEA0
:108A600056E346A38C431B66239A3A370C1F4E737A
:108A700084762B0C4B069CA206BF1BEE608DB8CEF5
:108A800008D528EEE9502E0EA0B8BCEE7EE6C6FE54
:108A90001BDC508C752A5CF65B752C552CD4DABE29
:108AA00026E37B661FD4EB46BE3F752C552CD414B1
:108AB00047BEE3D4141FA2E39CE04C437E9EBE4716
:108AC000DCD4E3DCA07E83A28C1BD013D0DCA26BB1
:108AD000552C4C752DF3BEB6AE60EE5D1E5C4C930E
:108AE000063003562FC6FB462746FBC68606A6372A
:108AF000D4BEE31ED3752CD4143FBEE3A2D414EB32
:108B0000D61B1C501CA63033A6E00D2AC6A6C6A64E
:108B1000F306F6C70BE0DC201FD4EBA0E0A28C1B11
:108B2000D013D0DCA2E0A01E7E7E43ED28D91CEE3F
:108B30002526DC10FEE0DCD0D07C70D91CB07C7027
:108B4000061C4AD36A2775B0AB3020DE7E2320494D
:108B500026E8D309CA008CB3F12E461AAEBCFA1A25
:108B60003A30E63A303CC61C3CA2BC02F6F6DE6B5C
:108B7000F6277CD90E7CAE0819BCF90EF6CF75CA63
:108B8000AE5851000E389C0A983CBEAE2838FC26E0
:108B900084E6C67C287E7E677E01CBCDC63000EEA3
:108BA000CC4371CC66250E22C8EE66A30B000000F4
:108BB00000000000E55CBB6100A3E55C8838FC6652
:108BC000E6876B1CC4E666664B095010841CEE01F8
:108BD0003041A478901C8C476A550E4DA43DA49D4D
:108BE000A48C1F7CAAB18CC1B0041D1425FEA55015
:108BF000EED44B4670B87C588CED02B070EEF0E0CD
:108C00004EE8286AB3B83C58A020BC30C1FC1CE038
:108C100000105B504B903BF3D023BD8E103C064CB4
:108C200023308006708C83AE1CE2EEEEEEFC5C50CE
:108C3000303CE6E60E9CF83C5842A65844D91C301D
:108C40002006861CB86AF3AA6A37C6E8A8B8D3F823
:108C50007E60BEB03AE006B8588C233055737C581D
:108C60004C3305BCEEE91BB8580CDFB05A3C06305B
:108C7000667E679CD0FE431CD03EFE53FE470658DE
:108C80000ECD90EE87B00EB85830505E7C067C302A
:108C900076B1B5BCEEB85CCA46A80C2BE21B1C2210
:108CA0009C5858CEBC30147C301C50BC5870305985
:108CB000E2B858E0D8A686251CC1B030E02D1404D7
:108CC0001D1030E09C58BC0E66483D3A44251C1DE2
:108CD0003C984D14987A30F6453AF6F6167A3016E6
:108CE0003C5804D89CA298A2580C9321382B4C5184
:108CF000370C33BD386520A30CB5374CC9370CB7DA
:108D00008CCD378C8F5E7B3091AEFC9C425D1CAE6F
:108D10004D32C1B0711C9DBC110C1D028C1B0CB3DB
:108D20001538838C6B4CF53B0CF53B4CC9376520F3
:108D3000838C653BD32D38DB4C41370C3381346554
:108D400020A3203C0A30836A7F3031E82D383B0C69
:108D500081356520C3B8FB0C3B8C678C1B4924060E
:108D6000A6A6B8A6A803B8F8E806A6F13B4924B819
:108D70003C0E8CA730CD8C2FD91CD532AAAEBCA806
:108D80009858889858653A4C5330AEAAAEBCA80C97
:108D9000571B301E0C0B668CF39C98D844D8581C7B
:108DA0003001AAAEBCA8C1B030D02D14A83060E804
:108DB000D53649249C98D848D858D91CBD1C090ED2
:108DC000042021386B4C778C5F0C1BBD3865209BD1
:108DD0003030E81B30305E172EE83CBEFCE8953A98
:108DE000BEFCD056E82138430C1BBD386520BBB80B
:108DF000E04936BD1C1314201538BB3020A8A8A8A4
:108E00006D7CDC100E304C66CF21B0DDAC49249C6B
:108E10009858B81CD04C1B1CD0AE7CA2813A65205F
:108E20009B3057BE5E2B2666DF03305466E3834ECD
:108E3000BEFC1CD0E81538630C276520CB4EBEFC69
:108E4000D0E81BB8E0301F43301F23301FE8E8E8AC
:108E5000DDAC4924F81C98E8B83C58880898FC6DAB
:108E60001C61001106DCD01C0EB87E584CE706F8D9
:108E7000425646BE47A6E606E6E646A39C98584CF0
:108E80002330804686DDAC4924B80E8CA76686E682
:108E900083DDAC4924B80E30C8E0C8CC3B66E32083
:108EA0001938436D00C1B020492495BC110C9C9821
:108EB000D84C3B4C1FAEBCD1A6D84E5CD070AEBCDB
:108EC000FE6D076645023040E6C8CC6D0266DB04E5
:108ED000B1703C30E866FB59364924A5BCB8D88847
:108EE000D8A84E68D91C1538734CD13E957CB35D1B
:108EF0001C8498A84936492478EEAB7C4A68251C26
:108F0000D91CB81B0CCB6520E36D7C06251CB6BBB9
:108F10001C307F6A93303A6A73302E6A53302C6A61
:108F20003378EA1FAA0A3C68EED91C21B0B30000CE
:108F30000000000049248C931C78EE4B255068B843
:108F40005884986D1CB83C06300F6A291A86D91CC3
:108F5000DDAC492478E0DCA01CF2251866301E1C2C
:108F60006ACF78581598EE8FB858F83C9C580C5F2B
:108F7000B80E95BC110C810A4C37587C7048840C93
:108F80002B88B0A11C44B8D80C23584898589C583A
:108F90004C4B1D3C4924980E1DBCB80E86813A8C62
:108FA000537C560EB858AE444D32587CA11CB8586C
:108FB0001C98BC580C5B30E61BD03B3A30E617E0FF
:108FC0009010589C583532F8E6C1B04CA066664CFB
:108FD00013061EA1143020E8E060B0303360B030DA
:108FE0003A70EEEEDADADAEEEE7CE041A4584DA407
:108FF000EDA4D8E05CF84A0EBEBE175031020E8CCC
:109000002248E30130028C043EAEC242880480BE96
:10901000202C51C0202ECC0DA241A9AA84F902C453
:1090200050020D3384537FBC3F00000004DC78778E
:1090300077A50400DC4E0DC0AD804070097E441061
:10904000226323144F8CCCC30DC912942379D33FD0
:109050000030004100E45C480640200180840B3071
:109060003417E33B03614413D323C1903331FAF443
:10907000E4D2CA44F24DD4908823743880DFCFB351
:10908000F3BC6C759792E288CFD3CE4060C1562175
:109090001E168C74E8237655D4B87088323931D5D1
:1090A000D193F0E04D472E1FB82F2C89617420C258
:1090B00040844410A0363513834E847F64D84E55C7
:1090C000E88080D274124C1BE360A307800F28CC89
:1090D0001B31841C91DC3E01FC279EC001316D8256
:1090E0000FEEFF13DFCFFBFC27D90F9E1BC43013FD
:1090F00072813CF7F73CF743182F2EE388A4033C1A
:10910000000010D544483012D070C5713003B0173C
:10911000470C3C12C470CC030D8BCF8002470C4D22
:10912000F348CCC44C7888871F871EC715335F84EB
:109130008F2341C0084013CF4688CC00253840CD4E
:109140007512080A0D21334073C4044383C700F825
:10915000B1C44CFC72FC85BFDB87C4040C232031F6
:1091600023715CC00E193400C6848914C3703CD1CD
:10917000F3CF90E150CE6192DFF120A955A34A15BB
:10918000A82A166262403C8777F8480491C33833B6
:10919000C3400431F3B0F7C9C4E4C88DBBCB34700D
:1091A00038E013130741C43C7324232378D1C43D12
:1091B000215E141F13CAC53884C4AC737C7CC8B547
:1091C0001012024080D844C84417612520B33D20C6
:1091D000C623FCECD36EC8C1EC0B5420F944001537
:1091E0004F1534551823FBF73284FC4C018B8773E1
:1091F000E1F81727FF0113C760D19278AF17C603B4
:1092000094D754508F8FF450E4E5A41F659A3D8A9B
:109210006BDFCB3C02CA23A3CA8DC94D8842132001
:10922000668633F3ACFC18FE43A28D0B11A2CA83F1
:109230004813144140001733CC0C0CB26D33847DBD
:1092400003C74F3CC48314F3303D14CA20CED191E0
:1092500010CC3F3CC03EFD2EF2C6F1EE98127337A3
:10926000D673F4480C30CDC980CB3483D88F2072AC
:10927000CA2033DEF32003C48A6D1458608219A813
:10928000C5878C047931ACCCF07340CC1EC97667AD
:10929000F2355B43440B1D38CF7ED0C162733F0A69
:1092A00001630E80B8B3007C8E3C05B0F4D203108D
:1092B000BB0030CD0058885CC574351A37C3D2ED79
:1092C000E2D03010A2633C03F10C4D0CE1E8CF304A
:1092D000FD1107723C7012948ECB9025A18C23094E
:1092E0001C480F8A036AC214130FE30300A3388BD0
:1092F0002AA04C03C431CF0C0CC02C0200DE0AE2C1
:1093000038FC494000C0001D841057195F3DC44E11
:10931000C47FC3FF5DD64BD524CE0358C8CA19629B
:1093200081D117FB420808B2338443F5FC414CCC91
:10933000125328C634B952B9CE0350C400C846F2FD
:10934000CE7FE00932713233F100402233870C8C3A
:109350002CC5C40123EF0B0725F653843401339049
:10936000CC4C04E415AFCECC013931C710733303B4
:10937000188101C831313E1E080700F2C38071FC1C
:1093800063C5C8C4AC85332246E31F3B380720833E
:10939000DC0741FC13C33F6F88F8DDCC5050D57318
:1093A000444C18C04C58F8F883CC7132C3C10C0738
:1093B0000692BD78413BC4BD8F1304B3F810FA1870
:1093C000F3274ED1C7C7C7C7EBA48C080081ABE316
:1093D0007B48B13013223AC467233F437632168864
:1093E000C0F0303F32516308408F12F357B0804BCA
:1093F000F0CC0CD3C0C4DBD8567F5D34F2430503F8
:1094000041460000020103044247000027242120B6
:109410004348000028252200444900002926230053
:109420004540000F800000981E19B0456C63AB13D7
:109430000D08B0C964F0B8C9640EB01D6088C96475
:10944000CBAD130D08B0BEF053ABB063840F0DB0BD
:1094500071643BADB0BE001D606902AAB03560D337
:10946000A5A6A6B035603102B21E18B00EBBAFB0D3
:1094700061603B930201B05EE0930F030151848869
:1094800008080176008435928C031201595A860827
:109490001301215E8E0913015184338E1301A99E9D
:1094A0008F141301715E8E0114015184AB9705096D
:1094B0001601910E008883900505023007455A94E5
:1094C000130200418A940103012E8603355A810C50
:1094D000034E68A8E828E08F141398F0E0840C038A
:1094E000410C511E900C03318A87120C0308CD5E8B
:1094F000CE0C03C15294130C034E2868A82B980C71
:10950000034EE8090299100F039586922D04B005C9
:1095100066870504715E84011207995E84011289D1
:109520005E8C0504A18A0000BD8A8513047D5684E3
:109530000E05870E0548015A9E1205140E05B550FA
:10954000B8E81102981E05B0296A96040175BCE0BE
:1095500094030106B0B162BF0306AEAEAE2BB12DCF
:10956000181E0548B0296A833F030635586B9809D1
:109570000688015A940E098823831206B0ED66BF4F
:109580001306155A833F13063558C30065A68F147A
:10959000079208B0C966930D0888CB8713098481A8
:1095A000568C020C8E0CB0156E870F0C88CB96056E
:1095B000041341743B8E01050DF9709502902D1234
:1095C00051842574BB86060FE03009999C1508610B
:1095D000004106982F31B02D62922D105184080859
:1095E000D578CB8B0301100182880325BEBEBEB0A7
:1095F0001D606666B869603102851310CC2308EDE2
:1096000004B10E94100D0F1210810E842D12B03182
:1096100066900F1413A50E0000751E982B310E0CCA
:10962000B0CD6E981413010C38EE238C03128CB558
:10963000514E70EEE8B902930803B0FA1BBEE8B3CE
:109640008910A06964EE3A460BBE3C1898F01B8E58
:109650000412F552840E12BD2A8E14120D9E9E1213
:109660009552890313015A8613295AAB4E2172ADC4
:109670004E88DB8705124E655A930F0351846B8E1B
:1096800001145184438E091351848808E17A851AA4
:109690000913555E94121113B0F9629413130081EB
:1096A0008A8E0F4552AA14134950356043AB1413E8
:1096B00049501D60B92EAD141398A0BE589BAF142D
:1096C00013495061607B981E3031E16E850E0F1496
:1096D000795A97050916BD0EBF304D18455ABF1966
:1096E0004D18A55ABF303C18E956BF303D3C1825EF
:1096F0005ABF193D3C18055A993E3C18F8AEB8E8D7
:10970000AEA8B902BF193C18BD56BF303D18195A52
:10971000BF193D18515ABF303E18C556BF193E18E3
:10972000E156001D92910518830504482394030F08
:10973000B0E57E8E070913D13E8E0F0188ED0471CE
:109740001E86060F0184BB00009D7CAB0000201C20
:10975000E2E2E283B87CD84C1F481344D83C98A876
:109760004451064DBCE27F410C8C3B8498A8448553
:1097700006880CCB53410C04840C1F08830498A862
:1097800009B8634EE6BCAEB90C004A545C6FD6CA49
:10979000767D4D453C8C92989EA4AAB2BBC2C8CCA3
:1097A0003AD1E0E7EDF3F901097C0E2B14242D32B8
:1097B000353E4763545A6B717C82881A91993245C1
:1097C00093779E28A4A620ACB94F30C8A3DCE761EC
:1097D000EC4209FC600EC01F2E52575CB265696DE9
:1097E0007177883792989EB0B9A8C1DA1582D0D621
:1097F0000EDCE8EF1A14E208F6204CFC286B2A0075
:10980000C88C2409E71892C29EA3E7274DE0489E22
:10981000ECB83C5808987CA8E04E70F8E085B5E0BC
:10982000FFA0B0BE001D6070E0FA174EA05CF6A06D
:109830006636761B26E0F61B4E2B4A6A56D4D4E0D9
:109840004A545C6F0820F66D7132454F61ECDCC004
:10985000A66B982A3A47ACCA63887C82987DAA2B6B
:10986000D67654DC1A20E80E777C0E0E999357308A
:10987000F3FC42F96052280114E237EFB9B2B2E0CA
:10988000141F1A3E155CBBD192FCED453CC8094D36
:109890002EDAB0B9A8C19E2DD677A48C716535D0CB
:1098A000E7FDBCEEC10295BE69CC886B825A23F0FD
:1098B0009D585C0EAEF0AE6E70D494CBE0A55043D4
:1098C00032EC4E70783C0602E01CEA603CEB4CA4A3
:1098D00091EE6E98AE6150AEA0FEA03E337EE000E9
:1098E0002800D58818B550B902B550B5504E70381B
:1098F000AE7828B868F8A8AEE8E0A04E6E60EEE05A
:1099000047710E834140424348700E0078464567D8
:109910006075E00017141110534C0F00A8869C725C
:109920005259911C1815121A515CCF96A94E9D766A
:10993000565A901B19161305575DD085AC4F9E984B
:10994000505B08000C0C0C00555E07770C0C0C00EB
:1099500041460E4E5155593A617E0E5E2D2B2A2FEF
:1099600042474B0052565A2062257F00373431302F
:1099700043484C4F53573D2C631D9A0D3835322EBA
:1099800044494D5054583F05643C9B243936337E3E
:10999000454A08000C0C0C00653E07870C0C0C882F
:1099A000EE61501BDA26F6EF1D64989417D44AFA3C
:1099B000EE58AE0EF09C4A5CEA271C505C0E0A4A38
:1099C000EEEEEE5C262666421FFA06E247FC4626CD
:1099D000E21FFC468C13BE70981D60580E38A60618
:1099E000DA661FFAE7461AB160F08898AE8C5385A4
:1099F00050A0B0EED33E1BBB85508C97A0B03E7BF1
:109A0000CB8550EEAB630EB07BF8615070B0EE5377
:109A1000630EB0CBB8AEF86EB7CC6F4E70B8D84C02
:109A20003FD88C27AD7062C102B8AEF86E6760CCCB
:109A30004341A4E5A8BD8C834E70B8D84CA7D88C00
:109A40003FAD70641BCEB0EE8F2BEE702BCEAE0010
:109A5000B0A8AE58711C98AEE0B0A558B0AE4E702C
:109A600078BC46063C68E078BCAE300560061972EA
:109A7000EE38A02E6EFE433E2F385E3E537EF61B20
:109A800056765CE2174E60EE0EF0386E334C810B6A
:109A9000C90ACEF0AEE0CE7EFEBBA118CC60B858AD
:109AA0004C608CA00841B0B83C58084898FCA8E02D
:109AB00046705CA0D4D4542FCE58E09CD251B5A3AC
:109AC000983C98FC58B83CD88C132E0C1B2E2EBCFE
:109AD000F375583005755830087558300758B8BCBC
:109AE000D80CA0C4D8584E30FFD8BC0E7CA0BE60A5
:109AF000F1585B657387A1C90B3F8F15B01A30A66B
:109B00007E677E777E8F1ED8BEFBA6DBE0D8A6F3ED
:109B1000E0D800A6EBE0D80000A6E3E0A95C98BC82
:109B20006D1EA95C88CBA95C08ABB83C588404E0E6
:109B3000044E70783C5A70AE38EEAE0EF0386E605F
:109B4000EE0C134EF06EAE7BD55C542B1C52F0E045
:109B50004EF0D460AE7038DCDCDCDC93D55C544B6A
:109B60003CDC5010F070F03BD4C7AE7038DCAADC9F
:109B7000DC7C94E36B300870AEE0DCA05C38521CF7
:109B8000AEEE6FAE0E7038D494BB5CF260DCE09C3D
:109B9000D4D4F2EBE048A670851458C15C4E708EA8
:109BA000783CC6B0C67F08CEAE584E3CE6BCEE78D8
:109BB0005A7AAEC39806374C098348E07806BCEE63
:109BC0005A3AAE5878E62BBC1AEEF0EEAE0C3306DD
:109BD00033AE2E6366E3AE70FABC1A3CE638EE3C58
:109BE00070662FEEF098EE41A4CC17266E78063CF6
:109BF000063C063C686E4435BEB8584898A8E0005C
:109C00004E1B4EBE5C501B2E7AD898463E5ED81C2A
:109C1000D4763654E3EEEE6BD86EEE4B2687D86ED4
:109C200026DFAED80E23D8AE2BD8AED86E9E5E5BA4
:109C30008E1E263BD8FCD86EA66E264B66CEBE1E68
:109C4000D4D4C34EAE98EE2E76767600CB2E7AD84C
:109C500098463E5ED8065E139E0ED8DCDC8E132E30
:109C600062F354CB98AED898FE1B66CEAE5C4ABF6A
:109C7000EEAE5C0EE66B3A5BC62622DE6EFA604EF6
:109C80001EE0C6C36E63424F66EAE32EFAAE4ED8BC
:109C90004E5C50EEAED8AE332E7AD898463EFA23BC
:109CA000D8465E139ED85EAE6E2E2BD8EE66D85C7C
:109CB0004E13228EF32EEED4D4D3AE98C1622EFA78
:109CC000AE5E1BB5A23ECE6EEEEE0EEE5A0EEEE688
:109CD00013BA4E9C4217AE8E4E6EDC50CE5322CE3F
:109CE000F34EEE94C963D4CABBA63BC3FEB7F6A736
:109CF0000E8E1CEE8A5C4A9766061B36E04E22CE1C
:109D00003EEEC21BAA260EC223EE2EFBDE338A6E67
:109D1000262EFB6A626B7E5BEE865A5E2A4EBAE0A6
:109D20004E709ECE68B8A606A8E07E78EE68B8A60B
:109D30007EBB4E7078FED8B8DED8E01D648CB5626C
:109D400098941FD44AC9622EFAAEDCCED86ECEF6F5
:109D50006026E63B66EE1ED44ECF66E076FA3B36D2
:109D60007E13484623B6AE932EF0BEF01E06FA8E42
:109D7000FB2EEE66DB8EB0B5604CA0FAA00EF81D8F
:109D8000620E6964EEB03D60556469620E556435DB
:109D900060696475624E5C2650E04ED88564EECEF4
:109DA000E05C4ED01050D050105090D0D050D050D9
:109DB0005CE0FAA00E8E2626065C4647D4941BCEA5
:109DC000E066D34EDA8C93DCD4239D642BDC9D6457
:109DD000D4D49D640ECE95620E9564DCD417DC95C8
:109DE00064EE4EEE93CA0A0ACAEAEA4A8C330E06B9
:109DF0000E46E04ACAEAEFE0BE6E8ED8988E4E2735
:109E0000980EE026CB5C626EA5622EFAAE045E135D
:109E1000081E1A6ECEE673CE5E7FDCD494856B2668
:109E2000DBF568A3B9685C336E66AE333A8EF32E09
:109E3000EE66539CE22B62E24F225C23AEFAAEE266
:109E40006B4E5C6A0E1C500C13A66E0E4C1B096008
:109E50008C1BBE1E1162228EF32E543FEE66D4EE92
:109E60000BEE4C2B2968AE6EDC909CFA9BDCE23347
:109E7000628ED89883268E7E9BCECECE626E0E0CDE
:109E8000396153AE7EF32E7E982BD8988EEEEEEE8F
:109E90000E6ECEEE2798AEE066CB8ED82695626E1B
:109EA0005A5E0E0C1BE1644C1F0160416AEE5C902F
:109EB000D010905010501050905050100B4E54979E
:109EC0007A103AD4E7543F148F94CF54FF9CD05C5F
:109ED0006B9050D05010D050101050905CEEE000BD
:109EE000D0501050D050101010D0D09C8B1CD0D01F
:109EF000101050D0509010DC2B5CD0D0D01010D06F
:109F0000505CDB5CD0D0D0D0501C9B1CD0D0D09CFF
:109F10006B2EFAAE8964B861500EF85EBB06BAF6D5
:109F2000330D62E6EB66EE5ADFE64FBE1EFEFE1E06
:109F3000FE1388B85E2EFAAE08DA77D164FA1B9861
:109F4000FE072E11622EFAAE3E5EBFDAABA606E623
:109F500083461BA6080E5E5A5C8A62228ED8988BB6
:109F60005CCE62AE4E4D6E422766EEE3D8A5608BA6
:109F70000160B32EFA0EAE0E26E6B35E57AEE56470
:109F80005C4EA60E6E3B08CB54F7D43E26DB738E98
:109F90007EF3982EBE333E6EEED4940BAE8EEAEA7C
:109FA000EAAE9CD086C6E35C8EEEF568A56CFAE35B
:109FB000D4BB2E9C822E8EB5680C376E8E6E2E6EA4
:109FC0001CA56CFA3B8EDBEEDB8E235EEF665E0C2F
:109FD0001BBE00B5600CCBD164496098FE356AA603
:109FE000EEDB8E29686E5C1B2E62F34226DCE08C71
:109FF000A04ED8B968EE75620EB968B03D60EB004E
:10A00000000000B0094648167616810B70C15A014F
:10A010000C10080120040114010401140120051290
:10A02000120F120D050D0F1219200C0F13140E0F25
:10A030000E0518091314050E140E150C0C10120938
:10A04000160114050F1514200F062012010E070526
:10A050001001030B090E0714121920010701090E44
:10A060001905130E0F12010D120F0D08B060303AD2
:10A0700070BC5C50100EC1B0AE307A0656A856D3F4
:10A0800049240CA08DBCF10E2170B8F0B00E4C2309
:10A09000BD701BB57069708D70B00E356069704C05
:10A0A00023B9701BB17081704670F84C1F48EB0EDD
:10A0B000B835606970AD7081700E626970A9708D7D
:10A0C00070F04E70F8280D729D585CEE615060EE95
:10A0D0006670EE38D494B34E70138CA0BEBEBEE052
:10A0E00025601B1D60A550F05CE0D4D4D4D4D460AE
:10A0F0004E7078BC26DCD4EB667038A05CE0217032
:10A10000B5701D74F0BD700EA970EE4E70EE6162F8
:10A11000842170B1700EA970356081648C27B57090
:10A120001BBD700E3560BEBEC9643160A970696028
:10A130008164A9702EFA0E0960C9644D60FE89031E
:10A1400005608C60F088B9706BB0FA33FE238888A4
:10A150005EF00E35608964B80E3560D164316005FB
:10A1600060F00EB8AE6160FADF0ECB8C1F88E08421
:10A17000E0AE88FE13485EF0B0FAA00EEBAD74E3DB
:10A180002E0E7AFE4B480C338C238488445CA60642
:10A19000E6B177468FCECE235C62EE570C0785641E
:10A1A0000EA6AE3D7A0C0D633960AD746ECE5C5A6E
:10A1B0005E26E6433ED454D3EE3D7AD84E3ECE6B77
:10A1C000AED8221ED8AEAEBEEB1E2EAE8ECE93D82B
:10A1D0003ED86EEED454B3EEBD606ED8469CEEE130
:10A1E00078EE132E62F38E42FA1BDC9B0CE389643B
:10A1F0000160A9640960D16449601E0560B05ED841
:10A2000098464D60A606E6A176B176DC6654EB5E14
:10A21000B5608C3BBEBE696431608C2B6964316073
:10A220004C87696466660075608C3F4E5C66503D85
:10A23000604C13BE0C60F0E04E6E5E546F94EFD431
:10A2400027544F14679CD09CE0DC90901090509065
:10A2500010505050905CE09094F3631C5D789C50DB
:10A260005C109CE05C5D789C50DCE05C5D785CE0C0
:10A270001C5D781CE00808AE0E2EBAFE43880C1B4D
:10A280008C13485EEE4C457B8C2BAE0ECECE4E5CD6
:10A290001050EE66F62F661B268EEED898EEEEEE88
:10A2A000CEEEF69F8EFB2EEE66DB4EEE98EE4C1B4E
:10A2B0008ECEEE8E5B2EEE98EE4C0BE6F7EEEB8C30
:10A2C00047884C1F48734463840CC38C1B842B88C1
:10A2D0001B8564436E8E00AD743B26F6278EB32E2D
:10A2E0006600B5604C5F98EE66006960696449601D
:10A2F000D8AE0E263B6EEE3BD454B726E36E4EEE40
:10A30000E178EE133E8EF32ED4CEEE549BD88E8E93
:10A310004E5C50D89C90905B8A8ABEEB1ED8AE4EA5
:10A320002ED88E1E62ABAEFAAEFA0B7E661E8E9BE8
:10A33000980C4F8C3B396023B0D898464D60F0D1D3
:10A340006449608C13F08C13BEF00B5ED8AE98AEEF
:10A350000C1F8C1F866EDAC3D8A5600C7B8964D174
:10A36000644960016005600C8739604CA0BEE04E16
:10A370005C6A560E8E0CA02300ED64FA0D63B04C9F
:10A380009F0E1E4E5C66D01D604E5010D0D0D01077
:10A39000501090109C506960F60D62E01CA09C6EFD
:10A3A000138E26F34EAEEEEEEEEEFCA0A2E0CED47F
:10A3B00054AB139C42E60D63B0221FDAEBAEA24E03
:10A3C0002E5C105CEE22270D622EA2F3A637EEEE75
:10A3D000EEFA9BAEB04A1C5090B562B0064E3055B6
:10A3E0007C067C30E04924B83CD88C1F881384D884
:10A3F0007CA8E0302D9C58A051B698DCD0CB06C08C
:10A400001000000000800000000000048080042094
:10A410000020030001080CC41431000D320003CCED
:10A420002B28900210003314900130021028400CA9
:10A430004070A2015039980332900004800000005F
:10A44000C0000580000000005002420AC035003004
:10A45000300000DC000C8A04000068CC39000000E9
:10A460001AA031C1030230B9C040000C00008C00BA
:10A470001303C680088000B32100000850C80032D2
:10A480000800088000080800040001D9200C80C8DA
:10A49000A024933920000000C38D06083068000313
:10A4A0003000F30125000840009013900343A64DAF
:10A4B0008E0C307003190000000003000000000043
:10A4C0003000030000003000C3D0000004C0004290
:10A4D00000380C20153700F7CA89886FC8CB02F303
:10A4E00033840090D00300000240D95555555505DE
:10A4F00095657116695AAAA9EAAA2AAAABEFAE0312
:10A5000054285A3FEFFCE3C38B000BEE2A1E80FC5D
:10A5100000AF02542196A9C091EB95E5286ABB05CE
:10A52000550AC467A25A0A99872352F51188FE4F2B
:10A530008D13EF6E4D0CBA3833CCCC2000002CDAE2
:10A54000555555551500155515005555154055557A
:10A550001515551510001000000000000000100037
:10A5600000401040101560D50CEBD10C448A12123B
:10A57000FFDA8C88221341418B63680C8859206272
:10A58000800C302003C0083E2CC100AFC4C0F8BC12
:10A5900007B3CE204F11138087FC110AA08A8028B0
:10A5A000B820C938808C02FEECC17FFB38FF40C266
:10A5B000BBCFE3684E4C4CBCFF4E5CA80300953902
:10A5C0002292DDDB4B2FF470010F3FFFE12040F2C0
:10A5D00004C631E2C8C8FF310AC88CCCDF8720012D
:10A5E00009C9BFF3EF0B1220131124C40889E01B23
:10A5F000484322C4008F24003E46402C26233C3F83
:10A60000800314D0E76361134F1344343619314D7E
:10A610003B442A400129924FFE51D23C70212838F8
:10A62000CCFC3E400C04506029064CDB60F74E0128
:10A630000C002554D8F36063F7F187AAC1FF8DE3BE
:10A64000224BDC7136EE03C5084A8E288C927410BA
:10A65000CD0420812BCEEF8983040040B74FB00793
:10A660002010224988B04ED24F861258EFA11D0FFC
:10A670003BC0323C3F11CCF21C6F974072FB423D15
:10A68000B51F02300004E3844B12F4760BA2788CE1
:10A69000B30948006262173B0202862D52B8FF11CF
:10A6A000E25E5D50B2C46D0A100C403040866831E5
:10A6B0002658594D241452330029410718240720E5
:10A6C0002900A48002C0C4808CFB0B9522000B786B
:10A6D0008E00AC928400A75423CFF8092044F630B2
:10A6E00043C0B5EE5E298FF0735A2323CEB4001118
:10A6F0008C3CCC0B480C4442BC90393E9320082142
:10A7000000203D460000040040000010000004044A
:10A710000001000001400000410441B915376CFC04
:10A72000D1170304C3CC500C0C330860C4CCD0CC7C
:10A73000800411230A3FC6C80080FFBF78EE8A3F1D
:10A74000034C0322CC3401304C21002330108028EC
:10A75000C33062E2500005C01088C0FCA30438C5B5
:10A760008424B34DCDE02B2F043C123028DE40383A
:10A77000647D1374C6374208403EF6030000C140B2
:10A780002194C83E312220022085006B84CEC8046B
:10A79000599D5316097D7F71D8C532E1463B8038FB
:10A7A000133040C785224E5523DD0E054F4490CC13
:10A7B0001CDDBFB88B44A074125022129130970355
:10A7C00000767FF74C17DF8445CE98F2D949140202
:10A7D000C42012513222C900048C4A3B4BFC800336
:10A7E000050B0051482B0E31EC502DF0DF38C8130B
:10A7F000ECCCD8513D300451FBC73EF37F0CD00C5C
:10A80000441348AD7056390C51844E584488A18089
:10A8100095BCF0B3D5888A3E23E6D7ABAA0A704D23
:10A82000A47E7C81BC8D8CB0AA39887309504E5BA4
:10A830000CDF98EA2DBE0AFC4DA459A4AA0A582997
:10A84000A48A41A4CC57980647662F022762130AB0
:10A85000AEFCCA7004B00A8AB0CA70E5A47CE21FDC
:10A86000F6B362BF62ABF62BF61BF67F0C5B980A61
:10A87000468D8C59A498AA58081304B00A7C060F78
:10A88000662F02EF62DBF5A8B0AA70E5A4EA987023
:10A890001CA18C98622362626E6258B06A775582FE
:10A8A00046FC708A980A29A4BD8C6ADB20B07038F7
:10A8B0009C5898700E388E8E1CB63FB6DCDCDB02DE
:10A8C0007B4AF01C6A101C02BBA666700A4EF09808
:10A8D0007CAA698C70389C98F0467078A6682E66C1
:10A8E0000DBA6670EEF0EEC34670781C10701C0A4C
:10A8F00038E039883E37FEFEFEB183980A7CAA69AB
:10A900008CFC4DA4AA58B00A4DA4AA0A70E5A47CF8
:10A9100022DDAFE078E64E30C058708370383E9349
:10A920001CEA277CEA2371841B5584C606B0666F37
:10A93000E07EEEA0FEDC58B098701CB0FC6A6F7C24
:10A94000705584DE7985AB00000000000000000037
:10A950000000000000B0702E70380E3B55849870D7
:10A960002E58AEF0E07858EE8B1598EE810A4CEF39
:10A970000C27D588671CB1182BCCC3A918AEBC30E6
:10A9800076767627D588437AFA851406DA1A300661
:10A99000098366E64670787066BCFA38D884D8F0C9
:10A9A000BA3A301C62027CA23C0E3A300A7E27EE94
:10A9B000EECBEE3C7066EEAEF0EEBC663FEEAEDC8B
:10A9C000901C3B3C2606467078A6681C02C4BD8CD1
:10A9D00009B81D02B8463C584484B0E06259A66EDE
:10A9E000E0C461A4CAD844D885A43C0AED1ACCA01E
:10A9F000D5886A66A08CE746E000000000000000F1
:10AA0000386B3823380338E338C338A338FCE00008
:10AA100038E038933873385338333893387CE03C17
:10AA2000E07CE07CE03CE086EA667038CAE086E6DE
:10AA3000667038C64B42EAEAEA22E2E61FC61BC647
:10AA4000360A1B261B62620A707C3020FCE0AAC317
:10AA50007CD80CE92F758879A085140CCD071902D4
:10AA60007CD80CD12F758841A4F80C83E6DDA9654C
:10AA7000504C1346261366E8DD8CFBE61F26E8657E
:10AA8000144C1938655026E8E55C75067858EE8751
:10AA9000CC1F41A4A1A48584CDA8884E66480B157F
:10AAA000981CEE1B0C7B810AAE668F840C731B888E
:10AAB0004E704C47CCC98F41A4F8CD84E844B044D3
:10AAC00070198C4C27B066CB95A47CAAFC61A47C41
:10AAD0000A4CA9A76550E62398ADA01D0245BC11FC
:10AAE0000C711C2DA84CAFE0390C0860BC580CA0B0
:10AAF0000498DDD83BA188B030C570CC1F4C1B79C1
:10AB0000A055C42DA87BAA0A584888F5A898AA5829
:10AB1000334E59A48D8C986ACFE0AA8A700A7C3093
:10AB200083FCE0AE1C8A700E7C3080B31DA44BCC3D
:10AB30003F4E70F84666E8467038AA0ACC57E213D2
:10AB400022E21322E2132228E04CC98259A49DA4D8
:10AB5000AA0A29A4AA5839883E5F488C337EFEFE93
:10AB6000FEE3B0E098EE4DA4E5A41C6A4F06E64E65
:10AB70007005BC95BCCE581C0A59A43988FCEE98C7
:10AB80007C1D88EE7CEE6A461746363606277676BA
:10AB900013266A698C980A84F5AA584A174A4A23E8
:10ABA000666262E6E6E6E61322CA101C0A986D8C1D
:10ABB00098E0B9844C1187AE41A444F8E633E5A887
:10ABC0004C3748655026E8DD8E30DADADAEEEEE012
:10ABD000B02BB03A707A258CF3B02BB03A707A254E
:10ABE0008CA3B02BB03A707A258C53B02BB03A704E
:10ABF0007A258C3A3A3A7CEEEEE0B0703C467CE046
:10AC000066BC1C3A3076F6E7E23FEAC3666AAF03F9
:10AC1000222222227B9C229F224F3A3A301C22275A
:10AC20004E4C7F488EA9186EBCCB3A3066AF7A7A0C
:10AC30003C1CE044448641A4CC3FC6BC584C1B4D50
:10AC4000A4E5A47C82E2DFE237E2AFE223DDAC934D
:10AC5000F68384763CAEBC9C98161C66673C0E2935
:10AC6000A48C29A54E70AAE03C0EBB59A4A3E2E730
:10AC700036C736C739883EA74C2FED1848234C3BC2
:10AC800041A44DA4DD8C4E70E0E5A4884B7D9C98DA
:10AC9000CCBF4CAF4C9BCB5C42EE2B0E4E701C4A93
:10ACA00033AA7C8E8ED33C58681598EE9B0C1FC43B
:10ACB000934C7B8CA758B8E683B85898BC30E64BC9
:10ACC000E0C81C0A1DA4A37D9C8411007EFE4B8D50
:10ACD00008063064069B8D901C0AB8E6B38A636A46
:10ACE0008686A644D190EE60810A4670CC2FB85873
:10ACF0004C83B80A38AAFC0EF8FCAAE8AE0930ABBF
:10AD0000EA0130091E04CC7F4C6F06984C8D900CE4
:10AD1000870ABD8CC102CC330A0238BC3A30A6B6D1
:10AD20003A30FCE64738AACA0C4B8A3B384AD3086B
:10AD3000EE41A43DA43DA4AA0A559CEE530C3BEA67
:10AD400049A4E5A4D6E63342EAEAEA22E2E697C657
:10AD5000EAAD3CD86A8C8346425366985846704B9D
:10AD6000C63673A2A2B3AA62620DA48308AD3C8466
:10AD7000D8064891900AD8662702331B061B04AAFE
:10AD8000464223666262E6E6E6E61322CAE641A48C
:10AD9000EDA47CC63CFAFE8D8C59A4CE7C8D8CE54E
:10ADA000A4D8840C1388D88D8C980A7596190856E7
:10ADB000A08A16CCC3468B02A6588C3B84980638D2
:10ADC0004A4B0638AACA237D900A499646BBEAEA4E
:10ADD000868638E2AAE2270DA48B462222421B6611
:10ADE00053A2A23B047D905841A470986627023379
:10ADF0001B061B08AA0DA45697E6567FE68AB0AA42
:10AE00000C1322EAEAEAE63C8D8C9825961C903CCD
:10AE10001E98EE6A21B0001CF61B101CEEEA3CEAFC
:10AE200023BE2F7B3CEAF358845C4E7050FADA9CC8
:10AE300030583A30E6575CDA22A3E5E200D0881CAD
:10AE40003A308C97E63A30C61FE663E60EBC427C89
:10AE5000A67CCA70BCA6F6F6F6A33A3A0E303C1EA3
:10AE600078AE7E3A3A306A677E8E8EFE2F4A2F4445
:10AE7000E34A97BC631C06461F4EE030DF0647C618
:10AE80003C020ABC059AA6FCCA221C70BC0E98AEF5
:10AE90007A30EA8304D88C1B8408D86A3F8E8E0CE3
:10AEA0004F4A777C8C173C019A4ACF48B09C108C53
:10AEB0009F0E3C7A7AFAFAFADAFAFA9C98FAFA9C35
:10AEC000901CAA08E0781C101C0A70383CE6359AE1
:10AED000D5883ED37C62588ACAFCCA0E4DA459A4B8
:10AEE00098EE6E6E1CE5A46E1C6A578E8E986258A2
:10AEF000E24B4A871CCE7C0ABCA34ACF4670CE7C6C
:10AF00000444E0441CCC1F4C3BF80E38AA7CEAEB0E
:10AF1000C8E247C4EAEAEAE66FC628AE4A7CE8F827
:10AF20004666E8890AC6369B4E7048D3C44CA0F8E2
:10AF300046E8CC5795A43C0AED184435BEA918DB69
:10AF400036AF335836C7369903CC1F4CA349A43DBE
:10AF5000A41DB43C3E6B980E4670110C1B19088C56
:10AF600060D91CB8492676C321067858EE319EB8C0
:10AF7000AAA81598EEA19268B806FDBCEE3BB80EE3
:10AF80000801AC1B95BCB806EEEE787CEE0CFF78A1
:10AF9000AE3CEE1C4DA459A4C1A46E1C6AA06E1C4C
:10AFA00058EE8D8C1C98EAA0AE4670855201AC0C10
:10AFB000604ECAFCAA3C7EEE1DA0EE3F706E85502E
:10AFC0000982705838EEF0982606C3E08E85506EE0
:10AFD0000801AE41A4CC2F46CA4602B8AAA8E08C0C
:10AFE0009F061CC3300B0604B898A8A63CB0FC1CF6
:10AFF0001086BC5C221B29CA30E6D3E000000000AA
:10B00000382338F338C3389338633833387CCA3C34
:10B01000B3FCCA7C933CCA7C737CCA3C537CCAFC9C
:10B02000333CCA7C13CAF01CE03CEA7C23D588225E
:10B030003803389338633833380338D338A3730070
:10B04000385B3833381B38EB38BB388B387CEA3CFC
:10B05000EB7CC2D63CF0AA0A6E701C1BFCEA7C7327
:10B060003CEA7C537CEA3C337CEAFC13EACA47F0B6
:10B07000983EAE4670E011A0EED3A5A461A47C1D5D
:10B0800088E6132E698C980A3C1C2376DCDC76E378
:10B090004E70786E682E70E638E66670E6F0E6264A
:10B0A00066A7E6AEF04EAAAE38AEF09870384AF019
:10B0B00098A9A6980A4329A44685A47E58FEC74CA1
:10B0C00013C809824E1C70786E700638EE2F30C09F
:10B0D00006A04EE0CC8795A43C0AB18C41AA2DA8CD
:10B0E000669FE68BE841A4CC2FA1A4D84A2709503B
:10B0F0001B29A4EDA47CC4483BFCCAAED851ACD8F3
:10B100008AAE06B7662F02976A833CC9AABC08308C
:10B110007A76EF3C7E45AAA3583C0A4DA4EDA49C48
:10B12000D08D8C98E041A4AAD8A1803C1BD588D8AA
:10B13000063F6660021F62607C8ACAFCD83E67D800
:10B140003CCA7CD8447EFEFE1348E6170A4ED8E07F
:10B150004E70381CCC17E20AE01CAEE6BD9E5A26A3
:10B160008F263B301D7C44D1026666FC084DA8C585
:10B170000278101C0A703988E62709503BD5883EB2
:10B180006F4DA4E5A47CE21FF6D3B06ADB11A0EEFC
:10B1900009829C101C3020F0B070660A38D88408F0
:10B1A000D8F04E70786668C4B18C0180BD9CC10235
:10B1B000CC53AE0EBC30E04DA459A4AA0A707C302A
:10B1C00021FCE0C6C2A0BB1CCCB76262627186CC17
:10B1D0008F1C23A237A2A22FA2E0A2A2A2A2A2AEFB
:10B1E000E06EE0469C5845A4AE58707C9C98E61CE6
:10B1F0003084FCE0C98C8ECE5C581E99A49EFE5B08
:10B200003E3EBBF5A891A4CDA883FE95AAFEF75CAF
:10B21000224BFC261CE2CF8D8C8B22A70422170820
:10B220008DA4300F0C2391A453F5A82691A48DA4CE
:10B23000CDA841A459A49DA4698C7C698C0C63FCA5
:10B2400061A40A4DA4DD8CF846E8C502FEFE37CEA7
:10B25000DC95A4BB5C62439CE2B790FC5DAA628370
:10B260009CE26FD0BB8DA4FEFE33FC261CE20FD007
:10B270001DA45378EEA091A478CECE68C330F0AE72
:10B2800058782366CECEEEE798AEE0F8261F66E04B
:10B29000044E6EA05CE070CCA795A40C133C52D871
:10B2A0004A431BD5883E33E6DF09503359A4E5A451
:10B2B0007CC4488AD80EB0CA70AED851ACD832AE71
:10B2C000724B06AF662F028F627BAEE3A9184EAABF
:10B2D00058AA0C41A4B0AAD80E442BE5A84C3F7242
:10B2E00098121B0ABFAE707C066550A01C4C60A66D
:10B2F000E8B00ADD8CF8E0C41BC488CC27E5A403C1
:10B30000AABC3A30F6EB3A3076EF7A76E11B488CFD
:10B31000A91A7ABBA24BAA626266700A387CA27C28
:10B3200082E2FB2222A0F62BF61BF64FEACA8DAC76
:10B3300082E25322223BF6ABF69BF68B29A43CCA51
:10B34000E0E2EBE2FF36EF36DF8C258F8DAC8DAC83
:10B350002237484C6029A429A48C173988ED1AE2B9
:10B360008B8DACA253AA101C66700A38FCE0A27C3C
:10B37000E0E22FF66051AE7660EA8DACEA76DB0350
:10B3800004781C10581CFCCAEE30BF26AED8666B81
:10B39000D8AE7070383E437E1E1C6A237C6AE74A32
:10B3A0007F1C8A8AA6B63CCA087C7E137CF03B0CC4
:10B3B000234A3CB33CD84670D8E0B083D813AEFCE7
:10B3C000EE707C1C0A3988E6CBD5883EDBFCAA0EE1
:10B3D000584DA4E5A48A1CDA7C0AFC6AB74A574691
:10B3E0001CDA707C0EB0EE730C33466E8D8C3B987D
:10B3F00008231C980A7C8B3020061CF86AF3B8E0FE
:10B400007F61626364650060060405010C1D7E0DAA
:10B410004EF05C90308C3C0EE5A41CEA5730051CC5
:10B42000426AB7C1B06B3CC1B0E02B6E30051C4224
:10B430006A9F9E301F0C23E8BE3726BE1FE8EBE054
:10B4400020DE6DBA5E270C71B049241CE5A43C8E49
:10B45000D91C7C5675B0AB3080A330C08B0616303B
:10B460003A66AB302C66A3302E66F7304006B8D86B
:10B470004C5F8C4FD8DC101EDE7E3353D8E8302072
:10B48000DE237EBE7E70E8E0163020069730600630
:10B4900073A6D844D806B03070A646A0061B4E5CF2
:10B4A00090101C30663322E3303A5B3C56363B0E3C
:10B4B00041A4C1A41C426A60FC5C021DB48E9C586D
:10B4C00006164670307F66851DCE0E1C7C66DD8FAD
:10B4D000FC0E1DB48E9C58467051B473E0200C6075
:10B4E0004C3FC8CC37486D00CC603080E666FBE04E
:10B4F00030107030FDF09C4ADC909C905C901C9069
:10B50000282828E049246E1CCCE5A66EC9A6381C64
:10B510003CEA6D591C387C0EF87C0AAE28B87C0ACF
:10B52000AEE8787C0AAEA8AE9C9868E0E6251CE6FA
:10B5300056069C58B87CD804D83CA8F6F62F468707
:10B540008CE70C23300BE08C273077E03087E0303D
:10B550001C66273054E09D580CC92289BA84B898DB
:10B56000A82B88B898A80CA78CAB307F069C98E6CF
:10B570008D2666AF652083B83CD808D87CA8D92032
:10B580007924BD2025241D0239B478FE37FED91C4C
:10B59000B81B09B8469875B031B8638C41BB41A45B
:10B5A000198C4E70D92041A41E8EE5A41CEA2B6E86
:10B5B0008DA41E46700C1B29B8E05CA078A0FE7B11
:10B5C0009E60FEDE7E5B8C4BFE301A31B8B37E602F
:10B5D000FEE0D4577822AF145762DC5058D4A099BB
:10B5E000A4130C778CC37EB77EA7C314B794A70CA3
:10B5F000931CA0301B31B878F65329B83BA08DA41A
:10B60000042BA08DA4088D141D02301C9C5899A6F3
:10B61000307F66937846977EFE2F410CBD8AAE8DB3
:10B620008C29A44670AE68633E236520E3AE99A4DE
:10B63000BE008B1E41A459A4BE1EFC1CD08D8C7E66
:10B640000723781E9ED91C5EA0BEB8E3301FE830E9
:10B6500020DE7E6F1E3E5E23E8BEE346F07068E0AB
:10B660005ED3B8580C373CD888D87CA8469C98063E
:10B67000307F667F781CEA3FDC10FED91C1B09B8BE
:10B6800061B6851CDC10FEC1B051B6C98C9C9870A7
:10B6900041A41E30F19C5899A4B09C5899A4AE7E48
:10B6A0006815BA4E705C105CD0100EB8B03C06FA4B
:10B6B000FA7C4638BCA606583C28E0E6174E7009CE
:10B6C000503344A180AA70040A4DA4EDA4D80C27DD
:10B6D00004D8330804D88D8CB00E3988E603D58899
:10B6E0003ED7AA0A704DA40CEB08EDA47CA24BAA8D
:10B6F000626266700A387CA27C82E297E2EFE277AF
:10B70000E263DDAC4BB0E60F700C4B41A44E70E829
:10B7100028DD8CB8584CA0D5885FE27FE217365FF1
:10B72000364F59A4E5A47C22D7E38DAC0BEDA47C65
:10B73000563C8D8CE5A41C4AEECE8D8CCE7C63E508
:10B74000A41C4AEECE8D8CCE7C1BA6FC586E1DB47C
:10B750001C980120C3AEBCD91C0C733A3A3006A623
:10B760003C2EEEB9BC04D5124D140912D91CB9BC3B
:10B77000CE3C061EA114B81CD0E8661EA11463A618
:10B78000EE1C1084101C421F02889C1BDCDCB6EBF4
:10B79000E6161FDCD64E94602213E2B6F30EF88C48
:10B7A00017B858B0E0EE2798022398AE4EF0E0CEDE
:10B7B00070989801207B0C3FB858B0AEBCE06E4D3D
:10B7C0009CCE0592810A4404040C4745A4E5A45983
:10B7D000A42B6E2DB46E66E66ED91C4CD9B0D9126E
:10B7E0000C23EE58EE04D80C23080408D8E0BD1C46
:10B7F00018120F0D20E000000000000000000CB93E
:10B8000062204038238038C4F800C4039D1033D42C
:10B8100010D0CC0C0011802C2E122151C04411717B
:10B820003333809043A21A1F0035802093C1477F95
:10B8300020C4A3612032E2CCA3C838491C524981FC
:10B84000304443C8C64304224B1204F1EB003038A5
:10B850008431000000A00091869B8CE3321070D0F0
:10B860002A8348F420B806B3F836E2C90F0A92805A
:10B870003D86330033E3C94D03DC50C1832303000D
:10B88000440400300C00C07C373B280C0A5359CCD0
:10B890008A6892C4BDCC0431BD4C0C0E04E2A07881
:10B8A00038E00326143003DA203E180470483C4B7D
:10B8B00040E000002920CD9C84FC92EE2E4F87C0F2
:10B8C000804CE14430D00F461263E483E0384E10E0
:10B8D00086E1330334141258D131B2348A104D400A
:10B8E00004C0A0A20894D3206A153E053D0BE132A6
:10B8F0002138FCD7913944E6109943648E7A557209
:10B90000B4EBE27EAA2FAEEF8804E9AB701248C414
:10B91000C87675C4BED2C4D03CC8E4E8E2E1121ACD
:10B920003180CB4E02C258F8F06F8E0808A57D6DAD
:10B9300041C308EA1433A4015FE083F2604382004C
:10B94000C02C50CE0743710E6E4C8FF7C40C0D0601
:10B95000211895C54C4851A37B8DCE8DD7D40C139F
:10B960008A5A851332020C836C3854C8030C2CDEBF
:10B97000D1C404F37FC49C46D74D41334CCC3C0F1B
:10B980006195D01805C2D2A0C47A84C1E3121ECD3D
:10B990004EB838910C51A57DA23EBE8C3DD2704F61
:10B9A00060813B152E2DF67C3C70BC08A456179484
:10B9B000824F240AE00A40330108CF23F240F808FE
:10B9C000BA08D92008553CE038ECA8FA0C5021C43C
:10B9D000722208C7805E0808CFE1608E388E16623A
:10B9E0000B622F880833C20F01E7A0080328232227
:10B9F0006060FE084B0087B8C3913F2759227B0047
:10BA00000400008C00444400C820CB0DC4CC8C281A
:10BA1000C404008C0C4AFA0011110088093E06404B
:10BA200088508FEFB82BA0880F0260824D3180B90B
:10BA300008E01A12CF000522EE0741338C3C00418A
:10BA4000F0F3DFD43ACAD5C843078D40F3F3004979
:10BA5000515BECD038508380486C28C91C1132806F
:10BA60008C2CCE8CC094688C8B3B003040FD0C49F4
:10BA7000520D500D40145D55373324C34902C3188D
:10BA80004A4C50D8821B6449133184331103820419
:10BA9000D0C03C09CC4B0EE0394F8EBBB33EBE0745
:10BAA00049EFF1E22100414403880F230F051024E0
:10BAB000F3F30F015540C544CD03013C13FC0C4882
:10BAC000E4EEAE11E1816ADC861EE11086D2ED2340
:10BAD0008788181116CF704444301ADC878313B856
:10BAE0004C01847421983DCDF02034C9E0868D014D
:10BAF000008580438D30C40C208103604861F4FFD1
:10BB0000000000004C71B204FCE0180143C461BCA9
:10BB100013D30422336110447C7C4CF4217B0C1F32
:10BB200042FCC4C470D7F14CCCE3313821E310306F
:10BB300081F11008040CC2DEF228DFF9611C20300C
:10BB4000D50148E23A7B1D76D411D30434F777351A
:10BB500000B1C4714C2C48F0C74F128D33C2FD0D9B
:10BB60003131A0301310B1108010200B030A302A9D
:10BB70000A3204AC608A38CC3C23C2CC4C800A32F6
:10BB8000C1141333F18E22020C2222327131E443AC
:10BB90006ACCF771203937EBFCD4DF4C312DCE1055
:10BBA00032CE880C41CC30830236DF5B91D1B8C1F4
:10BBB000E4008D3C4D0F140E4A4C2007AA71DB5156
:10BBC0001DA342A0C3FB102632B21ACA083200BC21
:10BBD0000C008F0002D0805EC834233310F30F7343
:10BBE000DB2E0DDFCFF152F7D84B123A30000FC5E4
:10BBF0003043CBC810240C3341B4E43F000E004066
:10BC0000193F0097013B01C60A430AD2057C01D2C5
:10BC100001520A19008809B409AC0D5B0D630C16BA
:10BC2000016907F7037206B20E6205730E3606ACA1
:10BC3000080B0A7B0A85010303AF02B5068600B133
:10BC40000DE403490F530F5B0EC30EBA062D085FB8
:10BC50000E690E2F08050F2C0F350173035703C013
:10BC60000C0400AC009D03B809A300E306A20B2F4F
:10BC70000AFC00F7012001290132023C02CE066CC9
:10BC800000009319050B0C030B8045628432200ED3
:10BC90000306201418052D8D0F0F1213010B80556C
:10BCA0006A8E0306201418052018032D851A09131F
:10BCB0001001C870F868385C581C0E38AA28B044C7
:10BCC0005D5C385CD8284C9B5D1CCC274C09820DF0
:10BCD000FC0E0F20120F0F0DF1FE80BD6A981209A5
:10BCE000040D0581408001620DFC04151020060C36
:10BCF000F1FEBF0705124E78BC067CC6007DC68EDD
:10BD0000130110A9D09868F8F67B0DFC0B051903F8
:10BD10000F0405D9FE009D0E809D66BF0E0E3D18D6
:10BD20000B802D4ABF0E0E4D180B805D4ABF0E0EC4
:10BD30003C180B808D4A870E050C01F9C41379C499
:10BD40000C1B06434E3005EA6DCC66A606E0980F44
:10BD5000140179C40C1B2E53468D8C9C985606F505
:10BD6000C4B94A851A09130C068889E8B08BBF0547
:10BD70001A0913C15C4E70783CC62B0E1B841E3012
:10BD8000107046F0A1144E708C60DE9C7E7E2726DB
:10BD9000D4E30A061E5C422FFAA6E30E8EE0E1C44D
:10BDA0000459A4EDA456E63F3005426AAF089C58FA
:10BDB0001C38FCAA0A7C28E04E703830081C901C05
:10BDC0000A838D150E0179C40C600B801162940FEB
:10BDD00012010B80696660B0307CDADAFC3A307CA4
:10BDE0000B00E00B00E0D05C3066603AC60E300617
:10BDF000A075227E477E59F37E19637E0D4EEDDAE3
:10BE00003CFE4E66A63A5C105C223730C6E3692ED3
:10BE1000D05C30C6D7CC2B71CC66D3550E7C1C3091
:10BE2000060E7A30EA592FA6D3CCDD0E5D1C4CDF0E
:10BE300071CC66BFE92EBF0E0E3D3C180B80714AD7
:10BE4000F80E30E82BF80E3000E6AE6150600E566A
:10BE500037300306E3AE8D080626D3E07E7E895395
:10BE600060065E46FAA056607CA647FCA62FFCA69C
:10BE7000B5A2E10A814081C866BFE6856813A36662
:10BE80003168C66687E61568D34BD05C30E613E0B0
:10BE90007CE046E098E0D91C788C2B84D8842388F9
:10BEA000D888D8F0492660A0D91C783CD888D8FC1E
:10BEB0009B81130F100B80096A0B80F96A0B802598
:10BEC0006A0B00CD9E0286C6E0BF0E0E3E180B80A8
:10BED000C54AD91C30126A5F78D88C1F881384D861
:10BEE000F06330706A63411C30186A9D7E4EF00525
:10BEF0007E78E2D3411C4CC76100D1441BC17E193E
:10BF00007EC676C3A5D00C60C6762330EE13469667
:10BF1000864686AE0E7C0A85D026E61C4E8223A677
:10BF2000A2A2A21F26E386EA02AA0AEAEAEAAACAAB
:10BF30002AE0856813E0A6062658D944E0EB5D1C8C
:10BF4000214687010C060C0312B830FF3CEEB94ABB
:10BF500087010C060F14130B80FD6600203C56066B
:10BF60009CE23BA0005D1C21463087E099050B1444
:10BF700005070B801D6681408488ED64BE58300241
:10BF800089408808AD402570BE981D608CA7FE1FB3
:10BF90000E5B0E300555703BA00EAE00D164EE89ED
:10BFA0004C690208A140257088A393100C03100B64
:10BFB00080696E9807120C030B80C162863E3C18A4
:10BFC00015C845CCB87CAA3CA845CCF5C4CEE871D0
:10BFD0001E5CE6A616E61376A6E6E6E6C6A6D4142A
:10BFE000A3E09828C488C4FD7E3E4E302C5808300B
:10BFF0004070387CE0304070387C063CA6BCF0E0F5
:10C0000059A413A63040562B3001B6166660A5D051
:10C010000CA01C4A2A704E5CAA0A7C9C4AA606F018
:10C020007C70383CA606BCF0FBAE0E7C1CAAFC0E55
:10C030003040562B3001B6167030EF06383C662380
:10C040007666471C4A2A703866F308AE0E7C1630B6
:10C050000156BF0670F038665BA6360670F038668B
:10C060001B062B1C90D0061CE076173670383C66F9
:10C070008B3001763F2BEDA45626E66630075A1327
:10C080003AC6F306E6BCE2667CE62B4E2E1CEA8539
:10C09000D04666064B66861C82A0A2A27BC666A519
:10C0A000D046A063044E70F8EECE71C8700439D04B
:10C0B00006B0BCA6700C1F08B30C60783C06B03C00
:10C0C000063C068C3BB958BC70B95A3C70E06EA077
:10C0D0005627FAA6F330030C1B6608468EAE608D19
:10C0E0000A304056A03001B616E0041308081B04BD
:10C0F000044E7038DC901010102884444E5870386C
:10C100001CFCEADCD0BEEB59A4EDA48A1CEAAB0A05
:10C11000302C6A1F48B3885E5BBE980C23AA3C1B78
:10C120007CAA581C6A3005426AF78A985E630C2B19
:10C130003C58BEC37C1C9010CB2E5F1C38FCCA7CC4
:10C14000288C6F0C0B0CA0CC23D5886A41A47B0CE7
:10C15000A0986815980EEE734C670C771C9DA47C14
:10C160000E7C0AFD1A0DFC0E010D05D9FE83051289
:10C17000140507884B8305120C031201840B80A160
:10C1800052E54C0CA0983C063C4C3B0C17060C139B
:10C19000463CA63C9C4A0EA04E2F8C7B5C628E6671
:10C1A000665C1BFAA642EB8C13BE600D544924F862
:10C1B00028AEE8B5BCFD5A064C2B48B03C06CE7CF8
:10C1C000A6FCEEB0FC061C0201D08408CEFCAA0A34
:10C1D0007CEEEDA456E6C6762697CE7C4C1F261341
:10C1E0006603047CAA0ABCC6BCEE8CC3B07CA6263F
:10C1F0005F0C4FA646BC26BC703A4BA626E6EDD097
:10C2000063FCEEE626E6EDD00C604388983CAA7C01
:10C2100058E0CE7C0698E6B07C463C70B0FC70BC22
:10C22000A63C66063CF0E09301051601130B8099CD
:10C23000568891D04E70F80E300255701BB5A2AEE4
:10C24000BCEE514C4E70783C06F8C4FE1388CEF616
:10C250001348A67C9C4AFE1348A63C583154BCEEB9
:10C260008940A808B156BF0E0E3D3E180B80A14A6A
:10C270004E75F0EE600DFC0E0F200412091605F14C
:10C28000FE8C06130F1049F0F9C40B80E6E956BD89
:10C2900056585D1CCC604C6060B03AE08D0F0F12B8
:10C2A0000D050B809D5A8215131405074433901415
:10C2B0000507480B80594200BCA8E04E0070446856
:10C2C000780605BCEE59DE785E3E683C06660401E1
:10C2D000AC0EC1B01C0C0742271D145BAE012063DD
:10C2E0000C77AEBC4D14DDAC4924E304B1BCC36E85
:10C2F0006EC9A46E085346F059A4E5A459A4046677
:10C300008E060404D91078065830301C622B30B0E9
:10C3100062275613B6D91CB8B81C101C8C3342B80F
:10C32000302DE876B63CA23C3E1E7E7E8518492420
:10C330005DBC99C844785CE291DF3084CC2766EB21
:10C34000B371CC663F785C62683DDE309366FBC8B3
:10C35000CC2FC8CC0D541C101C02784CBB426F76FD
:10C360005B6267A21C10101C021776A268C34E5CA9
:10C370006244D302FDDA3668F6F65BE2E21FF6337A
:10C3800078562268E201DAFE435CE2234830F02B63
:10C39000C1B0BD1C03011420050D101419DDAC083B
:10C3A0000170650E4E9C90CC67601B7A1F7ACB881B
:10C3B00059C8550E1CA020E2F9CFD91C7858492441
:10C3C000300501ECC27012C38700233BB313BB0DD1
:10C3D000549B8CE378068605BC95BC66866608018E
:10C3E000AC4359C85B785C42688859C851DE8CEB15
:10C3F00048C393011405070B80ED520000000000B4
:10C400009805160113883398140507843DF0B0068B
:10C410003C2606F9FBE6C622BC70067CF03DD04EF9
:10C4200070F8AE708C2F38EEB94AAEF0E048F9C41F
:10C4300046C10238467CA65849F0DDD4B0E622FC5D
:10C4400006023DD08A983C0A05CC98420C172E0A69
:10C45000F9FB4EB07C5CD070FCE090051601130B2C
:10C46000803D6A4CE57A040D7CF57A0B80694606BE
:10C470007038F61366663C1EE0D09C30583A1C3A81
:10C4800030E63A30C64FE63F5C50D0D0F19AE60E27
:10C49000BC427CA67CCA70BCA6F6F6F6E33A3A0E1D
:10C4A000303C1E78AE7E3A3A306A677E8E8EFE2F22
:10C4B0004A2F440B4A97BC430E98AE7A30EA830465
:10C4C000D88C1B8408D86A3F8E8E0C374A77BCFD07
:10C4D000E24AE748B19AE6C532308306CE3C56665A
:10C4E00037B85CE2E2E2313238FC9CA262CF1CA297
:10C4F0003C28352EE0DCA0DCF2C156A00EAE1C724A
:10C50000CD564EEB514CD1C8E653D144E0C4F57E34
:10C510007D6813BB664670385C5228A658BDE0BEE5
:10C52000EF983CA6BCBE580948EEEB86983C7038A4
:10C530000EC67066E6386E33EE773A6E5F300406EC
:10C54000983A7EB75826371568A30DFC0E0F2013B6
:10C5500015030820010C0DF1FE266F29E60948EEAF
:10C56000DB33D1C8E62B4670F828B8EE4670CEF023
:10C57000F1688E1C527C706944E86E754CA8987006
:10C5800038F6274E70AB98267038463C05688D709B
:10C59000CE0EDC52BC702626694468454098803D2A
:10C5A0006A84050B800172840C0612038443930194
:10C5B0000C0612038801C8E6B5A2DC908C133E6815
:10C5C000BDD00881F08CA1C34E70780666263DC2AE
:10C5D0005AEEAE3C700698F00DD0A6065870CEF01C
:10C5E00070088C6366700201D030FF8D8CA658985D
:10C5F0000E0DD0A65870B0662F704EF09B0C234ED7
:10C600006EF0C102847E1788B0FC580670BC9C4A4C
:10C610001CBCF004738C060C033EA5E8B07E7E2B98
:10C6200089F63E8C1B78EE55F2BDD07DF20DFC12E2
:10C63000050320140F0F200C0F0E07F1FE920803C4
:10C640001010018408B5E00CAFCEBC06B07C8C2F76
:10C65000A63C707C26E6CEFC0AEDD0AE7C0E980699
:10C66000CEBC4630FF063B3CAA8D8CB03C0698E61B
:10C6700071D8849803920803130E09884349EA830A
:10C680000512130E0904B5E00CA7B03C51D8CE3CFE
:10C690000E889826587C9C0A7C1C0AAE7098E6EDA1
:10C6A000D0B0AA7C0EEDA4AEFCAE8D8CAE7C0E7C20
:10C6B0006A93846262901C622751EC02AE8C2FFC5C
:10C6C0000E888B987C0AFC66588C9BB383051210ED
:10C6D00010014404B9E049D8987C0EFC2BEDA45914
:10C6E000A4AE7CAE8D8C01D098663758AEFCAE738C
:10C6F0004C6030FF8D8E8C061A1305120B807D4A1C
:10C700005ABC1A203C06B0303AE62366DF461AE0EF
:10C71000411CF53E30EFB616666F3001B670387CBE
:10C7200006562306B66666E09819050B1405070B36
:10C730008005427924B5BCC10208D8284E2E687005
:10C7400088C4651C0488ED0600000000000000009D
:10C7500000000000000000000000000000000000D9
:10C7600000000000000000000000000000000000C9
:10C7700000000000000000000000000000000000B9
:10C7800000000000000000000000000000000000A9
:10C790000000000000000000000000000000000099
:10C7A0000000000000000000000000000000000089
:10C7B0000000000000000000000000000000000079
:10C7C0000000000000000000000000000000000069
:10C7D0000000000000000000000000000000000059
:10C7E0000000000000000000000000000000000049
:10C7F0000000000000000000000000000000000039
:10C80000810F1418F8EECE7EFE595A15C89C58397F
:10C81000B69209040D052E009170A56CBDCC06469C
:10C82000BCA63CF0BDCC26BCF0883E4E5859F08CDE
:10C8300053C1B01C4E901A987C5875B0BAD33020B2
:10C84000E8B03000E6E6C67EE3E8B0DCD00EA11426
:10C850004924385E285DBC8001529CC22B387C661E
:10C860003B0D54663002C61306F5C44E708CB551AC
:10C87000EEE8D5CCA6A62FB5BCFD5AC1B0BD1C04B0
:10C88000091220050D101419DDAC080170B902DC85
:10C89000901BDCD0FE84480453DC501BDCD0FE042B
:10C8A00044848404040E30407030BF0638661B0890
:10C8B000634C537C66B5F7EE7CE6FCEEAE0E3CA610
:10C8C0003C263C0E0C7F7038AED86E1788D8AE2E42
:10C8D0006F8C1B6E582DD00CE7A6067038FCA60690
:10C8E0007C7026E63DD00C6F4C278C5F83CE7C6637
:10C8F00037FCEE4B84AE0E3C06704E6EF00C278C6F
:10C900006B8485D0C6A686A6A5D0469330EEA62613
:10C9100086065C424F9B880C2FB0BC16DEBCDEF353
:10C9200076E30DFC060C2014191005D9FE0DFC064B
:10C930000C200E0F1420060F150E04F1FE1C3040C3
:10C94000704C57AE0EBC06387CA6BCF00CA04E2E28
:10C95000BC30BFF0E09208030C0504884383051245
:10C960000C05048449F08808E9D48CF9FB8C7B4ED3
:10C970007001C898A658CEBC06B07CC6E698A6063C
:10C9800027C6DB0686A6467098C60658CEBCA6C645
:10C990003CAA8D8C98E63C0AEDD0987C83B07C460E
:10C9A000707C707CF0CEFC0AD9D0CE7CAA0E84EDCF
:10C9B000A4F0664BB0561C2A13886A1CF0AE7CAEFD
:10C9C0008D8C8C60A293A63040562B3001B6166633
:10C9D0002F70383C06A2A2A28CAFAEFCAE88338C7E
:10C9E00006121510A068A5E88EB05A580881F09874
:10C9F0006E46262642EA4E7078063DC3BDCC46BC44
:10CA0000F0AE0E3C0A3DD0BA3CE6A670A638EE70F9
:10CA1000EEF0DA3C66A084A63040562B3001B61604
:10CA2000661FA5D0668C27887B981205160113888F
:10CA30003B9812140507843DF0B0588891D0B00699
:10CA40003CC61306BCA606BCD870E63C4626832628
:10CA5000E698A658B0FCA61C223DD098EEDB9214B6
:10CA60000507843B920516011388DC90FE95E8C10A
:10CA70005C4E70783CC6A660E6B006978C730DFCE1
:10CA8000050E04200F0620060CF1FE66A6C686BC25
:10CA9000A6BCFAB0FC060DD07AB0FC70BCC626BCB1
:10CAA000F0AE7084448C57A67CA63CA6700488B374
:10CAB00008849B90011713070512484B85160F0D2C
:10CAC000070512448491D0E6136670063C063C06C6
:10CAD000B958BCB958063C0627883C70B00E3CA635
:10CAE000BCA670840404B07C7038EEB07038EEF0F0
:10CAF0004C33B07C70CEF0B03C66603C048C7F8CD4
:10CB00001B661326700C600CEF3C080C9B700E2DFE
:10CB1000D0B0A68BAE7C0EB0E622FC06023DD08AD9
:10CB2000AE0E3C0A05CE94100B050513844B811400
:10CB3000100B0505138889E84E7001C8FCFA1E7EAB
:10CB40007EB0FC70BCA6063C463C7080C15A941076
:10CB50000C031284438114100C03128889E8B03C42
:10CB6000A6F5C4CEF07C06F5C46EA05A233003C6E9
:10CB7000B01D60EEB94ABD1C20051212DDAC0801E3
:10CB800070ED8AA188C1B0BD1E492404CDB4734E96
:10CB90005C90D0D010309C6262BDC06B49A43DA4B3
:10CBA0008A3DA4E5A4581C22071CAA588CDF6AED14
:10CBB0001898EA6DCC3010701EA114D91C7E9EBE50
:10CBC000B8BEF37EBAFC8518F90E46F070B85CE288
:10CBD000E2E24660E21BAE4BAEBC067CA63CA63C45
:10CBE0005EE0000000000000000000000000000007
:10CBF000000000000000000000000004320605E80C
:10CC00000000000000000000000000000000000024
:10CC10000000000000000000000000000000000014
:10CC2000000054000000009001000000042AD08899
:10CC300022282280008051018045028001C05504D5
:10CC4000C02422006024110054005001400500243B
:10CC50000204100D2002C05000000C0C00E0344F04
:10CC6000C8834F8A4F3C372C8E20C13B08E16810A7
:10CC70000D204E064065F3B8144DBFF48308922290
:10CC80000159C91D744FCC78E4452FC2F1020054FC
:10CC9000D450C1D8C430FD3A06FE876130164E41EB
:10CCA0008660434BC43D898BBBD1D3BB031011516C
:10CCB000D100034035312DE212133131D5C172500C
:10CCC00031E04C0005D10444151E50455D4C762FD3
:10CCD00003005C000000194207C9C4004066021648
:10CCE000F6460522501012B4CD460A001900740011
:10CCF000318F4F40384454F37F2B4147888714E0ED
:10CD00004331410F3C4A349009941140314166301F
:10CD1000CD2823514ECA60CAC01F8FC2E72F080119
:10CD2000B60501C2C8105D07FC2210301100FB04DB
:10CD30002244448C738748E0C4073D03A3064AA4F9
:10CD400080C1084B31C1142013044B03D60F1B02C2
:10CD5000023D0CC1E724E20051086000800000524F
:10CD6000D147842000923374CDFD6405C1111104B4
:10CD70000004F04020800661761402C404640012AE
:10CD80000012EE450D0511A0803900102148410028
:10CD90005238B18C40225015F70500549C0B0060AE
:10CDA0000020409A25CE660040050002205D3EA985
:10CDB0002686E8B534D00C004033C14149C223A3D4
:10CDC0007463C71333CDEFD27188521027BAD2E300
:10CDD000C4B84EF9F3B5A78448F623C2BAA24521D8
:10CDE000A28D6CF63300004E32C884B83260301D1C
:10CDF0000100104CE98608B7203B2AE10E0019001B
:10CE00000008804278001A0A820280078F442200BC
:10CE1000215410E1417004001D65155D2275F3B8C1
:10CE2000E322C140244354689FA88F2F638F854B12
:10CE30008B3D1F4FBCA244C05C357A9F2B0896D413
:10CE4000C515724F45A1214505910921A130E24444
:10CE500029BD290000603C981F8E04884668819196
:10CE6000089282470BA9C55401110002008620A236
:10CE7000833C683D40964089240204500189800724
:10CE80003A8A500A640200E8C0A48C0800006000DE
:10CE900080C1612444020555582C00146001800EA5
:10CEA00000040F80996110440009001073CD003C0C
:10CEB0007D840900500011C8000049C01D000074A5
:10CEC00094D4CA63114113480DD4000051DC70980A
:10CED0001913000000000000000000000000000026
:10CEE0000000000000000000000000000000000042
:10CEF0000000000000000000000000000000000032
:10CF000000804A0C00404613912302090D54171D5E
:10CF100053B58F34215E94A01611043630C5D10C60
:10CF20000080938C20000802F01246CC800200148E
:10CF3000482734878189904020227082815389025A
:10CF400031057041D43D5124230060080000601079
:10CF50000215828F8403800080427218468451C477
:10CF60004820514800511110204241B420B02C00FB
:10CF7000F0514CD008550B3C00094048A4803E03BA
:10CF800052098180487F314103FC038000A0104298
:10CF90000451019D4400480420002800E0D43022C0
:10CFA00000008640040480620208117C1F0000001B
:10CFB0000088488851C41004C14B02824022380CBA
:10CFC0008838C693C014400854000003000C184071
:10CFD00081124404C000C0000454E0440030809337
:10CFE000CCCC4406F5BF5A318CBC41400484CC40C3
:10CFF0003708C25EF501D4080C00000000000040B4
:10D000001A24005D0B6E08060F380B670B5F02D702
:10D0100002E202EA02F306340407010002C102C878
:10D0200001790089016E0122011701350B010423EA
:10D03000040F0B440CE5056009FB00EE09410054A8
:10D04000006902D0007A007100610000850D0914AA
:10D050002018032D83322020050D09142D9410175C
:10D0600013C5DA810D0C010C0341E68D0C010C0394
:10D070001289E6930D0C01120C03C9CE00000000CA
:10D08000000000000000970F0404A140F944694823
:10D0900063C1B0981E7E3570DDAC6564983102586E
:10D0A000300370C158CE6152814084D54CF88C1346
:10D0B000B86ED330200C3330188C1326E6A18804C8
:10D0C000B17022D91CB8C6E86564ED8A389C4AE084
:10D0D0003E3E3E8A1E4E62EFCECAD47EC31E4EAA8C
:10D0E000E05830107030FBF0E8E0850D0914D96885
:10D0F0008E7C5E61446948BB6ED9708B85140104D7
:10D10000D968754C694843C1B008F548656498EE24
:10D11000B94A97130C0312514C04E5449B86010C49
:10D12000031295445B514CF8BC6944FEA0DC50E00E
:10D1300097130E1512514C68E08940A838A0FE1BC9
:10D140005C8A0E9E1EB1644E46D95C5C19688D7077
:10D15000CE0E5C7CEACED95C5C4AFA1F4E5BA00E18
:10D16000665C1BFAA642EBAE0E60E099040DB8BCFB
:10D17000D844D87CA8E0990D04B8BCD848AB0E8E32
:10D180008EA04E5C504E4E9C3E3ED05C4140603C7A
:10D19000E00408E0DCA046F098067038F6136666F6
:10D1A0003C7E60BCA6BCDC100EC1B0AE5C900E46EE
:10D1B000F03C70380C435C04F2277CA2E370D91C6D
:10D1C0008EB07C7075B06E8E5E4B5CA2A39CA2AFDD
:10D1D0007AD30CE361009CD2BB9CD2A0C1B0DC101E
:10D1E000FE04041B300B3C0E1CF86A1FBEE3B8495A
:10D1F000243E616A856869547008A968E60670383B
:10D200001CFC6A6A1E6A337E7E98A658B08148ED7F
:10D210004E6954BE3E0165DB000045DA00000000A7
:10D2200000006954F693E0DCA01CEE982670380EDE
:10D23000A0F2A65EEBA6728940387C323200003242
:10D240001F12EF662792B2939260981D68A6049809
:10D2500070CE1C42F0861E81487E98C6BE6066EB8A
:10D26000F613263C5E9E9870380C134E7098532629
:10D270007038A670A6F066A60626AFC670B0F0BEDF
:10D2800033E0300870A6DCD09C1E387C4A3CEE604F
:10D29000A6BE60A6067038BB8940387C4666E6A606
:10D2A000260E4B361CE2172AA6496870383E607E6F
:10D2B0001C128B1C42F0935C0A6029FEAB05140122
:10D2C00004D9CE93190104048DCE980D0C010C03E2
:10D2D00011E6B2310B0C03DD48449828E0B4320B60
:10D2E0000C03DD4848AB940B0C03DD48846B8414BD
:10D2F0000B0C03DD488823514CAD72754C46178EDC
:10D3000030020C6BE01CA01C50509C30057217665C
:10D31000884884DD6C0C0BDDAC4E30200EB8B8B8FC
:10D32000662F7EB86623D888D8E8492438D91C9C53
:10D330004A9EF9447E3570492659CA85683389402A
:10D340004EA8E0454A93000099CA08C1B04944007C
:10D35000B9620058894068F858A8B80E4EA07A60A3
:10D360006E1F8CA0A84E2828A82828E8E828E8A83E
:10D370002828E8A8E04970136BDD48A00E3CAA7C81
:10D38000C6A670663004062B301246BA9A4EA6BC6A
:10D3900001700EB01A9A70DAA5709A7C2B816CA07D
:10D3A0000E0E4924389C0AAE284A7C0E4E5C50D0A2
:10D3B00010101090504E5CD0905090DC4140AEBCAC
:10D3C0000E389C4ABC70BAA57070BC0E4E1CD010B2
:10D3D000903A5C49404E5C100E2BCE7A1A23AE7CFC
:10D3E00006B0A6705A0170BC30120EB0BA5A7A66F6
:10D3F00006237AA646FCDA3C5CAA7C0EDD48694628
:10D4000094030512120F034843850D0914051344B4
:10D410004E7D4070CD6C49503C2EFCBB8514010400
:10D420001405134E7E708140EEB5A258CD6C448435
:10D430004950704570380EB0284CD3492478AECE90
:10D440003010956078AE68CEF0AE5C4E138A0A302C
:10D450001095607858B075604E3004583A3024BC4E
:10D460004960709544A0EE1FA01B2D60B02560EEB2
:10D470003961216CC4F57C856813E061481CCAF9E8
:10D4800072E0AEBC0EA01C30120A334A2356134A77
:10D4900016E004E0DCA005688EB03E777E4970138C
:10D4A000730950EA0A4BAE3C0E1C12D1501B84ABE0
:10D4B000D8EE271CD2D3D54CB540EE4D704E1C5043
:10D4C000501C0A1BCD4290901C0AD36E816C4E0EEC
:10D4D0008D70CE4EFD50A0980EE09ED95C4D70131D
:10D4E00063D95C8A8A4B30030455701B616A8A8A4F
:10D4F0008A1ED95CA04E9C909C0A931C3C0A73A087
:10D500005C99704E5CA5700E0E60E00E695013EBD6
:10D51000D95CDE7098067C6627B00E2B6670C15809
:10D52000CED95CFE23A03E2B6E6D50234C670BD9E9
:10D530005CDEA05CFE138A0EB0FE138AAECE5E6F78
:10D540009E2146307A66FB61020404981D5C5AE114
:10D55000080698467CA6BC58E01C987038E09713E3
:10D56000783CE64EC67CC63CEE514CC4780ED1E207
:10D57000B1640E681CE260CE3C58B96C6100CCED21
:10D5800057080C7F44E544CCCFE05CB5708C171C89
:10D59000D85346F0987CB95844CECC37FE2BA03EE9
:10D5A0007E538C2B2D548B234970630460B1702201
:10D5B00008D91C495C638ECC4FE01C214CCCF55C37
:10D5C000A0CCCF6089406C9BF89CE27B4970CC1D5D
:10D5D00070CC4F89403031E8F9561CF8EA23A8385E
:10D5E0000E98BC62EBCCAFA2023C580CAF0844AE24
:10D5F000F544CC47214CE05C115C3B6046F03013B5
:10D60000716487138474348575358676363718824D
:10D61000C21283C37300230B36363636363636369F
:10D6200036134B237BFBFB6B53306E66FBF1568B43
:10D63000030F0C039170E5EE995ABB05D40D5449C4
:10D64000248142115AB95A855A0DD49170A56CA003
:10D65000F9CE73AB8C374C73195C061C62131C42F9
:10D6600062315D33D38940F81C0CFFEABF4EA82815
:10D670009B4C8FB570A88C1B281368580C2555F34C
:10D680008C178C1F883B842B4CD73032155CA08CB8
:10D690002FA6FB415E66134660315C315488E54C31
:10D6A000AB8C9F4C8F0C1F0813042D5404434C3734
:10D6B0008C370CCF08A55A044C1F481344989C4241
:10D6C0001C4258C3155C044C374666B64893367600
:10D6D000DF1C862233A24C47C62B629C86A24431B3
:10D6E0005C4CCF3154BB4C778940A838700C255521
:10D6F000987CB958B004F544987C70AEF0C8CC7BE7
:10D7000008488C2D55C8CC3BE01CF55C46F0983C95
:10D71000A02660F61348315C7C26BC588CE54D6130
:10D7200000987C26167616577038AE98F038AEF012
:10D73000986E4971F9560CA04C43C8CC60A060208B
:10D74000E0CCED57E006983C0CA03CE03C0C173CCC
:10D7500058E0302E0C1B303DE830128C1B3004E8B2
:10D76000195CD95C065E3E4C1B3E234C17E63030FC
:10D770007CB6163C761B301FE8E67EABE0A0C1B05D
:10D78000600C495CD95C6EE00C2B5E4BD43B5E13A5
:10D790001C4C135C2BE01CA05E0EC1B03E04885CE8
:10D7A000421B3EC3EAE0DCA07EBB830491704C4F79
:10D7B000D8C9705C422F3E33D8885E3EFED91C78B3
:10D7C00068786860E0EAA09C9A5E339A509C029068
:10D7D000DEDE1790D95C13D07EF3D0D0D0D0D0D07D
:10D7E000D0E0DCD08C7F0A9417904C276210135045
:10D7F00050DC0210CA683828380AAE28A046F0E08B
:10D800009401030D0C017D681B796666A65E3E5887
:10D81000C4440D54E0C170843D6404CDB47B758C68
:10D82000E06564E04871682B65644164E04544EB61
:10D83000B068CDB42BE5AC88138478703D64E065A6
:10D84000443B8CE5AD3D6413208C758DE020843322
:10D85000985E580D54214C492498FE2BCC6F1568C6
:10D860004330FFCC3766EB235162203C560630181C
:10D87000662D5A308766D3309366FBC8CC6100FBB7
:10D880004E9C90CCA7601B7A1F7ACBF55A894858DA
:10D89000C17085641385644B1C20E2B78C73E54C22
:10D8A000300671643470C28412C300133383533B57
:10D8B000DBBBD14413037966E168E09C83016442D9
:10D8C00049621B985E3E4962E54C2B3008716480CA
:10D8D0003482C2848712C300CB033B3B6333538B38
:10D8E00073EB1568E365203BF168E05CE17084410F
:10D8F00062F168C1B008ED48B3447168008B294EED
:10D900008568668698663315C84D68CBC658E02092
:10D9100030F1CC256366E3E0E008017201EE884156
:10D92000DE9870C4F57CB058E0000000A09C4ED09A
:10D9300090CEFBE0B87CD88C6089028D0C011A195E
:10D9400018300289407D4070514CE83888084D50AD
:10D950007C46EE173A70842689400EEE6B8899500B
:10D960002B301AF1424E360ECFAE7C466860094825
:10D97000B0300446068C1B66367066A658851406C1
:10D980009806678826260613848568238C97A188C5
:10D99000C1B0BD1C0E0F20120F0F0D38F8214286AA
:10D9A000C626704E7EF0C6704EDC90901090F0044B
:10D9B000A96858B0C6260E2568869806B05568989E
:10D9C000A658A670660638D87066D8F026ABC67022
:10D9D0002658B0F65BF04670780E98702658AEF078
:10D9E000B09C629F0948EE173AD87026D8F0BE3F27
:10D9F000A6667006388BD152982B148140CD6C2EC0
:10DA00005899501BB5A2A0DE1B8E0E70984E5E3347
:10DA10000ED164AE734E9C501090D05010D090AE8A
:10DA20000E874570380EB00E286B8606B05568C656
:10DA30007038FC1CAA0C2F0A3967134A7CF026A602
:10DA400004A568A6A6E0A6496870381C3E607E1250
:10DA5000B3E0067038F61366663C46FC0606E051F5
:10DA60004C4EF0E0DCA030C0085C905C0E13664EBB
:10DA70007078067BA60670383EAF7E62A0FC5646E4
:10DA8000EE770CA0A398496870383E6F98A658E0CE
:10DA9000894833D144E07EA060B03AE06954F69BF7
:10DAA000982670383C05688D70CE0EBC555CD91C2C
:10DAB000B83B4C604EBB514C894038339870384667
:10DAC0003C0E0430059C5A109010DCDCDCDCA0FA23
:10DAD0005A13229AF33A0C534C2BC8CCA023CCED0A
:10DAE000576627D4BA73945BFA5A5CD0905CFA46B6
:10DAF00026139423FA10C3FCAA0E60E086011405D5
:10DB000013514CE838288140EE8349701B4E5BDC92
:10DB100050AEFC1E1B261FE6EBBC89403CA8E8E08B
:10DB20004EDC5050501090E084E80444D828E8308F
:10DB300029E8E0EE514CE8380E4E70AE68A0E09750
:10DB400013140513417013339E048D501BB5A24D61
:10DB50004C98DE1BA08E28E0B432050D0914018418
:10DB6000887B850D091401843B8514010401888498
:10DB700044417013CBB87C1C50600691704C23D884
:10DB80008813D8492430260213A222D888D88C7B47
:10DB90008662271CEAEA0604E948E2B308A3068C79
:10DBA0004FC9705C4267DC906B095060AE3C0E134D
:10DBB000FA4C47DCD0A25D6C6E4BD91C9C10D0A2F5
:10DBC0007CE89CA2BB8C608C603020616C30414C46
:10DBD0001B3050616C304D6E5851B6B6A31C8C7F13
:10DBE000A25390909C5D6C6E167693D090BBA2CFA2
:10DBF000302F0C4B664C73B8D848D81B4C3BE84BC5
:10DC00000EEE0E0EEECEEE0EE0CE30046944A0E035
:10DC100081400E3001A0A65C4636616B7606138A01
:10DC200066F3E0A0A01CE0DCA04EB2CEEE4EEEE02B
:10DC3000F16804E09C23E09C08A0C1B0AE707C5E5B
:10DC40000EAD5C0C60D91CF8F8B00EED4A7E7C1A63
:10DC5000FA5AA57013150E0D0F0E141505170504AD
:10DC6000140815061209130114B01A30E83ABEE37D
:10DC7000E09806C44924B8BCF6F6F6A088E004C5CE
:10DC8000703059D866F31BC570301E0C1BCC8766EC
:10DC9000DB2308C570302DD80C1BCC1F66D3C458AD
:10DCA000A60658E030107030FBF0A838238940F801
:10DCB000D8E0AE8444BC0E30121C0A776A53A0CA66
:10DCC0000A374A881B563348234ADF0660AE3C0EAB
:10DCD000E00E4E7078EE894078A0AE8E0E68E09728
:10DCE00013100F1413514C28E060FCB07CA0EE0E12
:10DCF0001CD09050A636369C133AA2F38E76E3AE33
:10DD0000BC0EDA3CDAB0BA5A707A9A4E5C109C417A
:10DD100040AE3C0E3C5A4E1C50D010509010AEDA23
:10DD2000CEFC70B01AE05D1C0C13C88498A8150CCA
:10DD3000711EE1688CD972E0C97020E0894038A07A
:10DD40002E2E60E000000000000000000000000037
:10DD5000000000000000000000080B6CBB8CAB0E44
:10DD60004E70B89CA2A8B5708C1B585B4C43C1B0D8
:10DD700048042BA16C044484617604588940594CB2
:10DD800038580CC76C2F4C517EDBE8F8D84C4D76D8
:10DD9000D80C1F4CC34670B83CD80C738C674C57DA
:10DDA000D80C7BC97491704898A828E8381CEA57A9
:10DDB0008CA30568EA274E907BF83CFECFFEBF603F
:10DDC0003D5BCC4B3B4E36682B854044E804D8A8DD
:10DDD000288940BD6C88044408844484608940F8E4
:10DDE000D88C3BD83038E8FD7E0C27D8D57E5848F3
:10DDF0003031E8757A980670389C62CFF613666603
:10DE00003C1EA6067038AE7E1B4E23267038AEE050
:10DE1000DCA05CEE5D7AF237B2EEEE7CD37C0630AD
:10DE20005EA61C6A873C5CB27C0E4EB2EEEE521BC4
:10DE30003CD31CEE25510E917004E6C61CEA4BE063
:10DE400008F174A8E8557E3C305E6A478E8E8CBF20
:10DE5000CC87A3FE97C68C7F4C6FD844CCD3655437
:10DE6000D0F0F9700D7EC6A16C49240C37B8D844A7
:10DE7000D8A8AE6841683B8DE2F174A8E8CC9974EB
:10DE80005D1C0C330498A809B8BC5884983CA87849
:10DE900058EE091E44D5420C676554D0F09888BCF2
:10DEA000983C589974E020F97098BC584C93C1B0D4
:10DEB000BD1C14090D051220010C01120D20534543
:10DEC000441333C17098BC5846F06666FB610098F5
:10DED000DC1044E05830F1CCFF66EB2030264C2BB0
:10DEE00008FD7046CC9F66EB987E4B4C1F482B4834
:10DEF0008C979170A56C6B2020441C583C1C0A49DF
:10DF0000CA30C36A8B2E4C4544000D54654400460C
:10DF100066CC3766EB0D54411C4C5F9C985606301E
:10DF200072665F4CFBD57E8C6B480D7CCB4168BB29
:10DF300098E3970F0E0D0C01514C88C4084860857A
:10DF4000684B2315684389400EDB6631687038E6FC
:10DF5000463C0E8940F9740E630C474C3F8C271CDD
:10DF6000C217D5764C43F8D88C1B58E058AEA8E8B9
:10DF70003038E84C60E00C132049244CA7CC091F32
:10DF80008C8B91704C37D88C53C502603D5BC97443
:10DF9000F90C9170048498A82860A05D1C98CD9E0F
:10DFA00058B8EE514C6C9B385888989CC2285D1C20
:10DFB000089842A84B4D4C38580484D91C783C89A9
:10DFC00040A8FE63084E2B00E080E02E6889CE4C0E
:10DFD000EBA56C33587D6813DBDC90F091708CA757
:10DFE0006148D6F970736576817ED968C97071BA57
:10DFF000D57EE976008B93CBD3DB0003320D14CEB4
:10E000000000000000000000000000000000000010
:10E0100000000000000000000000000004000000FC
:10E0200000006C454C54434D613076314C4C8C4C67
:10E03000C1CC34CAAAF4BD031FC60F60481110003A
:10E0400066C4781400404503401794EB00D4DF28E1
:10E050001B505047BB402060CD3D3930B30FCCDC66
:10E060004B45DA6707C225523BE40D172330723364
:10E07000300173171992E4E3C4793F7D6055402461
:10E08000A348451455922000508E404ADEC7B14245
:10E090007CF45845324211EDE291008482183D62D1
:10E0A0001F2246E435C9C708060B94B8FC3838006F
:10E0B0000400020000C07503700D700EC07999CD88
:10E0C0002144688C43D910FDD3B31F8E505448713E
:10E0D000300DD21847374FA8C3E0129BC4139A489B
:10E0E00043315140140AA790161A425812250507C9
:10E0F00029C05104E961838D01501188137A71564A
:10E100000080008018642B00006242E4C615594864
:10E110001122B05884214406012921804253B16D57
:10E120004D79CC4C3C7220125843C53149500611F0
:10E1300036063D6474670E11D01311F643423C3E1F
:10E140005190798704E5501A90281C3EE16288F4CA
:10E1500054B848C554429F0C0388D434242344F255
:10E1600025D28109C71972A2320444064DC1405D0F
:10E170009C371CB6DD05353DD50E91263405A61C11
:10E18000040000000050AAAA5645851700069754BF
:10E19000CC998911501ED521961D5B33B72DF316EE
:10E1A0003E7719A53409564948885810C210C00452
:10E1B000914520A1BF00E353659537581944293E86
:10E1C000393D501CAA504A92A43442826DD5F227A0
:10E1D0007F17CE091D12C7C44521481C9311EF3388
:10E1E00052043033002134C623334E16DB03830C34
:10E1F0008040CF1708042E12308010011F0004F059
:10E20000005050605B1294719219441A681820E40F
:10E210008111732E51556463F4782414576CF98B73
:10E22000C8843851445398464100C080724C06D18E
:10E2300054587410000004BC600A0664D978675C06
:10E2400015CDD4F479B92790C444030AF5B70B006F
:10E250008419356F23B2967C84E1336A844D124968
:10E26000CD3A57333300601F288AA82014585154E0
:10E2700084469A8F868896862C26A619685C8051DB
:10E280001DA01835109015047F850914C2808618CA
:10E29000554C09EE9F488D763112ED113E24EE4328
:10E2A000DE5422D1C4DD6625291E6D36DF5C0709E8
:10E2B0005684F52F6017F2F3C92F10050EB0E40055
:10E2C000D4644280818877CE08D907773035213AE7
:10E2D0000004744025CA00C000C0003010CE99C5AB
:10E2E00070D4E03F4F1F1610D8239810837030036E
:10E2F0007F3CC745C405403EC11F34DE01F237FCF8
:10E3000065BD1FE556C86AC2BE84C0D5260232204C
:10E31000990FD365550000000000E4DBDF31D55FC5
:10E32000A54E458C539531BEF4617C1C0F553C6362
:10E33000134C7C428772483200D44B0852E8D43BDD
:10E34000858100E561462545102EA32F6192F48753
:10E35000EA0000000000D44C786C333009D95757DC
:10E360009D83357303E17F541319DF2C724270488B
:10E37000F5601CF11D6D0B1ECF01C13581952C522E
:10E3800047828002B226FC5FF03B073FBE930987BD
:10E3900012DA311F4E3030565B05853C8F46104AED
:10E3A00002FCF4B3398AD6461379D53003000088CD
:10E3B00001D5AC4BA6C5F82D15E3B97866D406DCBB
:10E3C000C4805107BE57C0500C94531B0100D56246
:10E3D00081719009D8D108CB7EC0F383013B4738C7
:10E3E00063304C4561FE89344D7D7F24CE57FBE47C
:10E3F0001D40B70D9315ABF6665D665456FC0B8851
:10E4000000F8615044FE1348260E7676B5A3D91C59
:10E4100078D88484D88C1326F046F009C886E64B59
:10E42000309EA62BA058F142CC2766EBA3D91C78CE
:10E4300058203C56069CE21B4EAB3012664761C822
:10E440006686A568E330C4064FC64ED0A646263C75
:10E45000A3E6761C4E906AC6FB303162276A13A68B
:10E4600062AA3C26048C2B08A07E60585D1C98BCD8
:10E470009CE22B0602A2E6C602A23003622F1C42D7
:10E48000136230088C270C237B0C134630555EFC3E
:10E4900006BC30E61BF61B2E03068C2FC16813C387
:10E4A000A60EA05A7C1AFAFAFAFA56233C3AFCEE67
:10E4B0001A46BC26260E55C4604C61008859C8789F
:10E4C00028B86898A859C4EA005ABC1AB0303AE68D
:10E4D0002366DF461AE0BDD065F04C2FA18002DB39
:10E4E000CC3F4E70B8584C7BCC6795A43C0A59A4DD
:10E4F000E5A4D88C1744A180FD188A8514064E70B7
:10E50000CA685878A6C6026A6DCCB05E3C062B5D20
:10E51000C4C830DA7004B07C0E01D0EDA4AE3C6605
:10E520007F7098AE59A48D8CAE7C6606FC5843046F
:10E53000987C1666C3084E70980E78061BA66878FD
:10E540000E59A430C08D8C4DA4468D8C4E587078D9
:10E550000E4C23C4BD8C783C667BEDA4D884D88D4A
:10E560008C29A429A4AE0E584E70780EB8BC5884DD
:10E57000E0DCA0DC1050121C8AE5A43C5CF2CB7EEF
:10E580000F02FF1C8A4DA4EDA47C6A22D398AA69CD
:10E590008C0A588C574DA459A4468D8C980A29A4EE
:10E5A0001B1C6AF5A89B623C5888821B59A4468DA7
:10E5B0008C42D762101C021F023BA666700A4EF006
:10E5C00098AA698C7038989C50F09806467078A686
:10E5D000682E063B6670EEF0EECB4924F85A5EE8F2
:10E5E00030BF2684A80E78AE66CB70380E4670AE6B
:10E5F0003E8B1C8C137CEA330EFDBC95BCB88C1F83
:10E60000884B781C0A29A429A4B8AAA8A1801C397F
:10E6100088E68F0C2F59C4F0000DFC03080B13156E
:10E620000DD9FED5883E434670AA680A4DA4E5A4DC
:10E63000AA704670785816468386FDBCEE4B66B8C5
:10E64000FCEE0825AC1B95BC780EE3D1486E2B5927
:10E65000C42E1659C41916D1486ECFA3D1489D486F
:10E66000FE738BD1486E4BBBD1486E439D48FE2351
:10E67000FBD148CB4E3E304C0EB87E5B81C806784D
:10E680003C06B9586E63AE6E7F3A3A3A3A3C7038FF
:10E690000E8E844E70F8E030546E9B305A6E736666
:10E6A0006E53666E33B5A20EA04E3E7EC37E7EA034
:10E6B0007ECE7E574E43EEA0663346F6A0BEE04EB9
:10E6C0005EE76EE0CE7E1B5EE0E0DCA0DC5EEE1F6F
:10E6D000237CF2F3AE5EEE1F237CF2F30E03E0A583
:10E6E000CCBC0E4670AE6881F04E70789A66AE680B
:10E6F000304070AEF03E55F04E7084B07E7E7E2F7E
:10E700007E89F68801C8E6B5A286B0668DC61C066D
:10E71000A54FC678A6063DC358B0FC06707C26E619
:10E72000F002223DD0AED8E63C7006023DD0B0E605
:10E730000CC38604304006A5D00C49D1C676431CD4
:10E740000A6AA5D049D066B0E6C67038A670A6F0B1
:10E75000986666776651ECA606704EF09866BF8D97
:10E76000C68451EC8C276688D326E67022FC06020C
:10E770003DD0A658B026E6FC063DD098BCA6588CE5
:10E78000A3BA44DDD47AFA9A983C0698767FA60616
:10E79000BF0DFC060C2013091A05D9FEA5D00C9755
:10E7A00098762BA5D00C5F98E63CA6B0FC707CF068
:10E7B0005DC40A3EE6B006A63CA60667BC704E7075
:10E7C000F8FE2F66A6067038EE472DD0983C66AF4F
:10E7D000BB0000000000000000000000000000007E
:10E7E0000000000000000000000000000000000029
:10E7F0000000000000000000000000000000000019
:10E800009CC2FFCC574626FBCC2F5DC4243C71CC68
:10E810006653309066FBC8CC6100839C4262E2A5DF
:10E82000684E9C90CC5F601B7A1F7ACB5DC4E01071
:10E8300071CC664FA5689C228859C87BA568D91CF5
:10E8400078583012662761C8CB30C266AF46F08C6C
:10E850005B59C8BDCC66E627652073BCF05DC42952
:10E860003C26662F8865C82B49F08804E9D48C2B98
:10E870005DC47E3E4E70088C2B4540061BF9C430AB
:10E8800018A6C6B07CEEBCA686A6061F04A666988F
:10E890003CC658B03C0671D84E70B87CD8040C13F6
:10E8A00008D8BCA898668DC77C0EEDA4E601D0AE52
:10E8B0003C58C69C584E7051B41C53BDD0C1D85E54
:10E8C0003E2DE0DDFCB1C0BDD04C1BE9D071F0B0F5
:10E8D000FC700602385AF051FCAAAE3C58C9C099E7
:10E8E000C0980A01D098AA0A5841C480E68741C45A
:10E8F0004C5780E6AB708D8C987C0EB004D88C138E
:10E9000008D826CABFAE3C580AB066577001D0413D
:10E91000C4808D8CAB0C2341C4804B081304980A2F
:10E9200030FF8D8CA156C1D8BDD04CD9C85E7E7E3B
:10E93000FE39E098EEB5F604DCD01EB07E7E2F08DE
:10E940007E29E331F40C533E85E0B05E3E7095F0D5
:10E9500059C0B0CE46CE6E6E68BDD071F04E7078A4
:10E9600058B0FC060201D0EDA48A0456705C0A0679
:10E9700076265766D88C1B086AD86A6A98AACAE7AE
:10E98000AA581C4699C4B0A1C46AB0664F7001D0A1
:10E99000EDA4A1C4B30C7B46A1C45B0830FF99C4AD
:10E9A000640530FFA1C469D095DC0C554AF9FA38EA
:10E9B000BCA6BC288804E9D48C434E30913CEEE9D7
:10E9C0005ACEBC06B07CC698BC1ABCEE4E70385C01
:10E9D000AA581C06BC065F3C0EEDA459A4E6AEBCCA
:10E9E0000EEDA4AE5884C61C6A17881C987C66E697
:10E9F0001F8CAF8CFBFC580A01D098AABCDBE156F7
:10EA00003BB03C263C463C7098E63C0AEDD02E8458
:10EA100049D463BC6658CEFC0A01D0B07C263C7059
:10EA2000983CAA7C5806D3B0FC707CF05DC45E3F75
:10EA30007E2F06ABF0837E7E89F788480DD4CE58B2
:10EA40004E70F80E8C2BEEC3F9FA3DD00698BC063A
:10EA50007F0DFC050E04200F0620120503F1FE6653
:10EA6000B03C065DD8554AA5CC06BCA63CF081F06A
:10EA7000D5CC663002C61306F5C459C42E12000068
:10EA80000000000000000000000000000000000086
:10EA90000000000000000000000000000000000076
:10EAA0000000000000000000000000000000000066
:10EAB0000000000000000000000000000000000056
:10EAC0000000000000000000000000000000000046
:10EAD0000000000000000000000000000000000036
:10EAE0000000000000000000000000000000000026
:10EAF0000000000000000000000000000000000016
:10EB00000000000000000000000000000000000005
:10EB100000000000000000000000000000000000F5
:10EB200000000000000000000000000000000000E5
:10EB300000000000000000000000000000000000D5
:10EB400000000000000000000000000000000000C5
:10EB500000000000000000000000000000000000B5
:10EB600000000000000000000000000000000000A5
:10EB70000000000000000000000000000000000095
:10EB80000000000000000000000000000000000085
:10EB90000000000000000000000000000000000075
:10EBA0000000000000000000000000000000000065
:10EBB0000000000000000000000000000000000055
:10EBC0000000000000000000000000000000000045
:10EBD0000000000000000000000000000000000035
:10EBE0000000000000000000000000000000000025
:10EBF0000000000000000000000000000000000015
:10EC000081C8E6B5A2064540B9CCA6BCA63CF048F2
:10EC100085F08C5BB0FC2670381CEE77709BD5CCF1
:10EC2000A04E70EE59C4EA003CEAF30E4E70AE6896
:10EC3000B01E4E3E1CBEBE33501050903B10BE2B3B
:10EC400010105003BE2B5050D0D3B046FC06F5C474
:10EC5000A3F85E5AE8A878E630C0062663A60670D8
:10EC6000383E334E7EF066A3A1803CD5883E7B7053
:10EC7000AE0E584DA459A4468D8C980EB0E66F7018
:10EC80005DC414218A4E6E56DC90688DB8BC08981D
:10EC90003C28441C6A8AEDA45606303A067B303084
:10ECA00006AF3020469C58DD201C6A4E30056A5B5A
:10ECB00059A46A4C8FEB48783A87783A8DC7B83CAC
:10ECC000D808D87CA88CB5515DC4333B3045663F2D
:10ECD000783A27301B83302B66832666378C7F304B
:10ECE0001A23266627301CD32666678C9F4C435315
:10ECF000F8EECE71C8700439D006B0BCA6700839E1
:10ED0000D0E6172606B0BCA670783C06B03C063CA0
:10ED100006B958BCB95826703C063CE64EA670A60B
:10ED2000F0B02606C78DC60E66176629C6BC069CBF
:10ED3000E2D330901C02AB30316A8B30460217664A
:10ED40009C024B501C62276A136AA6A606C6E6A25E
:10ED5000065E233008465DC46A27F9C40C2F70157F
:10ED6000C8E68DC606F8FEB0C6FB46DE1BA6C6A6E4
:10ED70007079C4AA58B0665F701C980AEDA49C58BC
:10ED8000461C8D8C51B47B4E1C10CC2F6EEB4E4B21
:10ED9000203C56069CE21B4E5330C4064FC64ED054
:10EDA000A646263CA3E6761C4E906AC6FB3031622E
:10EDB000276A13A662AA3C26EE61005DC42E1230BB
:10EDC000FF06F8BC66470EB8A6AEA88DC6B8BC66EE
:10EDD000B5A3840895D0302B06B006273C061B81CE
:10EDE0000A06B8BC13EEA6F30EB03CE630A8AEEEB1
:10EDF000176668A69C583508B0063C260677BC7096
:10EE0000783BF87EFE5F5C10EEAB1C7CEAF33C3393
:10EE100015C83C9C4A7079C40C2F8AB058EDA4AE3A
:10EE2000D87C1C846A1788D8AE987CEA1F8CBF4EA9
:10EE300030051C6A538C2F6A59A40359A4034E70E1
:10EE400030913CEE3B79C46DCCF5C459C4EA00BDA9
:10EE5000E0DC101E46FCBE77E6A670066638EE7053
:10EE600066EEF0BEAB5DC4EE00307A66FB61027800
:10EE7000E8380E38D81CAA28E09CA01C380EF8AA46
:10EE80007CE8AE7C280EE0D4948DC7A0EA73E267DC
:10EE90009846AE283B48084EDDE04E300BAAA0FA5B
:10EEA00060E6133AA6CB3C30030E51C45DC42E126B
:10EEB000B87CD83C30300693302E66370C60A6A65E
:10EEC000E0300D664F302D06E0303A066061DAB171
:10EED000D0AE0E3CEECEFCEA6DCC666686664E3059
:10EEE00007A63AC6F346703CEEBCC66804044CE183
:10EEF000C4E9D00881F08C4BB07EFEA1C3A1F4839D
:10EF00004E70780666263DC2EE4E9CCA1C3E70AE20
:10EF10003C06027098F00DD0A60670B0F07A4670EC
:10EF2000CEAA7C0EE5A4E6AEBC0E01D0C68D8CB098
:10EF3000A626A67A2770AE5B7001D0B08D8C0DD05E
:10EF4000A6704E6EF05DC4F000492438FC7006389F
:10EF5000FCA67C70E04670387CAA0A3C28E00404D9
:10EF600084E9D4983C1C0A0451FC4A2A2AE0306007
:10EF70000698467004261C7C4A300AFC58B8A6A89D
:10EF8000E0D91C78D8E0EDA40616D91C303A6643C7
:10EF9000302C6623302E6661DAE0B1D08E0441A4B5
:10EFA00044CE0637662FA20217484ECA686A054645
:10EFB0000000000000000000000000000000000051
:10EFC0000000000000000000000000000000000041
:10EFD0000000000000000000000000000000000031
:10EFE0000000000000000000000000000000000021
:10EFF0000000000000000000000000000000000011
:10F0000088DCD0FE95E84E705C380AB0AA2845D856
:10F010001388D91C78468C1326F0256C88080404C4
:10F02000E9D40C5B44DDD4CE7C06463BA6265DD8F5
:10F03000705B7C0A556CB03C46BC70C57E256C0488
:10F040004670387C1C0AEDA4563CAA7CEE3BCEFCF4
:10F050001C0A556CDABC06B07C063B86BC065DD843
:10F0600070DA7CE6917AAE4670CE68C1B0E0B07CD2
:10F0700006300B0697300D46DA7C06333017C63E55
:10F080009306301806BBB03C061EA114F87E7E9E87
:10F09000066646F098A6581CB07C26E6CE7C0A048C
:10F0A000EDD098E67CAAFC58CE7C0AEDD098AA5800
:10F0B000CE7C0AD9D0DC101E9E9E1C98AA5804084B
:10F0C00093EDA48A06D91C79B01CCCE746F06A01FE
:10F0D000D0987C6A6F98DE586A8744D91C987E2F36
:10F0E000581EA9763020E805768A48196C4479B014
:10F0F00098DE1EFCDC901E1F5E1BBE5E3C5883ED3E
:10F10000A48A06D91CCC33D9B008357679B01C6AEC
:10F1100046F001D0986A63DE3FFCFE9B0C8BFEDE5E
:10F1200004F3D91C0CE37E9EBEC7F8BEF3A3D91C22
:10F13000B8F8568A063040C64B46F06A196C1B79FF
:10F14000B0980C37FC1E9E3C1E3C9CE2042030F024
:10F15000E6E09CA0443020CC697766E3C666797708
:10F16000E699C8D91C9C6282B8A2F34C1B98F3069E
:10F17000E094339C98A60658A0D88444D84C77C60F
:10F18000A69C58301F6617260698069CE8D09C025D
:10F1900082B8A2F34C5177485576203CF64BA568CF
:10F1A000711C5DC4E01078581A7A7A4E203C5A1CC3
:10F1B0005D001AE000105B504B903BF3D023000041
:10F1C000103C56063044668F788C1B84138884D894
:10F1D000F0A5680C6973517626669FB07C06668C34
:10F1E00023300B4686BC0646F05DD8C97A26667782
:10F1F000B07C0646268C1B300CC653064349247847
:10F20000FC5CEAEE9C300842A17CF6DD7B30088C89
:10F210001F4200957C068C47C1681BC17A7C5898B8
:10F22000A6588CBB796C4A57C1B0BD1C0E0F20127A
:10F230000F0F0DDDAC78D884D8F049246D586100EB
:10F2400030FF66675ACCE3203C0630C366DD7A693E
:10F250007288489806C96C25E8E3CEBC06B07C6687
:10F260002326E6CEFC1C0A04EDD0988D8C0666861B
:10F27000B03C0671D8C97A3008957CE6EFDABC0656
:10F280001C3001667FE6CEFC0AEDD030608D8CB07C
:10F290003C9D7EB07C667766C6E6A658BC065DD807
:10F2A0007C26E633C626E6A658CEFC0A04EDD098A6
:10F2B0003CAA7C58066611F4D3F6278C557B1C06B5
:10F2C000300825400E7E9B9A0507088700D36B3BCC
:10F2D000E3FBEBD323DBB17E75F44670387C0AED9B
:10F2E000A4567626A3617E056C8C1B8413883D761C
:10F2F0006520056C8498F0A568F572796C0AA17B8D
:10F30000B96CB0684829E84670787083BB843BFBD1
:10F31000796C0A5788CEFC0AD9D0B03C26BC70ED77
:10F32000A456768CEBE6556CC6263FAA7C5CCAEEEA
:10F3300083B96CB0FC5CEAC41C59E8056C8498F095
:10F3400046F01B056C8C1B84138898F0C97AB03C7E
:10F35000E6C17A6606265DD8056C8498F0A56869D2
:10F3600072267F556CB03C06265DD80B4666E68853
:10F3700059C804C1B0BD1C07140F201E7E7EC63CB8
:10F3800030033E1B30017EFCE8BEB3DDAC0C3B46D7
:10F39000F0C6E10803A5684E5C10901ACC4F26EB2E
:10F3A00099C8BACB7976300B01ECC3847434857577
:10F3B00035867636370023363636363636363636A6
:10F3C0005B65209300000000E080E006C61C224739
:10F3D0001C8622279C860882CD7EC61C222B1C22DE
:10F3E000DD7B02A29F8C174230555EFC06BC30E0EC
:10F3F000000005CAF3EBE3DBD3CBC303180D14679E
:10F40000308AA630BD8B72201165E34F0B1D10238F
:10F4100050C604A89C60C74C81496A521BF515F37D
:10F4200014124485B60825C6205B15EBA2262A0ACD
:10F43000400C50AD3C362203820F003532388184B7
:10F44000D80400CCC040819010038074D184F5B002
:10F450004DC000A409302333CC5068BB881F88FB03
:10F460000D8C8C84D4CC0035C0A803033C3181863C
:10F4700021F25B38338A1CC3A1362321B22485E8EC
:10F480002ECD8843480C08000638622380C71082BE
:10F49000B02066CDC040FD657EFDF5E6D61831D1C1
:10F4A00018C0A82221727CBCEF43E2F030E363BBBA
:10F4B000EF0C2320EC20ECFF10A2A0802122282AB0
:10F4C0008221C0C3953C412282101102821108CCD6
:10F4D00004002088310089FD0CCF0B1042084991AF
:10F4E0009D3055C3080018E00D7800880350F08166
:10F4F00034242AF102000000000000000000000097
:10F50000C9E0331053FE72482113E20331158A35E6
:10F510001D23C6B0CB28320EF88A423203980C4025
:10F52000102131411204B81BCE392500C520F0044A
:10F5300052D9C408182044D915449146A603153D54
:10F540006D50210009076954011693A150421A4ACF
:10F550001B050452C7AC8EA0418010409A4F5D112C
:10F56000040481004227644114441785A2244348BF
:10F5700061542468441EC98009CD33A1DC50106A4F
:10F58000821041C1B30601194525880333D6404393
:10F59000482331E50800000610D014294304310047
:10F5A000000000000000000000000000000000005B
:10F5B000000000000000000000000000000000004B
:10F5C000000000000000000000000000000000003B
:10F5D000000000000000000000000000000000002B
:10F5E000000000000000000000000000000000001B
:10F5F000000000000000000000000000000000000B
:10F600002134432432A02C3222037A488414111767
:10F61000C54108160E3BD19008DA2308D40C50B827
:10F620000320AAC428201417170E003183AAAE7332
:10F630007F3703F17A18EB40E8C42EE340E044E062
:10F6400088114C2046211420D24F22D41E7F7C8C5E
:10F650003FCF143D4D34004238019D1008E1503237
:10F660000030344E4207C404A89C60C74C81C84097
:10F6700045D3F0D0801231CC44D401412433841BD3
:10F680008E32F62E61200609FD73B40CC10CF38C8A
:10F690002108C44098186081620F848B9EC008279F
:10F6A00008C70FEEC5174060865D2403B731315C93
:10F6B000C744C7CB50005044642384930C32E88C79
:10F6C000683D00088509240A6002040084C0000027
:10F6D000880E841800A3512E4891801E8508048945
:10F6E0004F2F313131B13C1432C3085200000000B9
:10F6F000000000000000000000000000000000000A
:10F700000B801A2838215A84720934015C0504954B
:10F710006824000054180D059034E248C5443411A3
:10F72000140F3113C411249811405844587841C41F
:10F73000084D700CC447E3244571A11991368087A8
:10F74000D0CC54010C8D2B033B0371330F45304655
:10F7500034D6061D20F4E668C8003744C8516C4B07
:10F760004C8C214BDD14E55131D0141E6300C000D8
:10F770004931CDEC56540E954414C339144A34879C
:10F78000064767C5C435C67D44753300E0B41B2306
:10F790002DBC141F595580D10A901110105C9C612A
:10F7A000C4004500148D4105090941465124C9444E
:10F7B0007155591055508296A0968978626E514DB8
:10F7C00085094A4DF5430186E051080816C68CB1FB
:10F7D0009C01B0079E01E6167941C088F20C200515
:10F7E00021A1F70C331654E3D21600000090AAAA08
:10F7F000884077282F3FC5A2474B85F630FF3F88CA
:10F8000000000000010000000200000003000100F1
:10F8100005000100050101000800020109000201C4
:10F82000090102010A0000020B0000030C000004A1
:10F830000D0000050E0000090F00000A0F00000B6C
:10F840000E00000C0F00000C584E5554302000588C
:10F850004E5554312000584E5554322000435846DE
:10F86000554E300054494D45522000435846554EA0
:10F8700031004164764C31200041647655312000DE
:10F88000416476553220004D6174683144005374F0
:10F89000617431420046696E616E63005A656E7232
:10F8A0006F6D0047616D65733100436972637569FF
:10F8B000005374616E6461005050434C20520050FC
:10F8C0005043552052001A1B1B1B1B1B1B1B1B1BD1
:10F8D0001B1B1B1B1B1B1B1B1B1B1B1B1B1B1B1B78
:10F8E0001B1B1B1B19007C204275696C74206279FC
:10F8F0003A204D652120202020202020202020207B
:10F90000202020207C007C20496620666F756E6474
:10F910003A20696E666F4070617865722E6E65740C
:10F92000202020207C00171B1B1B1B1B1B1B1B1BD1
:10F930001B1B1B1B1B1B1B1B1B1B1B1B1B1B1B1B17
:06F940001B1B1B1B18003D
:020000021000EC
:100000001640008F00A60299009E026600950247E6
:1000100003370309031E032602EC02F90451052FDE
:100020000557056A0577050C059104800485048A47
:10003000048F05B104630456045C046A047705A5C3
:10004000059A05D205A005C204E70504051204BE01
:1000500004C904A904DF04D004D7051604B0049E23
:10006000049704B704EF05CA054605290522054F84
:10007000056405710583058A05BA05360608066319
:1000800003B400008220160E0F03201604012DE099
:100090008E091805084830088B8E0914030F300F9D
:1000A000438E090E0902300244E6B83C5804CC1FC6
:1000B0008C2BC4840C5F04C1B0301F682668C668EE
:1000C0001E2B6520610049244E00309D3CFA7EB80D
:1000D0003C98FC6D1C3C587EFA7A6F605B0C2F08D4
:1000E0006B0B133C7A17FCCC8B0C67793C2E3812C7
:1000F000C6C3837711C08070301084743485753521
:100100008676363700E3E323DB53B300C3666666C7
:100110006666666666666666666666661B693CACAB
:100120004CE733FB300A06B34CA7DB5E23793CDE99
:100130002146A3B87CD84C1B441348D83CA8A34CF8
:10014000EF8B4C1B446B485B5E2F6100410EE0D986
:100150001CB8E6F8302006A8B8B856A66617B8A6A8
:10016000E826E8C6E8BE5E2B6D8CDF005D1C3C58BF
:10017000200BE066D91CB8569C5806E223E2E20642
:10018000A2263B66F8693C2403DC904C1B7E7E066D
:100190007E9BFEB806B8300A664623302F0626E856
:1001A0007E3E23C666E8E6E89C98E8EB5E6BD91CC9
:1001B000B8E63020E86606B8B8B8566613F866A602
:1001C000E8E6E84924793CC8B01A5A300CBC1A70E9
:1001D0008DBCF10E8498A8793CDE5D1C1106E0D937
:1001E0001C0EB89CE2337E7E4C137E7E302FE81CC2
:1001F00022A6F8B0E21B62DFA0FCCAF61F226656F8
:100200005ABCBADEFA7EF35AF8B0E2736263601E3B
:100210003009065C422FFAA6E30E6EC1B04924B83D
:100220003CD808D87CA8208CB55188EEE8E04E2058
:100230003C063018BC1AB0303AE62366DF061AE0F6
:1002400097050916180508F8AE6D8CDF8C3008008C
:10025000E66D8CDF3A5C005AD070088DBCF10E97C9
:1002600005091614030FF8AE6D8CDF8CAE0E9C00E2
:10027000E21B8902DCE2E7E2D7E05CA01C4EA202AE
:10028000E2EEEEEE3CBAF2BAA2DCD493300FE669AD
:100290003C51970509160E0902F8AE6D8CDF8C4EA5
:1002A00000BA1A3CFA1B8902E6EFE6DFE05CA01C0C
:1002B000BAF2F2F2BA42421322A2DCD4A33002E62E
:1002C000693C51B8AE6D8CDF8CAE00F06D8CDFE711
:1002D000A600F0EE3004EE465BCE1C58DC9886C3D8
:1002E000EE66F3BC463CE09918140F12793CC370DB
:1002F000793C43B0CBBF140902793CC33CD88C276E
:10030000D8B95AD8655A840E01793C43B0BC463CF2
:10031000BA6D8CDF6C6E008C9102A902920F793C51
:1003200043705B920F18793C4358AEB0D8AEAEB074
:10033000AED870D3940F0EF888AE6D8CDF8CBA00F7
:10034000BA005BF88458B8AE6D8CDF8CAE00D8AEC6
:100350006D8CDF8CD800E00B00A188C1B080B0307C
:10036000063000E6465D003CA6BC300656A87A562C
:10037000D3492408000170ED8A0B00C1020B00B9BB
:100380004A0B0089520B00B5A20B0089020B001921
:100390005A0B00810A0B0009828814010D201604F3
:1003A000012DE08D1614201604012DE00B00A1880C
:1003B00080E00440CC00F3004D50A631F27F3A6952
:1003C000111B1342A631F27F3D85C2032F0270C676
:1003D00000F600534952544EA605C8012F0470C6BA
:1003E00000F400535A3FF653495A453E3DA631A802
:1003F0001997738B9BF37585C8032F0000000000CD
:10040000050E04200F062001121201190E0F1420F0
:10041000011212011920060C0E010D052005121201
:100420000F120E0F20120F0F0D04090D20051212CE
:100430000F120E0F20182D0D050D0F1219150E0499
:1004400005062001121201199812140D201604013C
:100450002DE0AB14010D4EABAD14010D308073AA2D
:1004600014010D30203BAF14010D30A0D8793CD9D8
:10047000038D090414010DF86150753CD6CFAB090A
:100480003016F3AD093056CBAB0A3036A3AD0A3087
:10049000767B810A09130D30053B8A09130D301153
:1004A00058F86150EB8A09120D3013ABAB03130DF2
:1004B000301273AB12130D30323BAB03120D30927E
:1004C00058753CD606AD03120D30D2ABAB12120DEF
:1004D00030B273AD12120D30F23B810A09120D30A9
:1004E00007FB85160F0D0DC4483B900117130DC473
:1004F0008808F86150B80E785150753CD697BF0502
:100500000D010E0D793CDF22BF0D0904793CD62286
:10051000920DC433930DC4608848793CDFD0BF127C
:100520003E12C448C3923E3C12C493833E3C03C473
:10053000085B832B0319B86150C40888F8615075B3
:100540003CE5CE96091008048B820118010D1204B7
:1005500043820118010D030808844884F86150EBB8
:100560008D120E1204338D120E0308846B8D151339
:100570001204338D1513030888448404753CDFF19D
:100580008D1513883B82010D151384843B8D120E4B
:1005900006888844A3820118010D84845B8E090DAE
:1005A000882B98010D8488480804793CDF428D2A05
:1005B0000D793CE56793100E1214793CDF49960ED5
:1005C000090D793CE5259319130D793CE5EA94056D
:1005D000040D793CE58EB030CBB030F6F6366BB01A
:1005E00030F636F63BB030F636F636F61336F613FE
:1005F000363A70DADADA3ABC80E000000000000037
:100600000000000000000D50CA00F6004D454449AE
:1006100054A81B10A5AFCF66A90AA819A5AEAB199F
:10062000B6B2018BA5A8AC0AB6AA87A5BFA5A59BA3
:1006300073AC08B997F27F3FA9178EA5A57179A56C
:10064000AC9A73AC17A5AC0AA596B12A09A8157E79
:10065000BA0BCF6F06AC071DF34D5452A5A4C40CC2
:100660002F1F10C401F700434D45444954A81B07F0
:10067000A906A59283F74E4F542043505868124B59
:10068000638E75691A10101245A806AC06B1874B27
:1006900067B1838EB72701A90A73CF661242111A78
:1006A00010101141A819A5AEAB19D07D8F02AC0A6C
:1006B000D0778FE06683F352452EA5BFA5A59B7327
:1006C000AC08B994F27F3F8EA5ACAC06B98AA5966A
:1006D000A594A5ACA597A59509A815AC087EE03B07
:1006E00083F3494D2EA5BFA594A5A59B73AC08BA6D
:1006F00091F27F3F8EA5B0AC06BB8FA59554A5ADFA
:10070000BB880A7EA596AC06B25D0BAC0AD01A8FE8
:10071000AD06A596AD09A595B26D04A5A8111A1050
:10072000101140124385CF6FCF0FAC071DF34D540E
:1007300052A5A4CA1D2F2150CA00F6004D415452A3
:100740005801A902A81BF5524C2043588ECF68CF00
:1007500069CF6AB114CF67A802CF66F74F524445FC
:10076000523D3F8E616883AC024030511140A6215A
:10077000AB198E2083F152111B1C134240A59DC260
:100780000AF4004D5452CF6F02A908A907A815A872
:100790001BFC2041204920445420422053458EB266
:1007A0001904F152A5A0F44445543D9B737EB22830
:1007B000CF7BA808CF66F152BFB9CF67F152A5A28F
:1007C000B23ACF68AD02B4279F00B244CF6AE02DA1
:1007D000829A73F2522C9B73A5B2B254CF7CF15221
:1007E000AC029F00AD02A5BBB262CF7EA808CF6964
:1007F000E00B820FA807AC02A5BEA5BD03F152A570
:10080000926883511140A63175A819A59DAA198532
:1008100074401140A6218ED0926FC2162F3D30C079
:1008200001F4005A5E4E8030754F205371204271A2
:10083000054E01AC0485A815F2553D9B737EF2561A
:100840003D9B727E85C605F5004D41475A4FA81560
:10085000F2523D9B73AD047E85CC02F400655E5A76
:1008600081554E80B134CC01F4004C4E5A814F502A
:1008700080B141CC01F6005A5E312F4E8030131604
:1008800010714331754F20686053712068437104C3
:10089000E061049700B28185024F71214071B4116B
:1008A000C606F50053494E5A81325A7133E04C8ADC
:1008B00042225923E0518B4280B100CC03F5004322
:1008C0004F535A8132597133E0318A4254225A23AC
:1008D000E0358B4280B100C004F50054414E5A818E
:1008E0001242325A71124233E01D8B4023E00C8ACF
:1008F0007143762259714380B1000B83835871553F
:1009000043715840BD850C558360400D124385C02E
:1009100008F400615E5A7532717450427622421DAD
:10092000F3655E5AC003F5004C4F475A5034758149
:100930004F5024957195727580B100C403F6005A2A
:100940005E312F57327533753151713051402071FE
:100950004354762171432322C204F4005A5E578126
:100960004F504F75754F7175427540744E554E809E
:10097000B100CA03F300432B71067540754074B192
:1009800000C202F300432D547154B613C801F500A0
:1009900043494E56E00482B100034F607154714EDA
:1009A00085C003F300432A4F75754F757571754205
:1009B0007540744EB100C003F300432FE024021DC4
:1009C000F2432ACC012F5B70C600F400504C591240
:1009D00013A621AB198ECF6AF84445475245453DD1
:1009E0003F8E1245D00F6A71121146D0166A71A857
:1009F00000A903A905A9069116911506E04B8C974D
:100A000015B608E0448CCF6FA815A81BFC465820EB
:100A10005254202020204E45578ED0156FCF66A906
:100A200006901691157183838397159096AC059562
:100A30007342E1E18E9073909642AD0571F4463CAD
:100A4000583EE18B8FD0406F0DF1619015A631F3C8
:100A50007F3D3F778E919585CF67A619D0576FC898
:100A600015F40052545312141A11AC069117AC0528
:100A7000BB9390161141911590960C95959715BCC6
:100A8000079500A8050B2036213722382339243A50
:100A90009016121040A819AE73F34E3E358E85CFD6
:100AA0001911101A10101691149115E12E902DE0C5
:100AB000DC842A11E17191E16E91E16B91E1689121
:100AC000CF18289112543827911129911342269159
:100AD0001014424137901214429013514190104229
:100AE0009011514136A900E06397AA038503AA0239
:100AF000B1882D29453D2D2A453D0190133C129585
:100B00000C950D2D51901041661000111B1C1845BD
:100B1000E0358675523F2C2D4290111243416711EA
:100B20008361433E2C519012412D12424052940E4B
:100B3000A800E00287082C2E543E40372D2F543F4A
:100B40004036E02796850771777185CF17181A1000
:100B5000101691149115E08390AC03852DAC00E044
:100B60002C842811E0C191E0BE91CF162754124386
:100B7000838351264166B1A2524039AC00E00E8415
:100B80007476413AAC00E00584A9028505F4524F21
:100B90004F54E03B8F77E02C8D850154523B742BF2
:100BA00054AC00E00586A802850774F155E0208F5B
:100BB00074F156E01A8F74F155E0148F74F156E019
:100BC0000E8F850EAD068591979617917385CF0F81
:100BD000E00E0DF27F3D9B737E85CF10103D268386
:100BE0006167B4D0433E7690956140566811405796
:100BF0001146713C0A1110950C2E543E092D2D2CD6
:100C00002E42403D78858383E00B8E67852E4266B9
:100C1000B916BA200F909540429715BF099095409C
:100C2000901491157585CF119715012D424090951F
:100C30007191958504A803103D27362837E0D41616
:100C4000B300C0452F2320C201F600444946455158
:100C500019A621AB198EA815F54E414D453F8C8E36
:100C60009A07F74F524445523D3F8B8EA901977327
:100C7000A801FB535445502053495A453D3F8E121D
:100C80004331F458303D3F8E32F459303D3F8E337E
:100C9000AC01E02D800A2322E0958135E06B84369B
:100CA000E06784920683402340222183403440E061
:100CB0007E81254026834040134324E05482BA2B92
:100CC00001F559302E3D3F8E340B242322E0608104
:100CD000353021E0498636302120244025E0448506
:100CE0009206834030218340E034862683404025AD
:100CF000401343244034762625401343402183404B
:100D0000354276E00C82BB3F052340222140B29E53
:100D10000392027192038F980298037F8507202423
:100D2000402006124324407442234022744002AE05
:100D300087082142CC212F3A50CA00F3005643A91C
:100D400004CF6FA815A81BFC4450204350200D2051
:100D50004D2055568EA627D0176FCF7EA62DF16455
:100D6000CF14F27F3D9B737ED0286FCF7DA62FCF0F
:100D700068A62CF10DD01614CF6BA62AD03C6FCFED
:100D80007BA629D0068FCF7CA628CF0FAC04D04EEF
:100D90006FCF7FF2583D9B737EF2593D9B727EF27E
:100DA0005A3D9B717ED0656FCC0FF60043524F5376
:100DB0005383CE023042CE022342CE01947171940D
:100DC0000342742042234121744190712241CE712B
:100DD000A62785CF67A623D04E0FCF6DA624D09E21
:100DE0006FC208F300565361686877139474967461
:100DF0000F7591F496740F7591F496740F7591F4C4
:100E0000757585CF6EA625D07E0FCC05F3005652A2
:100E1000686175A627741342134090F3977290F29D
:100E2000977190F185CF66A626F3444F54D0CE1427
:100E3000C605F400444F54214271224240712342BE
:100E40004085CF6AA62BD0BD0FCF69A62B74F14D7C
:100E5000D0F114C005F30056453175327533757500
:100E600085C002F300562D1C11A62EC601F30056B4
:100E70002B920175920275920323222185C802F4F8
:100E800000565859CE0175CE0275CE03757585C8CA
:100E900002F30055564F90714F917077114ECE70FE
:100EA000754E85CC02F300560DA62BA62AA62BA6BE
:100EB000265D85C402F3005644A628A62B7485CA75
:100EC00001F300562A9470947142C8012F2030C05B
:100ED00001F30054521117A621AB198ECF6AA91B3A
:100EE000FA5A302C59302C5830203F8E13A62477D4
:100EF000F5524F540D3F8EA90567B198A805911082
:100F00007311CE71F7632C622C61203F8EA62B12D9
:100F1000A624CF6F01A81BA815A901FC5E4E205E78
:100F20004F202020204E45578EB117CF7DA622CFCF
:100F300066A801A630D008FFCF67A901A630CF7FF1
:100F4000F2583D9B737EF2593D9B727EF25A3D9B57
:100F5000717EB140C013F3004354AD01B38813A6B2
:100F600025A628AD058503AD05B2B611A62412A6A7
:100F700025A6239010AD015459A62E1130A6259018
:100F8000105A9300A62EA62914A62412A62511A64F
:100F900025A6269400A62A20A62E14E00783AC01DD
:100FA00085021304A625A629C00C2F00000000000E
:100FB0000000000000000000000000000000000031
:100FC0000000000000000000000000000000000021
:100FD0000000000000000000000000000000000011
:100FE0000000000000000000000000000000000001
:100FF0000B00D19E000000CBC30000311604011885
:1010000000000000000000000000000000000000E0
:1010100000000000000000000000000000000022AE
:10102000020000C0001800100010F223E3F3C4CE49
:10103000201214C16F3C5888FFE6EF080000000042
:10104000006804545555554D1CF1EC4CE30DC03D62
:1010500006CC23E2CCD14F333B3713F22B3353541E
:101060000D4FAB28CF1D48E80DCEB33713DBCF1C97
:10107000734C456417FC24E2F05112F1F2F2BA28E5
:101080000479EF2FD173C3C4FD7D138C14D5CA63CB
:1010900000004C444C10D705000013542274334018
:1010A0005513ECC10800C0041122DD0C5430B20706
:1010B000234C101304C12CD07530002333008C3C1A
:1010C000C300CC074CD033303F30E7E1B4003341AC
:1010D000220713141335CDD4650D74EC47C9D01015
:1010E000D0109010D01000003000C0348D0110419D
:1010F00041111462000011620010004444512100AB
:1011000001000001000001001000040010000004B4
:10111000000000000C0000014000104F02003301ED
:10112000114410410440001033000400014000103D
:101130004F00C40031400C4008C001C0CB1033093F
:10114000009300D330B0330D70000CC002C02CCC23
:10115000246000800080910C00022000088064134D
:101160000000800060008000024839054C0330090F
:101170003005300530D9744967746618DA6F050098
:101180000080010044111111511151444404515483
:1011900044441145114500116200004411050054FA
:1011A00055014544455114154011111441101011B9
:1011B00011411111111145140444444404454414CF
:1011C00051115104111151045015110144880100AD
:1011D00014110045444444004055541551454045C0
:1011E0000010454404000050141140141111111155
:1011F0001111111144101111111111114111114549
:10120000541545445551106200505555551441141C
:1012100044050014414405005511005445000015D3
:101220005455555541445515010055055541450046
:10123000405541554145004055554105555551557D
:101240005551555500505555000100555544450020
:101250000055555555550140555555551100555595
:1012600004401501004154550540555555110041A4
:1012700040880140441401005441515044444441C9
:10128000441011010000144444544544144414050E
:1012900010044544404511410010101111155144EE
:1012A00044545555114504540440445050411004D1
:1012B00051545154544545455145101551555554B7
:1012C00044454540415545555515551511545555FD
:1012D00015545504101144455041105555155504E9
:1012E00055114405101454554510550445500445F6
:1012F00050514414411015551555545555455455E4
:10130000555541551145454411155115454555054E
:1013100011620000451401501100501111000050DD
:1013200015400550115441414154555550555510E3
:10133000054055055550550551554155555555557F
:101340005510551545514455555555555421064090
:10135000444400000045101111444144440411412B
:1013600044101111441005511005010014151551B8
:1013700054551515514410110440551115511115AE
:10138000554410005554151111450404014055559C
:10139000151144144100545505404400445154056E
:1013A000005114550014451555004444540044544C
:1013B00000441462004444110100404501501411DE
:1013C0001501004511454400000045444404111135
:1013D000411444411401105144544451444445457E
:1013E00014114551444451105511210000000000D2
:1013F00000000000000000000000000034C003E016
:101400001839F738F77FF3A2007B00BC00CAF3CF8E
:10141000F81FF845F859F866F873F8A0F8BBF8D744
:10142000F90FF924F93BF958F972F981F98CF9A10E
:10143000F9B6F9C8FA5FFC470DDE0E280E3F0EB470
:101440000ECF0F5CF3DFFD39FDA8FDE1FE0AFE3093
:10145000FE53FE61FE6BFE7DFE8FFEA3FEB3FEBF5C
:10146000FECFFF540FB7F3AB0B900C350CA40CC19F
:101470000CE40D21000085160C0F1308793C2C6834
:101480004670F87030C070381CD0F0A04E68A8B01C
:10149000E80E4924B8AE4EEED74E9F30C7704E5C72
:1014A000229CD08628E806706048658C015C621B2F
:1014B000A2A230C770AE738705140E0904793C2CC4
:1014C000A8898C00900F0F0C0913CC37793C92C47B
:1014D000E0793C3BEEA038588C4F0C27693C924C8D
:1014E000E733784C270CB3B846FC064924F81E7E37
:1014F0007E37793C92895270A6A687A647A6B7A6E2
:10150000BF898C5DEE3B0E658C32EE2F58658C21C9
:1015100070658C3A898CC5898C50793C92793C1ADB
:10152000120503151213090F0E898C881E7EF87E92
:1015300023B87E37793C92895244793C3BEEA338FC
:10154000580C270C63AB8C9F884844CC13488843C5
:10155000084404CC13080898F04670B87C588C876F
:1015600088983CA86D8C9F580C1F04138498F04CED
:10157000471348300B0C1F301E06793C65E6534C70
:10158000C36D8C9F580C174B793C92793C1A0E0F07
:1015900020120F0F0D898C884E58793CD36AF3DCEA
:1015A000901E1C793CE5E698E6D63C58BEB31C98E4
:1015B000EA1F3CEB58681598EE1B4C33793C92813E
:1015C0000A5C420A0C23AA62231C29A430C3704E71
:1015D0005CAAF04D9CCC67B8584C474EE8380E0AD0
:1015E000AE28B80A30C370387CAABCF04E705C10CC
:1015F0009050105090105050D058681598EE1B4CD9
:1016000023693CBCC80C17C40E1C1DA4BD8C4D9C8A
:101610000E30C37038BCAA7CF0E0A18888C1B0BD90
:101620001EBA60A67066A638E67066E6F0A3BA60D9
:10163000A67026A638E67026E6F0A3E0DCA0467089
:1016400078E630C0067026CB38EEB33E8F7E5C1253
:10165000DC90905C726B5E725BFC560643A6262B98
:101660004EE0E026E046704EA668793C3BEE43A68D
:101670000670264338EE2BFC5606B3668646707815
:101680003CC6BC68860630C070383C1CCA60164632
:10169000A0A6262746E02B66E6C60A3C0A7CF03662
:1016A0006630C1464670783CA6C6A65ABC1A783C3D
:1016B000066626A666A6793C21A6E066866D8C9F06
:1016C0003E13664670783CC6BC682626C61B46E0BC
:1016D00030C00670383E23A626CB30C01E7EC646DC
:1016E0001F661E46707826467CA63C66683C06A6A9
:1016F0008630BF46BC265E1726463C5ABC1A667921
:101700003C21467078E67C0630C0704EDC9090FC40
:10171000A6B606167CE6F67CF04E68A830C00666D3
:1017200070383E274E7EF04626E0044460793C3B0C
:10173000EEA038588C13488CE30C8B084C3F0448BF
:1017400098F0B833844498F07858FB7858C44C1318
:10175000C88CBF6B0C1F4EE0B858C40C13C80C5794
:101760004670B87C5884983CA84670987C1CEAA0C7
:101770000E6D8CBAB858259E4924B0E888793C2A69
:101780000C27793C954C534924B87C588C1F450252
:10179000C502793C2A793C3BEEA0A6067026433868
:1017A000EE2BFC5606B38630C00670383C56062633
:1017B0000670385CEA273E1366A6066686A65ABC03
:1017C0001A6630C0E6793C2E662643A67026064E81
:1017D000F0C3E04E1C909C101C0AE5A456E6603055
:1017E00005426ABFE01CEDA43C3005426A1F1E1B87
:1017F00059A47CE000000000000000000000000090
:101800004408918C6B30C170385CEA1CBC0A46708D
:10181000793CBA5C6AC44213C81CBD8C4C091FC118
:1018200002793C95F858793CAB6BB058793C9558A7
:10183000793CAB793CA2F0418C78793CA8EE2769E1
:101840003CA10EB05EFE23693CAF1EA0BE1D6160D0
:10185000FE1FEE27693CF3793CA5EE63793C9F1CA3
:1018600002D0761613B6F0793CA86838E8F828B0AC
:10187000A8B80E793CB53A356060793C1D793CF2E8
:10188000EE9B793C6A0E793C1A793CB52626BE253A
:101890006160FE574E5C2226260E793C1A793C99EF
:1018A0000E38AEA0BE1D6160793C1D793C79793C53
:1018B000A2A0256060793C1D793C56D85EFE6B790C
:1018C0003C52A04E3E6EA03D60A5500E60793CFD9E
:1018D000EE9F793C56793CA2A02560A550600E7918
:1018E0003CFDEEFBF8700648693C00793C524E5CCA
:1018F000223AA3793CA5EE37B068693C71793C9FE8
:10190000F627693C6A76F0793CE7793C1DB00E79A0
:101910003CA8A0BE1D6160793C52A04D6060793C3E
:101920001D793CF2793C1D793CEC793C06A0BE1E49
:1019300060793CE3793C81793C990EF8AEA0BE1DFC
:101940006160793C063ECE63793C0EA0BE1E607994
:101950003CDF23793C5A793C87EE67793C5A793CE5
:1019600087EE27F8E82BF84EEED7793CA858793C5B
:101970009558793CAB793CA2F04670B0E8498C2A86
:101980000C27498C95B95AA04E5C66503D6030C812
:1019900070382560A5500E30C770AEE80E384E6026
:1019A000E0B0A84E68793C99E8064870693C00B8F8
:1019B00068380E793C99AEE884B0A8F8280E793CD6
:1019C00099A0BE1D6160793C1D793CA50EB8A0614F
:1019D000604E5C223ABE256160793C060E793CA2DD
:1019E000A01D60A5500E60793CFDEE87793CEC7936
:1019F0003CA2A05CFA37BEB626228B5E37FE373A91
:101A00005BBBFEE762FA1B2213667A00A5500E60EC
:101A1000793C99AEE84EEE27693C2A7870F80E7949
:101A20003C994EEE27B08C53AE0E06664870693C6A
:101A3000000E793CA85EFE23693CAFA0B8AE6160A1
:101A4000096060793C1D793C990EF8A0BE1D61606B
:101A5000793C52A0496060793C1D793CE7793C6A49
:101A60000E793CB5BE1D610E60793C99AE680E7969
:101A70003CD3BE1D6160FE9B793CA55E680E793C3F
:101A8000D31D6060793C1D793CA50E793CB51D6085
:101A900060793C06793C1D793CD386BE2561FE7396
:101AA00060793C52B0A0BE3D61BB793CA50E793C4B
:101AB000D386BE1D61FEBB30C970380EB0BE356125
:101AC000A5500E60793C99AE6888693CB9B026266D
:101AD00026BE77793CB5666666E0A0316060E07945
:101AE0003C5AC3793C56A3793C99F823793C990E2A
:101AF0003833793CA50EB8A0BE1D6160E0793C99F1
:101B0000AE0EE8384EE0793C52A0756060E0793C5A
:101B100056C3793C352B793C52E32E7A0B30C0709A
:101B20003868F828CEBE1EE8B8BA9CEAEAEABAA835
:101B3000AA8A8A8AE330C070EED8B81A9ABABABABA
:101B40001CEAE6A8F8EE38E87828BA463CFED8EE5B
:101B50005CE030C39C4330C41C2330C59C7038EE1D
:101B6000D8B8D4CE14EBFEAED83B793C52A0756009
:101B7000A55060E0AE0E58CE23793C56A049606077
:101B8000E030C070B83CA6BCA830C37038BE5CEA78
:101B9000F0E07038E0793CAB0E30C7BB30D0A330FA
:101BA000C08B30C87330C95B30CA434E707828B8D8
:101BB0006898A85CE04E5C22A0E01C38AAFC0EF8F5
:101BC000FCAAE8AE28E0B0A0FA274626765C5A5E6A
:101BD00050EE4670B87C0E9CA2467C60E6E6A0AE55
:101BE0001C2666E21B4213A6B67FB66F58860646D1
:101BF000B6504626561B26986E466030D070E000E0
:101C00004924F870B80E30D0704EF0F0586D8CAB9F
:101C1000AE5830C07098E8A0BE1D616030D0704EE4
:101C200028E8DA2F58693C3E793C5B30C070F825D3
:101C300060706006481344666630D07038F0EE5825
:101C40004670B028EE7004793C6B30C270658C0829
:101C50006D8CC6AE68F8F0E80666693C506D8CC6BF
:101C600078A01D6068B80EB86160AE0E58CE4960AD
:101C700009604EBE50503D60606D8C1D30D0707854
:101C8000A03D6030C070B82560A830D070F80E302C
:101C9000C07038F01D6060793C55B0FED830DE7001
:101CA00038FED83160606D8C1D30DE7038A6F07E55
:101CB00030C070CE284E900E30D070B8A01D60A8F5
:101CC0000E60693C0A30D0704EE86D8CC6B068304A
:101CD000C070AE6830D0705C4E90A830DE70385E58
:101CE00046F030C0704E28A830D070F80E78A01D95
:101CF000602830C070F80E30D07038AEBE1D61382C
:101D00003D60A550F05C4E22A80EA0B8AEBE1D618D
:101D1000FE2B60693C55B86960AE0E58CE4960E84C
:101D2000B80E1D60B82560F83D60B869604E6690D9
:101D3000503D607030C070F80E60793C62B03D601C
:101D4000700E30C070F81D60F00E60793C62E806DD
:101D50006660693C36B80EA0BE35612830C070B8E8
:101D60000E30D070B86160F030C070780E30D07036
:101D700038616030C07078BE2561B0256060793C04
:101D80005B78256068606D8C5230D070F870B8A0B8
:101D9000696078BE2561B02560606D8C1D30D070A3
:101DA000780EF0A01D60386960606D8C35A03160E0
:101DB00060793C5BF02560606D8C1D30C070787080
:101DC00030D070B8A0FA23DA50260EA8356009602A
:101DD00058606D8C95B0AEA06160B0256068EE462D
:101DE00070B80E78A846703868EE2E7A606D8C0652
:101DF0006D8C52A03160709E30C070CE2830DE7085
:101E000038A606F0B0BE256158380E30C070AEA8B6
:101E100030D07098E8780EB0AEBE1D6128B06888EA
:101E2000084E6830C070B84AFC0E4E1C50A8901C7A
:101E3000029C48021BAE44F08C1F04138430D07007
:101E4000780E4E5C10A035604ED0256068F80E30DC
:101E500007E66030C070B8AE26AE7038A0BE1D6117
:101E6000382560A830C070780EE0DCA01CF2525E0D
:101E70001B669230D070B85EBE1D61FE7384083060
:101E800007E66030C070B80EB09C02EB26AE70AEB4
:101E900038A0BEAE60267038A01D60783D60B8697D
:101EA000604E90BE2561FE1B88083007E66030D08A
:101EB00070F80E30C070B8A626A670AEF0B80E78D6
:101EC000A06160F82560E83007E6C66030C070B8F1
:101ED0000E0C33B0AE9C22A80227693C38B80E4CD9
:101EE0005730D070F826AE70AEF030DE7038A03EBD
:101EF000137E46F060693CE2F858606D8C9530D0F6
:101F00007038586D8CABAEA0BE1D6130D07078704B
:101F1000F858606D8C81980EB0A01D6060793C55BA
:101F200070606D8C521E30C07078A03D60B0FA4376
:101F30005A5E5066D414EB2560A550F05C58606D75
:101F40008CABB0A0A550F060D44B30C07038D888AE
:101F5000D8F0418C786D8C52A049624EA05C6650DE
:101F60003D6230D07038AEA0BE1D636630C10C1724
:101F7000267038FC9CA2023CF0A0B0A550584670D8
:101F800098F068A8E87060E0DDAC0170ED8A5470EC
:101F9000C600F40054564D1110A621AB198EA900AD
:101FA000CF7F773132333435D00BEF0FA815F27F66
:101FB0003D9B737ECF6FA81BA916FF204E2C204996
:101FC0002C2050562C504D542C46F27F568ED01B50
:101FD0006FCF7B111242CF66F14E31AB16A634BFE4
:101FE00036CF7C111243CF67F14932AB16A638BF0A
:101FF00046CF68F2505633AB16A635BF52CF69F3C1
:10200000504D5434AB16A636BF5FCF6AF2465635F4
:10201000AB16A637BF6BCF7EA815F3454E44AB0079
:10202000A800AC00F5424547494EF67F204D4F448D
:10203000457ED07F6FC817F2004E2267B49B111BFC
:10204000124336E02F8864BBA32864B29705F624B8
:102050004552524F528ED0A36F042325402467B5BA
:102060001443B18402E0068A015431850B6526656C
:1020700043318509E0118938E00D8939850CAC00C0
:1020800011AD001042850A2383CE05334026543615
:1020900061E0150B114024422623424067B55243AC
:1020A00026425485CC0FF30050562267B189E05484
:1020B0008727254226B2830125210224424054333A
:1020C00085C204F400504D542267B18BE036872757
:1020D0002542234026B28501232540210267B50011
:1020E00043543485C005F30046562267B18BE01493
:1020F00087244223402743B2860124214223400201
:102100005435850822111B124365214254553776F8
:10211000585422111B12434376E09D0B1140423666
:1021200085CA08F3002A492124422340254067320A
:102130006785A9052324E0BA0B403676244154254F
:1021400040374264B500211178B1842463B2900114
:1021500026274267B50027264354216053B3BB02AC
:10216000216011403226244266E065850D2250210F
:10217000425822114167B18343B2820121023811D2
:102180004124422221532642403921284122114133
:1021900067B18D4322422442B28E0311714D3285C4
:1021A0000121112141421243022921424029714358
:1021B0002754294371532242767132714D61111BAC
:1021C0001C1646BD59AC05E00785A90522B33506A6
:1021D000A80522603227CE0637C41A2F4270C600E7
:1021E000F50043464954A815A81B1118A621AB19A0
:1021F0008ED016E8CF6F2BFC207E2B2020434C7E08
:10220000204649548ED0126FCF689900709906709D
:10221000990C70D0206FCF66A61CCF67CF69D02BEA
:102220006FCF7BA61DD0326FC80AF300417E719933
:1022300006917447E021804774920574920485C426
:1022400003F300447E719906917448E00A80487453
:10225000930574930485017576507176715071768B
:1022600094705071947150990C85CF6A2B11415024
:102270000C2BA901A902A903A904A807FC4C20451D
:1022800058204C4F47205020428ED0976FCF6AA6DF
:102290001ED0E7E2CF6611A61FD0DFE2CF6712A6FD
:1022A0001FD0D7E2CF6813A61FD0CFE2CF6914A604
:1022B0001FD0C7E2CA10F500424649547733A980BF
:1022C000A907E01A81E02882E03683E0448420CC2C
:1022D00003F40046495430A880A807AE0002273214
:1022E000292A2628E0408511F34C494EBFB2032D20
:1022F0003229252C28E02F8512F3455850BFA10420
:1023000027322F24262EE01E8513F34C4F47BF9013
:10231000052D322F90102C2EE00C8514F3504F57C2
:102320000FAA0630850631719111422B434171216C
:10233000512B4341434276CE029011512B434143EE
:10234000AC07B78623714685A80607339011212272
:1023500042412B43AC0255AC04553185C214F40004
:10236000593F5821229071AE00045002424085032B
:10237000425542850571534285CF62307EF2613D00
:102380009B017EF2623D9B027EF4525E323D9B03D6
:102390007ECF0FF3583D3FA9168EAD16BC00A62088
:1023A000F2593D9B737ED0160FC00B2F000000002A
:1023B00000000000900901F86150F6134E88ED64AA
:1023C000DC86D058143B2B00E080E0DC58E051B4B0
:1023D000A09866A66BE000CCC75878AE30C070AE4F
:1023E0000663387C0630EE1C6A27498C955D1C9884
:1023F000CD9E0B800000E313FBCB0032160401B826
:1024000020020020222222222222222222222222F2
:1024100022222222222222222200222222004013D1
:102420000821A22815A04CC89E0A3A141532004D66
:102430000C0020B38FCE023303305840330F454495
:102440000CD2280D0CC3308F0000CEC430F3381AE4
:1024500007A89204A0F8E22DDEF331AC6144348A7F
:10246000CCA7F30800CE348FC54C607DE23922F34F
:1024700040523021E0C8034E6C2182685764E488E2
:102480004C08313085803ECD340A28DE28A03882C1
:1024900013398878FEC380E33C23381A390838A101
:1024A0009014D2CD375CA02244280425513432CD7B
:1024B000120AA9C191081ED4046A9152843906C532
:1024C0008852213E104302A122289E8ECEA34000B6
:1024D0000BB2041902C0A438787B63E2CD0F01CDA2
:1024E000314BDC32338F4E0E024E24A1C9221141F2
:1024F000118C0C1A3EB42478F0230603F30000007C
:1025000036870084333000CECC364373F3CC3CCBDB
:1025100014CA848222C32CB3D1E0AC29DA6C388F80
:102520003237CF2A28AC36CF8982F33C0BCE73DA10
:102530002C6A408E32CF02D82802C3CCEA2C38CC89
:1025400032E938D3ACE0AC388FF3386B8EF39C288B
:102550003823B3E6C83CC93C89A1363737CF20CCF5
:1025600031836C11025048A923CE0283DA4CA03685
:102570002B38CFA9B00ACECD02E468E3EC82CA883A
:10258000EC8A2890332A83D8AC004430342B932231
:10259000E03CA782B3E13CCECD42CED828683336AA
:1025A00082F3DC0CCEF3A860CE6830372A48481896
:1025B000903332A1FAAC2EF8FCFC2C7332A782CFF8
:1025C000A43E2B3E3F3B0F844510D14FFC8454FC6E
:1025D000411005101F101109F50E3D2BE014CC869B
:1025E000874185302ECFC5711CC73102C4B3CE9050
:1025F000208F820E81C3B025AB8011195A436438F5
:10260000011482CD14B6822121CD73382062854118
:1026100048D01C0E330034CD081442118014CE2152
:1026200046381C5238E00C8510388720214361421F
:1026300039853453C8E1400818F22125145E084258
:10264000018E2508E28450040401812005E139133C
:10265000140EE40C399046E18508E18549B800384C
:102660000F3B8781920038878590380BCE80733876
:1026700021C618013983020C122000CEB300218735
:10268000900851C8611408914138C6DFDD101286E8
